:020000040800F2
:1000000000090020B1010008592A0008F52900085C
:10001000352A0008F5290008152A0008B301000850
:10002000B3010008B3010008B3010008313E000825
:10003000B3010008B3010008B3010008B3010008D0
:10004000B3010008B3010008B3010008B3010008C0
:10005000B3010008B30100087D4C0008A54C00085E
:10006000CD4C0008F54C00081D4D0008B3010008F8
:10007000B3010008B3010008B3010008B301000890
:10008000B3010008B3010008B3010008F928000813
:100090000929000819290008B3010008454D000886
:1000A000B3010008B3010008B3010008B301000860
:1000B000414E0008B3010008B3010008B301000875
:1000C000B3010008B3010008B3010008B301000840
:1000D000B3010008B3010008B3010008B301000830
:1000E000B94D0008B3010008B3010008B3010008CE
:1000F000B3010008B3010008B3010008B301000810
:10010000B3010008B3010008B3010008B3010008FF
:10011000B3010008B3010008B3010008B3010008EF
:10012000B3010008B3010008B3010008B3010008DF
:10013000B3010008B3010008B3010008B3010008CF
:10014000B3010008B3010008B3010008B3010008BF
:10015000B3010008B3010008B3010008B3010008AF
:10016000B3010008B3010008B3010008B30100089F
:10017000B3010008B3010008B3010008B30100088F
:10018000B3010008B3010008B3010008B30100087F
:10019000B3010008B3010008B3010008B30100086F
:1001A00049110008000000000000000000000000ED
:1001B00002E000F000F8FEE772B6374880F30888E6
:1001C000364880F3098836483649086040F2000016
:1001D000CCF200004EF63471CEF200010860BFF39D
:1001E0004F8FBFF36F8F40F20000C0F2F0004EF669
:1001F0008851CEF200010860BFF34F8FBFF36F8FBD
:100200004FF00000E1EE100A4EF63C71CEF2000114
:100210000860062080F31488BFF36F8F04F026FB7C
:1002200004F0E4FB4FF055301F491B4A91423CBF9C
:1002300041F8040BFAE71D49184A91423CBF41F8C6
:10024000040BFAE71A491B4A1B4B9A423EBF51F86E
:10025000040B42F8040BF8E700201849184A9142B1
:100260003CBF41F8040BFAE704F004FB04F0C4FBC4
:10027000144C154DAC4203DA54F8041B8847F9E7D7
:1002800000F042F8114C124DAC4203DA54F8041B52
:100290008847F9E704F0ECBA0009002000110020BB
:1002A0000000000808ED00E0000100200009002027
:1002B000E0500008001100206811002068110020A3
:1002C000283B0020A0010008A4010008A4010008A8
:1002D000A40100082DE9F04F2DED108AC1F80CD0D3
:1002E000C3689D46BDEC108ABDE8F08F002383F300
:1002F00011882846A047002003F01CFFFEE703F00A
:10030000A1FE00DFFEE70000F8B500F021FF04F0D9
:100310004BFA064604F0A0FA0746A8B92B4B9E42BA
:100320002AD001339E422AD026F0FF02284B9A425F
:1003300003D005464FF47A7408E0F0B200F018FEDE
:100340003D4642F2107401E00546002400F016FE1E
:1003500008B10024254601F097FB98B9B4F57A7FDF
:1003600016D017B11B4B9E4214D1002004F028FA7E
:10037000ADB900F03DFE24E005460024E6E7002488
:100380000125E3E7032000F02FF800242546E8E7E5
:100390000125E6E704F058FA00242546E5E700F0D9
:1003A00041F8E6E700F074FE4FF47A7003F0CAFEFD
:1003B000002CF7D002F058FB401BA042F2D900F00D
:1003C00031F802F051FB0546F2E700BF010007B02B
:1003D000000008B0263A09B0302383F3118885461F
:1003E00080F308880847704708B50C4B187003283D
:1003F00006D8DFE800F00A06020E022000F00CFF2B
:1004000008BD022000F006FFFAE7054B00225A6003
:10041000F6E7034B00225A60F2E700BF701100209C
:100420006811002008B501F02FFB034668B9072BBF
:100430000FD89A0002F1006202F520421268B2F170
:10044000FF3F05D00133DBB2F1E70320FFF7CCFF1C
:1004500008BD1A4B5A689A42FAD3194B9B6803F1AC
:10046000006303F520439A42F2D204F0BFF904F08E
:10047000D1F9002000F088FE0220FFF7B5FF114BF4
:100480009A6D00229A65996F9A67996FD96DDA65AE
:10049000D96FDA67D96F196E1A66D3F88010C3F86E
:1004A0008020D3F8803072B6044B4FF0E022C2F8BF
:1004B000083D59681868FFF78FFFC9E700A00008DA
:1004C0000011002000100240BFF34F8F0549CA6899
:1004D00002F4E062044B1343CB60BFF34F8F00BFC5
:1004E000FDE700BF00ED00E00400FA05094A1368CB
:1004F00099B21B0C49F2690000FB01331360064BF3
:10050000186882B2000C44F2506101FB02001860CE
:1005100080B27047141100201011002010B504465D
:10052000FFF7E4FFB0FBF4F304FB130080B210BD4F
:1005300070B50E4614461D4602F09CFF60B9022DB0
:1005400033D1012C01D0002030E019A3D3E90023DE
:10055000C6E90023012029E0282C1FD00CD8012C4B
:1005600015D0052C06D114A3D3E90023C6E9002336
:1005700001201BE0002019E0302C06D110A3D3E9A4
:100580000023C6E90023012010E000200EE00EA3A6
:10059000D3E90023C6E90023012007E00CA3D3E937
:1005A0000023C6E90023012000E0002070BD00BF49
:1005B000401DA12026812A0BF017304A39059E568E
:1005C00078F6339F93CACD8D9E6AC421818A46EE08
:1005D00026417272DF25D7B710B4034600220260AD
:1005E00042608260C260044C07CC186059609A6017
:1005F0005DF8044B704700BF9075FF1F70B58AB05F
:1006000006460D4602F030FA04464FF4C870FFF774
:1006100085FF044404F51674184B1C60EB7E23B967
:10062000174B00221A700AB070BD05A9284600F0C9
:10063000E7FF0028F7D101A8FFF7CEFF9DF816408D
:10064000224601A90DF1170004F052FC48B90F2C05
:100650000BD80B4B1C70094A1368A3F51673136073
:10066000E1E7074B00221A70DDE79DF8141000291E
:10067000D9D0304602F0F6FED5E700BFB016002014
:10068000AC1600202DE9F041ADF54E7D07460E4633
:100690000CAC4FF4C4720021204600F0D3FD02F0F0
:1006A000E3F9304BA3FB00239B092F4A136007CAD1
:1006B00084E80700022323744FF0000884F81180B7
:1006C0000DF15200FFF788FF052384F820307F23C7
:1006D00084F821300DF1180C244D0FCDACE80F003B
:1006E00095E803008CE80300172384F832310DF1FC
:1006F000180CBCE80F00CDF86301CDF86711CDF8F8
:100700006B21CDF86F31DCF80000CDF87301BCF837
:1007100004209CF80630ADF877218DF879316FAD63
:1007200001222946204600F0CDFE80B205900495B6
:10073000CDF80C80B37E029306F1190301930123D7
:10074000009306A3D3E90023F17E384602F046FF6A
:100750000DF54E7DBDE8F081AFF300809E6AC421A7
:10076000818A46EED34D6210B4160020704F000807
:10077000F0B5FDB006460D462B4B1C7A6CBB07A9A5
:10078000284600F0A9FF002845D19DF81D70C82F0C
:1007900041D84FF4A6620021234800F053FD09E040
:1007A0002202214B4FF48A7101FB0433C3F8E42089
:1007B0000134E4B2032CF3D91C4C3A460DF11E016E
:1007C000204600F02BFD093CE219002353729DF8EE
:1007D0001C3023720BB9EA7E2272812200213AA8D2
:1007E00000F030FD5BAC012221463AA800F0CEFFBC
:1007F00080B20590049400230393AB7E029305F12D
:10080000190301932823009305A3D3E90023E97E6C
:10081000304602F0E3FE7DB0F0BD00BFAFF30080D4
:1008200026417272DF25D7B77C1100208511002088
:10083000134BB3F82C35834200D9704710B50446EA
:10084000002100F0CBFC01340D4BA3F82C450C4BE0
:10085000B3F82C0500F0A6FC88B1094BB3F82C05C1
:1008600000F0B2FC58B9064C0021B4F82C0500F099
:10087000B5FCB4F82C350133A4F82C35E7E710BDEE
:100880007C1100202DE9F041F0B00646274C94F889
:10089000D8304FF48A7505FB004585F8DC30002719
:1008A00085F8E870D82239463AA800F0CBFC04F16C
:1008B0000908404600F0BCFC8DF8F000D5F8E430A3
:1008C0003A933B97C2B241460DF1F10000F0A6FC0D
:1008D00006AD012229463AA800F0AEFF80B205908D
:1008E0000495012303930823029304F1D803019391
:1008F000302300930BA3D3E90023217A0C4802F0A4
:100900006DFEB84203DC002070B0BDE8F08102F05B
:10091000ABF84FF48A7202FB0643C3F8E0000120F3
:10092000F2E700BF78F6339F93CACD8D7C1100208B
:10093000B437002038B502F097F80546002408E0E7
:100940000532B3EB420F02D3FFF79CFFF8B101343D
:10095000E4B2032C1BD80E4B93F8D900204400F0CE
:1009600003004FF48A7202FB003393F8E830002B47
:10097000EDD1074B02FB0033D3F8E030002BE3D07E
:10098000EB1A034A1268F92ADAD8FA22D8E738BDF6
:100990007C11002010B586B0BDF828400494099C55
:1009A00003949DF8204002940193009202460B4666
:1009B000024802F0B3FD06B010BD00BFB4370020FE
:1009C00010B58AB0244802F055FD08B10AB010BD38
:1009D00002F04AF8214B1B689842F7D302F044F822
:1009E00004464FF4C870FFF799FD044404F51674EB
:1009F0001A4B1C6000238DF82030194B1B7813B95B
:100A000001238DF8203004A8FFF7E6FD144B197878
:100A1000C1F11004E4B2062C00D90624224604AB2E
:100A200019440DF1210000F0F9FB0134029408ABE8
:100A30000193182300930B4B012205A1D1E900017A
:100A4000FFF7A8FF064B00221A70BFE7AFF3008044
:100A5000401DA12026812A0BB4370020B0160020AB
:100A6000AC160020C016002010B586B001F0FCFFC7
:100A70000F4BA3FB00239B090E48036004AC01222B
:100A8000214600F065FD80B2029001941823009386
:100A9000094B40F2551204A1D1E90001FFF77AFF9A
:100AA00006B010BDAFF30080F1C6A7C1D068080F33
:100AB000D34D6210B41600207811002010B5024604
:100AC0000B46094C204602F0C1FD204602F0D2FC44
:100AD00038B1064B1B7A2BB10322054B5A71FFF735
:100AE000C3FF10BD0222F8E7B43700207C110020BC
:100AF000B416002038B50025084C002D05DA084A48
:100B00000849002004F0DEF938BD204601F062FA01
:100B1000013D04F587540834EFE700BFC8160020F4
:100B20001C38002025110008002202600273427365
:100B300042608260704700BFF0B587B0234802F082
:100B400079FD044600283AD002A8FFF7EDFF237B89
:100B50008DF8143003AB6068A16803C3236843F0C9
:100B600000430293002425463CB10DB3174802F020
:100B700065FD174B00221A70E0E741F2E80304FB21
:100B800003F3144A9E18D3581F6901F071FF124AEB
:100B900082184FF00003009341F1000302A9304690
:100BA000B8470028C8BF45F001050134E4B2DBE7CF
:100BB000074B1B78072B04D80133054A137007B085
:100BC000F0BD024802F03AFDF9E700BFB43700205B
:100BD00079110020C816002040420F00CA7EA04BA9
:100BE0001B7A9A4240F03B812DE9F04700AF08465E
:100BF0000024032C0CD89A4B4FF48A7202FB043366
:100C000093F8DC20437E9A4211D00134E4B2F0E73D
:100C1000002373B9924B1B68FA3340F6B832934203
:100C200000D913468E4A1360BD46BDE8F087012304
:100C3000EFE74FF48A7104FB01F1E031884B19446E
:100C40000A3100F04BFE0028EED1854B4FF48A723A
:100C500002FB0434012384F8E83001F005FFD4F8E6
:100C6000E030C31A192B05D940F6B832934202D9A5
:100C7000134600E019237A4AD2ED007AF8EE677A3B
:100C80009FED787A27EE877A07EE903AF8EE677A4A
:100C9000DFED756A67EEA67A77EE277AFCEEE77AE3
:100CA000C2ED007A3CE013464FF48A7202FB053332
:100CB000002283F8E820C3F8E020C546684B5B6853
:100CC0009B0A0133694A1381AEE7002042F8040B06
:100CD000013B002BF9DA2246304600F09FFA604BC8
:100CE0005B68002B4BD05E4B93F8D20000F05AFAB1
:100CF0008246002847D05A4BD3F8D430002B4ED030
:100D0000574BD3F8D430234453454ED85FFA89F279
:100D10003146534B586800F09FFA00284CD1C54625
:100D20004F4B93F8D9504FF48A7202FB053393F876
:100D3000E830002BC2D0E846494A4FF48A7303FBDF
:100D40000523D3F8E41053689942ACD1444B4FF4D7
:100D50008A7105FB01F15A18B2F8EC40E21C4FEA27
:100D60009209E03119440E314A4609F1FF339200ED
:100D70000732D208A8EBC20295466E46A9E70120C9
:100D800000F002FAAFE70024354B1C7200F030FA95
:100D9000204600F0F9F9354B0B221A818DE7304BD4
:100DA00093F8D200FFF744FDAAE72D4B93F8D20049
:100DB0000130FFF73DFDA9E7294B5A6822445A60EC
:100DC000D3F8D4602644C3F8D46093F8D20000F07E
:100DD000E9F986420BD3224B93F8D220013283F8F3
:100DE000D220D3F8D420A2EB0A02C3F8D420FF2CDF
:100DF00023D91B4C4FF48A7303FB0543002283F86D
:100E0000E820C3F8E020D3F8E42002F58062C3F8BC
:100E1000E42094F8D900FFF735FDFFF78DFE94F834
:100E2000D93001335A4203F0030302F0030258BFE2
:100E3000534284F8D930C54672E70024084B1C722F
:100E400000F0D6F9204600F09FF900F01DFE074A99
:100E5000108108B1C546E7E6FFF7E4FAFAE7704704
:100E60007C1100206666663FCDCCCC3DB4160020D8
:100E700038B505460C4602F0FDFA50B1E38A282B3E
:100E80001ED016D8012B10D121462846FFF7FAFBB9
:100E900002E0237E022B00D038BDE38A012BFBD178
:100EA00021462846FFF7AAFBF6E7052BF4D1FFF70A
:100EB0000BFB302BF0D121462846FFF78FFEEBE7E6
:100EC00021462846FFF754FCE6E700BFF0B58FB097
:100ED0000AA8FFF729FE002426461CB1002EFAD1ED
:100EE0000FB0F0BD01238DF80C3000238DF80D30CC
:100EF00041F2E80204FB02F21B4955188A5800200F
:100F00000021CDE9000197680DF10D0203A92846E3
:100F1000B8479DF80C7027B30023069307930893F6
:100F2000099341F2E80304FB03F30F4AD3585E69C7
:100F30000DF10E0304AA0AA92846B04707AB0BAA75
:100F400092E8030083E803009DF834308DF82430E4
:100F50000A9B0693DDE9042306A9044802F040FD3C
:100F60003E460134E4B2B8E7C8160020B43700208A
:100F7000014B1870704700BFB02700204FF000539E
:100F80001A68184B9A4201D0002070474FF0005366
:100F9000587D08B90020704710B5FFF7E9FF4FF002
:100FA00000531A7D104B1A720023032B0AD8190222
:100FB0000D4A4FF48A7000FB0322C2F8E41001339B
:100FC000DBB2F2E74FF00054C92204F116010748E2
:100FD00000F024F9E0220021204600F033F901203E
:100FE00010BD00BF9AAD44C57C11002085110020C2
:100FF00030B583B000F048FD1C4B188102225A71B5
:1010000000240CB300230193194B0093194B4FF4A8
:1010100080521949194802F009FA194B197809BB8D
:1010200001F022FD04464FF4C870FFF777FA04443C
:1010300004F51674134B1C6003F00EFC10B10B4B3F
:101040000F221A8103B030BD41F2E80304FB03F321
:101050000D48C258556801220C491844A84701346C
:10106000E4B2CEE7054802F0FDF9D9E7B416002056
:1010700031050008710E0008B4270020B4370020A5
:10108000B0270020B0160020C816002040420F00F4
:1010900008B50CE0114B186001F0EAFCFFF70EFDFB
:1010A00013E0C82003F04EF80D4B1B7AA3B1FFF7F5
:1010B00043FDFFF70BFFFFF783FC01F0D5FC074B67
:1010C0001B68C31AB3F57A7FE4D2054B1B7A002B59
:1010D000E7D0FFF72FFCE4E708BD00BF7411002044
:1010E0007C11002038B5044603793BB905682DB161
:1010F000284600F0D7FC284600F030FE204638BDD8
:1011000010B50446064B036000F583500C30FFF722
:10111000E9FF04F58250183000F0C4FC204610BDF1
:10112000D04F000810B5064C064B9C4206D0A4F5E3
:101130008754083C2046FFF7E3FFF5E710BD00BFEA
:10114000B0270020C816002008B5FFF7D3FC08BD63
:1011500010B503F007FA0A4B1880002406E003F0EC
:10116000FDF90444074A136801331360B4F5204FB6
:1011700005D2034B1B88034A10688342EFD810BD89
:101180000C3800201038002008B503F035FA08BDEF
:1011900008B5920000F1006000F5204003F028FA45
:1011A00008BD00BF08B5064B1B88064A12689B1A8B
:1011B000834201D8002008BD104403F0CFF9FAE7BC
:1011C0000C3800201038002008B5034B1B68184469
:1011D00003F0CAF908BD00BF1038002008B5034B62
:1011E0001B68184403F0D8F908BD00BF1038002070
:1011F00008B5074B93F824300BB9012008BD04490A
:10120000002381F824300822086AFFF7C1FFF5E7C0
:10121000E4370020704700BF704700BF002304E0A0
:1012200011F803C000F803C001339342F8D37047AC
:101230000346002000E0013013F9012B002AFAD107
:10124000704700BF034602E003F8011B624602F14B
:10125000FF3C002AF8D170472DE9F84380460F463D
:101260001546224B93F824303BB3204A126A02EB16
:101270008303834221D0FFF7BBFF0346E8B931E087
:101280001A4E96F82400C0F10804AC4228BF2C4640
:10129000E4B24FEA84094A46394606EB8000FFF77C
:1012A000BDFFC8444F442D1BEDB296F824302344B3
:1012B000DBB286F82430082B0DD095B10B4B93F898
:1012C0002430002BDCD10948C0F820802022FF21E7
:1012D000FFF7B8FFD4E7FFF78BFF03460028ECD1F8
:1012E00000E001231846BDE8F88300BFE437002082
:1012F00070B506460C46154613462022096802F0D2
:10130000EBFA2168203121602B1D0222304602F0C9
:10131000E3FA2168023121606B1D0322304602F09E
:10132000DBFA216803312160AB1D0322304602F055
:10133000D3FA21680331216005F1080310223046F9
:1013400002F0CAFA23681033236070BD70B50646F8
:101350000C46154613460822096802F0BDFA2168BA
:10136000083121606B1C0822304602F0B5FA216872
:1013700008312160AB1C0822304602F0ADFA21682A
:10138000083121602B1D2022304602F0A5FA216889
:101390002031216005F108034022304602F09CFA1A
:1013A00023684033236070BD2DE9F04182B00746C9
:1013B0000C461646984613460822096802F08CFA35
:1013C000216808312160731C0822384602F084FA33
:1013D00023680833236000250AE0731902330822CA
:1013E0002168384602F078FA216808312160013519
:1013F0000F2DF2D9B37C8DF80730B8F1000F12D061
:1014000000259DF80730AB4218D905F1100333448D
:10141000033308222168384602F05EFA2368083355
:1014200023600135EDE70DF10703082221683846F6
:1014300002F052FA236808332360E1E702B0BDE806
:10144000F08100BFF0B583B007460D4616461C4636
:101450000023FFF74DFF002306F11002294638460E
:10146000FFF774FF002306F1200229463846FFF7F4
:101470009BFF96F83231502B28BF50238DF8073050
:101480000CB1002417E00DF1070307222968384644
:1014900002F022FA2B6807332B60F2E704F5987309
:1014A0003344033308222968384602F015FA2B68C2
:1014B00008332B6001349DF80730A342EED803B007
:1014C000F0BD00BF70B582B005460C46164600213F
:1014D000019140F279122046FFF7B4FE33462A46C6
:1014E00001A92046FFF7AEFF01980730C00802B0FF
:1014F00070BD00BF70B506460C4615461346202247
:10150000096802F0E9F92168203121602B1D0222CF
:10151000304602F0E1F92168023121606B1D03229F
:10152000304602F0D9F9216803312160AB1D032256
:10153000304602F0D1F921680331216005F108033A
:101540001022304602F0C8F923681033236070BDC2
:1015500000B583B08446084613460021019101601E
:10156000C0F80310624601A9FFF7C4FF01980730D5
:10157000C00803B05DF804FBF0B583B007460C4625
:1015800016461D46009200230722096802F0A6F8BD
:10159000216807312160731C009300230122384623
:1015A00002F09CF82168013121604DB1BB8AC1EB8A
:1015B000C301C908B170B378102B1FD8002517E0FC
:1015C000B31C009300230522384602F087F82368F5
:1015D00005332360EFE773190333009300230822D8
:1015E0002168384602F07AF8236808332360013511
:1015F000B378AB42EFD8002003B0F0BD0120FBE789
:1016000010B582B004460A46037F13B1818A1229BD
:1016100010D80021019101A92046FFF7ADFF034634
:1016200040B9019B0733DB08227F32B1A28AD31A6B
:1016300018BF0123184602B010BDA28A9A422CBFDF
:1016400000230123F6E700BFF0B583B007460D463F
:10165000164653B1828A0B68C3EBC203DB083370B2
:101660003378C82B1DD8002415E0009208220968A1
:1016700002F034F82B6808332B60F1E7331901339B
:101680000093002308222968384602F027F82B68C7
:1016900008332B6001343378A342EFD8002003B025
:1016A000F0BD0120FBE700BFF0B583B006460C4655
:1016B00015461F46009200230822096802F00EF822
:1016C0002368083323603B466A1C21463046FFF7F7
:1016D000BBFF03B0F0BD00BF10B582B004460A46A0
:1016E000037F13B1818ACA2910D80021019101A971
:1016F0002046FFF7D9FF034640B9019B0733DB08BB
:10170000227F32B1A28AD31A18BF0123184602B031
:1017100010BDA28A9A422CBF00230123F6E700BF26
:10172000F0B583B007460D4616461C461346082200
:10173000096802F0D1F8296808312960737896F9B0
:101740000120002A04DB8DF807301CB1002416E0CC
:101750007F23F8E70DF107030722384602F0BCF8B3
:101760002B6807332B60F1E733190233082229680D
:10177000384602F0B1F82B6808332B6001349DF82D
:101780000710A142F0D803B0F0BD00BF70B582B021
:1017900005460C4616460021019181222046FFF79E
:1017A00051FD33462A4601A92046FFF7B9FF0198AB
:1017B0000730C00802B070BDF0B583B007460D46D3
:1017C00016461278C82A28BFC8228DF807200BB108
:1017D000002414E00DF107030822096802F07CF8E8
:1017E0002B6808332B60F3E733190133082229688B
:1017F000384602F071F82B6808332B6001349DF8ED
:101800000730A342F0D803B0F0BD00BFF8B50646DC
:101810000C4615461F4613462822096802F05CF85C
:101820002368283323603B4605F1080221463046F1
:10183000FFF7C2FFF8BD00BF70B582B005460C4689
:10184000164600210191CE222046FFF7FBFC3346CD
:101850002A4601A92046FFF7D9FF01980730C008A2
:1018600002B070BDF0B583B007460D4616461C4663
:10187000009201231022096801F030FF296810311D
:10188000296054B1BB8AC1EBC301C9087180738858
:10189000B3F5807F1FD8002417E0B31C009300230A
:1018A0000922384601F01AFF2B6809332B60EEE756
:1018B000331904330093002308222968384601F0C5
:1018C0000DFF2B6808332B6001347388A342EFD8D7
:1018D000002003B0F0BD0120FBE700BF10B582B0CF
:1018E00004460A46037F1BB1818AB1F5827F10D876
:1018F0000021019101A92046FFF7B4FF034640B93A
:10190000019B0733DB08227F32B1A28AD31A18BFAA
:101910000123184602B010BDA28A9A422CBF0023B0
:101920000123F6E700B596460AE040F3000C0A4AA8
:101930000CEA020282EA50000133DBB2072BF4D931
:1019400073460EF1FF3E23B111F8013B58400023CE
:10195000F4E75DF804FB00BF2083B8EDF0B583B079
:101960001F4B6A4693E8030082E8030008231D49E1
:101970001D4803F0CDFA30B304460369B3F5583F70
:1019800023D8418B40F27F52914220D100F11807B9
:10199000164A024402F110018B421BD39B1AA3F199
:1019A000100511490020FFF7BDFF06462A463946BB
:1019B0000020FFF7B7FFA368B3420DD1E36883426D
:1019C0000CD1002004E00A2002E00B2000E00C20F3
:1019D00003B0F0BD1020FBE70D20F9E70D20F7E77D
:1019E000884F0008DC5F030000A000080860FFF7D4
:1019F000F0B583B0204B6A4693E8030082E8030009
:101A000008231E491E4803F083FA38B304460369CD
:101A1000B3F5583F24D8B0F8661040F27F52914297
:101A200020D100F16407174A024402F15C018B42A5
:101A30001BD39B1AA3F15C0511490020FFF772FF2D
:101A400006462A4639460020FFF76CFFA368B342DA
:101A50000DD1E36883420CD1002004E00A2002E0AB
:101A60000B2000E00C2003B0F0BD1020FBE70D20A0
:101A7000F9E70D20F7E700BF944F0008905F0300DF
:101A800000A000080860FFF710B5FFF767FF0446E5
:101A900008B9204610BDFFF7ABFF0028F9D1044676
:101AA000F7E700BF10B50446037C0BB1204610BD1C
:101AB000006803F015FAF9E7BFF35B8FC368BFF363
:101AC0005B8FBFF35B8F8268BFF35B8F9A4208D94D
:101AD0004268BFF35B8F8168BFF35B8F521AD018E7
:101AE0007047BFF35B8F8068BFF35B8F181A704736
:101AF000BFF35B8F0023C360BFF35B8FBFF35B8FCC
:101B00008360BFF35B8F70470346406800B970473E
:101B1000BFF35B8F9A68BFF35B8FBFF35B8FD968AE
:101B2000BFF35B8F914209D35868BFF35B8FDB68CB
:101B3000BFF35B8FD21A013A1044E8E70020F4E7C4
:101B400038B505460C46FFF7B7FFA04201D200208A
:101B500038BDBFF35B8FAB68BFF35B8F1C446B6812
:101B6000B4FBF3F203FB1244BFF35B8FAC60BFF333
:101B70005B8F0120ECE700BF70B504460E461546AA
:101B8000FFF7C2FFA84200D3284608B9002070BD65
:101B90002368BFF35B8FE268BFF35B8F134433604E
:101BA0006268BFF35B8FE368BFF35B8FD11A884233
:101BB00007D971602168B1609B1A0344F360022069
:101BC000E5E770600120E2E738B505460C46FFF70F
:101BD0009BFFA04201D2002038BDBFF35B8FEB68B2
:101BE000BFF35B8F1C446B68B4FBF3F203FB12443E
:101BF000BFF35B8FEC60BFF35B8F0120ECE700BFAE
:101C00002DE9F04385B0814688466946FFF7B4FF69
:101C10000746002425460EE004AB03EBC40656F845
:101C20000C2C08EB050156F8100CFFF7F7FA56F8E4
:101C30000C3C1D440134A742EEDC29464846FFF720
:101C4000C3FF284605B0BDE8F08300BFBFF35B8F3C
:101C5000C368BFF35B8FBFF35B8F8268BFF35B8F9B
:101C60009A4210D94368BFF35B8F8268BFF35B8FE2
:101C70009B1A0B6073B10368BFF35B8F8068BFF37F
:101C80005B8F18447047BFF35B8F8268BFF35B8F35
:101C90009B1AEEE700207047F0B583B007460E466A
:101CA0001546FFF709FF04460190A84200D32C46D1
:101CB00014B9002003B0F0BD01A93846FFF7C6FFF4
:101CC000019B6BB1A34200D901943060019B73600A
:101CD000A3420DD23A68B260E41AF4600220E9E748
:101CE0003B68336074600023B360F3600120E1E778
:101CF0000120DFE72DE9F04184B088466946FFF70F
:101D0000CBFF0746002425460EE004AB03EBC406D8
:101D100056F80C2C56F8101C08EB0500FFF77EFA5D
:101D200056F80C3C1D440134A742EEDC284604B0B2
:101D3000BDE8F08138B50546FFF7DCFF04460146F3
:101D40002846FFF7FDFE204638BD00BF08B500B9A4
:101D50000120012103F0BCF808BD00BF18B108B58F
:101D600003F0BEF808BD704710B5026854681A4603
:101D7000A04710BD0020704700207047704700BF8B
:101D8000002070470E20704700F5805090F8D80072
:101D9000C0F34000704700BF00F5805090F9E000AC
:101DA000704700BF00F58050C0F8DC10012070477C
:101DB000F0B583B0BDF820500C6814F0005F40F01F
:101DC00089800C7B082C00F28880302484F31188F1
:101DD000446AA66816F0806F0ED1A66816F0006FF0
:101DE0006BD1A66816F0805F02D04FF0020E05E0BE
:101DF000002080F311885EE04FF0000EF4460E687C
:101E0000002E5DDB76050EF1180E4FEA0E1E44F82B
:101E10000E600E6816F0804F06D00CF118063601E1
:101E2000A75947F00207A7510F7B0CF118064FEA9C
:101E3000061E04EB061677608E6804EB0C17C7F8D5
:101E40008C614E68C7F8886154F80E6046F0010650
:101E500044F80E6041F2780E0EEB4C14044400EB93
:101E60004C1CE644CEF80020CEF80430D1F800E057
:101E70004F688E68C4F808E0E76026618E89A68204
:101E80000CF5845C9CF8144065F300048CF8144055
:101E9000C5F34006E4B266F341048CF81440E4B2A2
:101EA00024F008048CF81440002484F31188009571
:101EB00000F052FE012003B0F0BD4FF0010E9DE78F
:101EC000F60046F004060EF1180E4FEA0E1E44F816
:101ED0000E609EE74FF0FF30EDE74FF0FF30EAE78E
:101EE00008B5302383F3118800F58050C06EFFF7EA
:101EF000FFFD002383F3118808BD00BF2DE9F041E9
:101F000006460F4603462F4A43F8042B002444603C
:101F10005C609C60DC601C615C612B4B40F8283B82
:101F2000FEF702FE00220023C6E90E23A6F8404079
:101F300006F14400FEF7F8FD06F1580844467F25F7
:101F40000BE000220023C4E900230023238104F1D5
:101F50000C00FEF7E9FD013D2034002DF1DA06F515
:101F60008053C3F858804FF48052DA6500221A6615
:101F70005A66012183F8681006F582521832DA6633
:101F800083F8701006F58354183402250AE02046C1
:101F900000220023E0E80223FEF7C6FD0023A36130
:101FA000013D2034002DF2DA06F5805383F8E0700D
:101FB00027B9064B73623046BDE8F081044800F053
:101FC0004DFD00BF2C500008D04F000800640040B9
:101FD000A04F000810B50446034B19784A1C1A702C
:101FE000FFF78CFF204610BD14380020002978D060
:101FF00070B582B00C46424B994211D90A2341492F
:10200000B1FBF4FC013BDBB29E46581CBCFBF0F17B
:1020100000FB11C131B1022B65D9013BDBB2F3E703
:102020001123ECE7BCFBF0FC0CF1FF31B1F5806F44
:102030005CD2C3EBC30E1EF103004DD4C0F3C70046
:102040008DF800001D1AEDB28DF80150461C4FF4BA
:102050007A7100FB0111701991FBF0F189B2ADF8B2
:102060000210B1F5617F18D9BEF1010E36D4CEF35E
:10207000C70E8DF804E0A3EB0E03DBB28DF805303C
:102080000EF101004FF47A710EFB0111034491FB34
:10209000F3F1ADF80610019B00939DF800104B1C66
:1020A0009DF801502B440CFB03F31648B0FBF3F3EF
:1020B000A3421DD10139C9B20F291BD8E5B1082DA2
:1020C0001CD80CF1FF3CA2F800C000239370D17023
:1020D000013D1571012007E00730AFE70EF1070E53
:1020E000C5E700207047002002B070BD0020FBE76C
:1020F0000020F9E70020F7E70020F5E70020F3E7EC
:102100003F420F0000B4C40470B506460D460024DB
:10211000B4F57A7F0BD2736A5B6803F00103AB42BC
:1021200007D04FF47A7002F00DF80134F0E7002088
:1021300000E0012070BD00BF03295FD8F0B589B071
:1021400004460D46164600F5805393F8D830C3F385
:10215000800113F0040F00D1114604F5805393F869
:10216000D82061F3820283F8D82041F2780303EB90
:102170004513E71804EB451303F5845310331B791B
:1021800013F0010F09D0CEB104EB451303F58453CE
:1021900010331B7913F0080F12D07EB104EB4513F6
:1021A00003F5845310331B7913F0080F06D104EBA9
:1021B000451404F5845443F00803237509B0F0BDB9
:1021C00000220023CDE900230023ADF8083003A846
:1021D000FEF7AAFC03ABB868F9683A6907C3BA8A84
:1021E0001A80DDE90E23CDE900230123ADF8083084
:1021F00023681B6C694620469847CEE7704700BFAE
:10220000426A936913F0700F25D00023936100E0B8
:102210000133022B1FDC00EB431202F58452103213
:10222000127912F0040FF3D000EB431202F584523E
:102230001032127912F0020FEAD0426A064951F8C0
:102240002310916000EB431202F58452117D41F09E
:1022500004011175DCE770471450000870B582B0B6
:10226000044616461D46436A9A6812F0010F16D1BD
:10227000636A9A6812F4807F1CD1636A9A6812F4C8
:10228000803F24D104F58053D3F8DC0010B10368FB
:102290001B6998472046FFF7B3FF02B070BD9A68EC
:1022A0000121996000960195C2F340020021FFF7D9
:1022B00043FFDDE79A684FF48071996000960195BD
:1022C000C2F3402201212046FFF736FFD5E79A6886
:1022D0004FF48031996000960195C2F3404202218B
:1022E0002046FFF729FFCDE710B50B4B1C5604B174
:1022F00010BD00F0BDFB02460B4652EA030102D0BE
:10230000013A43F1FF33054951F824000028EFD08A
:10231000FFF7A4FFECE700BF2050000818380020AA
:1023200038B50446084600297CD1616A01F10C0CDD
:10233000DCF8001011F0030F73D0DCF80010616AB4
:1023400000F11B052D014D5915F0040F6ED100F160
:102350001B052D014D596D0DA56200F11B052D01C9
:102360004D5915F0020F03D0A56A45F08045A562CE
:1023700000F11B0501EB05156D6805F00F0E84F8E3
:1023800034E001EB0011D1F8B80184F82C00D1F849
:10239000B801000A84F82D00D1F8B801000C84F8C7
:1023A0002E00D1F8B801000E84F82F00D1F8BC013E
:1023B00084F83000D1F8BC01000A84F83100D1F86B
:1023C000BC01000C84F83200D1F8BC11090E84F86D
:1023D00033103821CCF80010A56AE06A216B6564DF
:1023E000A064E164A18EA4F85010A263E36300230B
:1023F000A4F8403023681B6C04F13801204698474C
:1024000004F5805393F8D82042F0040283F8D820D2
:10241000D3F8DC0010B103681B6998472046FFF72A
:10242000EFFE38BD616A01F1100C81E700F11B0578
:102430002D014D59ED08A56245F00045A5628CE7D8
:1024400038B50C4B1D5605B138BD0C4600F010FBDD
:1024500002460B4652EA030102D0013A43F1FF3330
:10246000054951F825000028EED02146FFF758FF16
:10247000EAE700BF2050000818380020302181F31F
:1024800011880021022937DC30B502E00131022930
:102490002EDC00EB411C0CF5845C0CF1100C9CF85C
:1024A00004C01CF0040FF1D100EB411C0CF5845C5E
:1024B0009CF8144014F0100FE8D000EB411C41F2DE
:1024C00078040CEB040E5CF80450DEF804409542EE
:1024D0009C41DBD2446A0A4D55F82150A5600CF5A9
:1024E000845C9CF8144044F004048CF81440CDE75C
:1024F000002383F3118830BD002383F311887047D4
:102500001450000808B5302383F31188FFF778FED4
:10251000002383F3118808BD436A9B6803F0E053EE
:10252000B3F1E05F2CD070B505460E4653B33023AF
:1025300083F31188002400E00134022C1BDC05EB3E
:10254000441303F5845310331B7913F0080FF3D1B0
:1025500005EB441303F5845310331B7913F0040F78
:10256000EAD104F1840105EB4111304600F046FB4D
:102570000028E1D100E00120002383F3118870BD21
:10258000012070470020FAE708B5302383F3118853
:1025900000F58050C06EFFF78FFA002383F3118897
:1025A0001F288CBF0020012008BD00BFF8B50746DA
:1025B0000E4614461D4600231370FFF7E5FF80F01A
:1025C0000103337025B129463846FFF7A5FF207077
:1025D000F8BD00BFF8B504460D4616461F4600F08C
:1025E00047FA02460B46297809B9307860B120468F
:1025F000FFF744FF2046FFF785FF3B46324629465A
:102600002046FFF7D3FF0120F8BD00BF302383F33E
:1026100011881B4B9A6D42F000729A659A6B42F0DA
:1026200000729A639A6B22F000729A63002383F31C
:10263000118800F5805393F8D83013F0010F1ED1A4
:1026400010B5044601B910BD302383F3118803216E
:10265000132001F067FC0321142001F063FC032127
:10266000152001F05FFC04F5805494F8D83043F055
:10267000010384F8D830002383F31188E3E770471F
:102680000010024000F5805393F8E030012B00F277
:102690002E812DE9F0418AB004460E461746954A30
:1026A00052F82320002A37D0E66184F82070914B3D
:1026B0001B68002B34D004F5805393F8E030012BD5
:1026C00006D18C4B186803681B6B9847002836D0DE
:1026D00001212046FFF79AFF302383F31188626AB5
:1026E000136823F002031360626A136843F0010366
:1026F0001360626A0023536183F31188012120462D
:10270000FFF702FD034648BB626A4FF400411160C7
:1027100018460AB0BDE8F081764A42F82300C3E7C4
:1027200041F2E800FFF712FB054610B10021FFF768
:10273000E5FB704B1D60002DBDD10023E8E76D4D1A
:1027400000212868FFF762FF286803685B683A4643
:102750003146984703460028BAD1D9E704F580539B
:10276000D86EFFF7C5F94FF0000827E020220021BE
:102770006846FEF767FD02A8FEF7D6F90023069328
:1027800041F2780505EB481504EB050EEC46BCE874
:102790000F006051CEF80410CEF80820CEF80C30AF
:1027A000BCE80700CEF81000CEF81410CEF81820C0
:1027B0009CF800308EF81C3008F10108B8F1020FC7
:1027C000D4D904F5805292F8D83023F0040382F86B
:1027D000D8300023ADF820308DF822308DF823302A
:1027E0008DF8243008AA31462046FFF7FFFB034648
:1027F00000286FD0636A61221A609DF822301B06A0
:1028000003F040739DF82320120402F47022134356
:102810009DF82420120502F4E0021343BDF82020A5
:10282000C2F309021343022F59D00021626A0B43FD
:10283000D361636A13225A61626A136823F0010349
:10284000136000212046FFF75FFC0346002849D0B3
:1028500004F5805292F8E0209ABB616AD1F8002218
:1028600042F00102C1F80022616AD1F8002222F48C
:102870007C5222F00E02C1F80022616AD1F80022D7
:1028800042F46062C1F80022616A0022C1F8142299
:10289000616AC1F80422616A41F6FF70C1F80C0256
:1028A000616AC1F84022616AC1F84422626A01216A
:1028B000C2F81C12616AD1F8002222F00102C1F8AC
:1028C000002204F5805494F8D82042F0020284F8E3
:1028D000D8201DE7626A4FF40041116018E74FF0FD
:1028E0000041A3E7626A4FF40041116010E7002342
:1028F000184670471838002008B50020FFF7F4FC90
:1029000001F0CAFA08BD00BF08B500210846FFF76C
:1029100097FD01F0C1FA08BD08B501210020FFF7BD
:102920008FFD01F0B9FA08BD38B504460D460068C0
:10293000FFF7EAF81F2801D8002038BD20222946D9
:102940002068FFF75DF9202814BF00200120F4E77C
:1029500008B500F583500C30FFF7E6FF08BD00BF57
:1029600038B504460D460068FFF7A6F81F2801D8C1
:10297000002038BD202229462068FFF7DBF92028F7
:1029800014BF00200120F4E7F0B589B005460C46DD
:1029900016461F46302383F3118800220023CDE919
:1029A00000230023ADF8083003A8FEF7BDF8694600
:1029B00005F583500C30FFF7D3FF18B980F3118869
:1029C00009B0F0BD03AB07CB20606160A2601B883B
:1029D000A381DDE90023C6E90023BDF808303B8070
:1029E000002383F311883B4632462146284600F0F7
:1029F0004DF8E5E700B59BB0EFF309816822684622
:102A0000FEF70CFCEFF30583014B9B6BFEE700BF69
:102A100000ED00E000B59BB0EFF309816822684645
:102A2000FEF7FCFBEFF30583014B9B6BFEE700BF5A
:102A300000ED00E000B59BB0EFF309816822684625
:102A4000FEF7ECFBEFF30583014B5B6BFEE700BF8A
:102A500000ED00E0FEE700BFFEE700BF0FB408B5E1
:102A6000029801F021FBFEE708B501F033FE08BD36
:102A700008B501F00BFE08BD00207047012070472B
:102A80000020704700207047704700BF2DE9F043D9
:102A900083B01E461B8813F0040F1ED105468946DD
:102AA000041D00F11C080CE02B68DB6B28469847DE
:102AB000338843F004034A46C1B220686768B847C8
:102AC0000834444509D00020009001902368002B71
:102AD000EAD16368002BE7D1F2E7012003B0BDE83B
:102AE000F08300BF84B0EC468CE80600002201E0D1
:102AF0000132D2B2022A18D800210291039100EBD0
:102B0000C20149680029F3D100EBC201896800299C
:102B1000EED100EBC20000F1040C694603C98CE859
:102B2000030001321A70012000E0002004B0704759
:102B30000139C9B202290DD882B000230093019354
:102B400000EBC100031D02AA12E9030083E80300A1
:102B500002B07047704700BF2DE9F0478AB00546C4
:102B60008A46BDF84870041D00F11C084FF00009AA
:102B700006E0636863B902E0B9F1000F16D00834CB
:102B8000444537D00023089309932368002BF0D0E5
:102B900017F0040FF0D12B68DB6B284698473B46B3
:102BA0005246C1B220686668B047E8E700220023B9
:102BB000CDE900230023ADF8083003A8FDF7B4FFEA
:102BC00003ABDAF80000DAF80410DAF8082007C3DB
:102BD000BAF80C201A80FFF74BFFCDE9000104235F
:102BE000ADF808302B681B6C6946284698474FF0B3
:102BF0000109C4E701200AB0BDE8F087026822F0AD
:102C0000604C0B6823F06041D80F92EA030F0AD49E
:102C1000C2F38072C3F380708C4514D08C452CBFF6
:102C2000002001207047002A08DB002B09DB8C45BF
:102C3000F8D08C452CBF0020012070474FEA9C4CF7
:102C4000F3E7890CF3E78242ECD1E7E708467047E7
:102C5000084670470846704708467047401A83B2D6
:102C6000002800DB7047203318B2FBE703780133FC
:102C7000DBB203701F2B01D900230370704700BF24
:102C80000E2809D8DFE800F01515151515151515CE
:102C9000150A0C0E10121400402070470C207047CB
:102CA000102070471420704718207047202070476C
:102CB00030207047082818D90C280BD910280BD9B8
:102CC00014280BD918280BD920280BD930280BD958
:102CD0000F207047092070470A2070470B2070476B
:102CE0000C2070470D2070470E207047034621F0DE
:102CF000604C20F06042C00F91EA030F0AD4C1F388
:102D00008071C3F38070944514D094452CBF00208B
:102D100001207047002908DB002B09DB9445F8D01F
:102D200094452CBF0020012070474FEA9C4CF3E7EC
:102D3000920CF3E78142ECD1E7E700BF2DE9F041C7
:102D400007460D46D0F82480B8F1000F0CD0464657
:102D50004446A4B169686068FFF7C8FF30B92368CA
:102D600026465BB11C46F4E7796208E0A04502D034
:102D700035602C6003E02C607D6200E02560BDE8DA
:102D8000F08100BFC37DC3F38402013262F3860386
:102D9000C375C38A6FF30903C382C37D23F0800325
:102DA000C375704738B504460D46006A04E00168F3
:102DB00004F10C00FFF74EFF10B10369AB42F6D1EE
:102DC00038BD00BF2DE9F043079ECD0803EBD604C4
:102DD00001F0070E06F0070372442AE00EF0070820
:102DE00003F00706C446B04538BFB446CCF1080C22
:102DF000A2EB0E018C4528BF8C464FF47F4121FA8F
:102E00000CF1C9B241FA06F74FEADE0100EB050901
:102E100019F8011001FA08F1F140C9B24FEAD308DC
:102E200014F80860714039404E4004F80860E644E8
:102E300063449645D2D1BDE8F08300BF2DE9F04F41
:102E400087B00393838AB1EBC30F80F087808246FB
:102E50000E461546DA0069188A4203D2D3B2F2B29E
:102E60009B1ADDB2DAF80C3043B3272E36D8C6F100
:102E700028039D4230D35FFA86FBCBF1280B5FFA23
:102E80008BFB00230093039B5A463146DAF8080077
:102E9000FFF798FF5E44A5EB0B04E4B2BAF8147098
:102EA00007F10057053FFF00DAF80C9028214B4648
:102EB000B946CDF810A005951F4626E0DAF8103087
:102EC000002BD2D100230093039B2A463146DAF827
:102ED0000800FFF777FF35E0AB46D2E72C464FF00E
:102EE000000BDBE72546CDF800B0039B2A46711A9C
:102EF000381DFFF767FF2E44AB445FFA8BFB651B61
:102F0000ECB2A9EB0A093F684146A7B19CB1CA4699
:102F1000B9F1E00F28BF4FF0E00A0AEB010846457F
:102F2000EFD2A8EB06039C42DCD35FFA88F5F3B23C
:102F3000ED1AEDB2D7E7DDF810A0059DDAF8100024
:102F400000B11CB928B207B0BDE8F08FCDF800B0D1
:102F5000039B2246711AFFF735FFF3E70020F2E7E3
:102F6000002070470139002307E0C25C10F801C05F
:102F700000F803C04254013301398B42F5D3704746
:102F800080EA0120002303E0400080B20133DBB27D
:102F9000072B09D810F4004FF6D0400080B280F41F
:102FA000815080F00100F1E7704700BF70B5164610
:102FB0001D46002411E0C4F12003A4F1200C26FAE0
:102FC00004F105FA03F3194325FA0CFC41EA0C015C
:102FD000C9B2FFF7D5FF0834A4B23F2CEBD970BDBE
:102FE00038B50C4604E014F8011BFFF7C9FF2A4668
:102FF000551E002AF7D138BD38B5058C072D0BD9E1
:103000000446D0E902234FF6FF70FFF7CFFF2A46B0
:10301000E169FFF7E5FF38BD4FF6FF70FBE700BF42
:1030200010B4016100F1040C002305E001EB43142E
:10303000CCF80040A44601339A42F7D80023CCF8DC
:10304000003002814381838103605DF8044B704747
:103050000346406848B102685A605A89013292B208
:103060005A8199898A4200D99A81704708B5FFF739
:10307000EFFF08B10023036008BD00BF2DE9F84F42
:103080008246894617461D46CB8AC3F30903052BA2
:1030900032D018460024042B0AD8A54208D9395D3D
:1030A00009EB0302D17601339BB20134A4B2F2E7FB
:1030B000A54218D9B9F816B0CBF3090BABF105024C
:1030C00093083D49A1FB0313C3EBC303A2EB8302A7
:1030D0001FFA82F8D9F8041081B15046FFF7B6FD07
:1030E000064601231CE02844B9F8163060F30903B2
:1030F000A9F81630012054E00024DBE75046FFF722
:10310000B5FF064601465046FFF7A2FDC9F8040088
:10311000002E48D04FF000082CE001339BB2164639
:103120003268002AF9D105EB0B02053A92082249D0
:10313000A1FB021292B2013292B293421AD2B8F1BA
:10314000000F17D15046FFF791FF306070B306466D
:1031500010E03A5D06EB0C031A710CF1010C1FFA3A
:103160008CFC0134A4B2BCF11B0F01D8A542F0D8ED
:10317000A54203D8A5420AD9C446F4E75046FFF752
:1031800075FF3060A8B106464FF00008F2E7B9F8C5
:103190001630C3F30902154465F30903A9F8163084
:1031A0000120BDE8F88F6FF00200FAE76FF002002F
:1031B000F7E76FF00200F4E72549922443680B60BB
:1031C00041604389013B4381704700BFF8B5064623
:1031D0000D460EE006F10C042046FFF737FD0146D0
:1031E00007682046FFF7EAFF39462046FFF730FD23
:1031F000686069680029EDD1EB8A6FF30903EB82FF
:1032000000200021F8BD00BF08B5FFF721FF0346ED
:1032100028B10022026042608260C26002611846EA
:1032200008BD00BF2DE9F04F83B001921D465B69D8
:10323000002B00F0998081468B462B8C1BB1EA69EC
:10324000002A00F09480072B18D902339BB2063372
:103250004D4A82FB03121344C3F38F03B9F81420C1
:10326000B9F81610521A92B2934200F286804FF0CB
:10327000800A4FF000084446474654E009F10C002C
:10328000FFF7C2FF0446002874D02A8CE969083091
:10329000FDF7C4FF288C013080B2FFF70BFDFFF76C
:1032A000EFFC431E9BB22B84013323746B691B78A4
:1032B00003F01F032A8C43F0C003224413724BF027
:1032C0000043636021464846FFF738FD0127384632
:1032D00003B0BDE8F08F002035E02B8CA34240D036
:1032E000013080B2FFF7E6FCFFF7CAFC431E9BB239
:1032F0004FEA4812D2B242EA0A026969097801F03B
:103300001F010A43F1180A724BF000427260013348
:10331000337431464846FFF711FD01373FB288F05C
:1033200001084FF0000A2B8CA342D0D009F10C0009
:10333000FFF76AFF064618B3002CCCD1019B03723D
:103340001B0A437202200628C7D82B8CA342C4D97B
:10335000EB691A5D33181A72013080B20134A4B2DD
:10336000F1E74FF0400ABBE76FF00107AFE76FF0FE
:103370000107ACE76FF00207A9E76FF00207A6E7C5
:103380006FF00207A3E700BF9324499230B589B0DC
:1033900004460D46202200216846FDF753FF0495A0
:1033A0002046FFF755FE8646A0B1EC46BCE80F006C
:1033B000CEF80000CEF80410CEF80820CEF80C307D
:1033C000BCE80F00CEF81000CEF81410CEF818208C
:1033D000CEF81C30704609B030BD00BF70B5044651
:1033E00000F10C063046FFF7D1FF054628B1216AEF
:1033F0003046FFF731FC28602562284670BD00BFCB
:1034000038B504460D46036A1BB1FFF7CBFC38B153
:1034100038BD0C30FFF7BAFF0028F9D02062F7E77B
:1034200029462046FFF7DAFFF2E700BFF8B5044669
:103430000E4615461F4630220021FDF703FFA76008
:10344000069B6360079BA3626A09B5F5001F01D361
:103450004FF6FF7292B2314604F10C00FFF7E0FD27
:10346000F8BD00BF037823B919B111F0800F00D166
:1034700001707047007870472DE9F84305460C4607
:10348000D1F81C90B9F1000F22D094F81880B8F14F
:103490001F0F3AD82846FFF7EDFF0646F0B9228CF9
:1034A000072A35D8278A032F35D849464FF6FF70AB
:1034B000FFF796FD47F6FE7303405B0243EA08639D
:1034C0003F0207F440773B431E434FF6FF720EE086
:1034D0000B8C002BD9D06FF001050FE0238A1B0263
:1034E00043EA08631E432046FFF786FD0246234653
:1034F00031462846FFF796FE051E02DC2846BDE849
:10350000F8836069FFF7B2FBF8E76FF00105F5E7B4
:103510006FF00305F2E76FF00105EFE770B58AB0D1
:10352000044616461D46282200216846FDF78AFEFD
:1035300002960395BDF83830ADF810300F9B059317
:103540009DF840308DF81830119B0793BDF8483036
:10355000ADF8203069462046FFF78EFF0AB070BDF7
:103560002DE9F04106460F461546D3692BB395F871
:103570001880B8F11F0F2AD83046FFF77BFF48B3F9
:103580002C8A240444EA08642A7844EAC23444EACF
:103590000724044344F080042846FFF72DFD02462B
:1035A0002B4621463046FFF73DFE041E02DD2B78F8
:1035B000012B08D02046BDE8F081138C002BD6D01B
:1035C0006FF00104F6E76869FFF750FBF2E76FF070
:1035D0000104EFE76FF00304ECE700BFF0B58BB038
:1035E00004460D4617461E46282200216846FDF770
:1035F00029FE9DF84C30012B14BF002301238DF8C8
:103600000030029703969DF84030ADF81030119BC2
:1036100005939DF848308DF81830149B0793BDF83A
:103620005430ADF820306A4629462046FFF798FF0F
:103630000BB0F0BD406A00B10430704708B5416A74
:103640000B6843620C30FFF7B9FD08BD2DE9F0416E
:10365000054616469846076A3C4619E02146284624
:10366000FFF7B4FD05F10C072B6A19683846FFF720
:10367000F1FA286221463846FFF7A0FD2C6A27465A
:1036800006E0216805F10C00FFF7E4FA274604463E
:1036900004B3A168E368711A68EB03030E4A8A4217
:1036A0004FF000029A41ECD22B6AA342D6D02146B9
:1036B0002846FFF78BFD23683B6005F10C0321468C
:1036C0001C461846FFF77AFD39682046FFF7C2FA14
:1036D0000446DDE7BDE8F08180841E002DE9F0415D
:1036E00082B0089E002800F0DF8014461D46074681
:1036F000002E00F0DC80013AD2B23F2A00F2DA80DC
:10370000012C02D1002B40F0D880002300930193BC
:103710006B4622463846FFF791FB071E3ADD14F050
:10372000070F0AD002AB03EBD40111F8083C624248
:1037300002F00702134101F8083C012C0BD0082CC1
:103740002CD9102C2DD9202C2ED9402C00F2B88049
:103750004FF0080800E0A046FFF702FC38BB002D40
:1037600072D0B4EBC80F10D0082C25D89DF80020DB
:10377000631E22FA03F313F0010F06D00123A340C6
:103780005B42DBB21A438DF80020082C64D89DF907
:1037900000303370384602B0BDE8F0814FF00108C8
:1037A000DAE74FF00208D7E74FF00408D4E74146C4
:1037B0006846FFF7D7FBD2E7102C0FD8BDF80020E2
:1037C000631E22FA03F313F0010FDED00123A3409E
:1037D0005B429BB21A43ADF80020D6E7202C0CD8F0
:1037E000009A631E22FA03F313F0010FCDD00123D8
:1037F000A3405B421A430092C7E73F2C63D8009D69
:10380000019A631EC4F12100A4F1210125FA03F3FA
:1038100002FA00F0034322FA01F10B4313F0010F07
:10382000B3D00123A4F12001C4F1200003FA01F177
:1038300023FA00F00143A3405B4261EB41011D43C9
:103840000A4300950192A0E7012C17D0082C19D843
:103850009DF8003033709DE7102C03D8BDF900307F
:10386000338097E7202C02D8009B336092E7402CEE
:103870002CD8DDE90023C6E900238BE79DF8003052
:10388000337087E7102C03D8BDF80030338081E710
:10389000202C02D8009B33607CE7402C19D8DDE94E
:1038A0000023C6E9002375E76FF0010772E76FF0A8
:1038B00001076FE76FF001076CE76FF0010769E739
:1038C0006FF0080766E76FF0080763E76FF0080717
:1038D00060E76FF008075DE7F0B585B005460E4676
:1038E000402A03D8144612B9012400E040240022E3
:1038F00002920392012C06D0082C22D81B788DF856
:103900000830012703E01B788DF808302746FFF7C1
:1039100027FB68BB14F0070F0AD004AB03EBD401FC
:1039200011F8083C624202F00702934001F8083C9B
:1039300000962B462246002102A8FFF743FA05B065
:10394000F0BD102C04D81B88ADF808300227DEE744
:10395000202C03D81B6802930427D8E7402C05D8F5
:10396000D3E90023CDE902230827D0E70027CEE7DB
:10397000394602A8FFF7F6FACCE700BF70B5064655
:103980000C4605E00D6806F10C00FFF717FCE5603A
:10399000E1680029F6D10023E360A3602361A382DC
:1039A00070BD00BF10F0800F04D010F4004F03D0A2
:1039B00001207047022070470020704710B5044670
:1039C000FFF7F0FF022802D0C4F3074010BDC4F394
:1039D0000F2014F07F0FF9D100F00300F6E700BFCD
:1039E0002DE9F04F99B006460D4603920493D1F8A5
:1039F00000904846FFF7D6FF0746022800F0E48013
:103A0000C9F30628B9F1000F80F2F38119F0C04F15
:103A100040F0F2812C7B002C00F0F181022F05D0C8
:103A20003046FFF727FD404540F0EC81C9F30463C1
:103A3000099309F07F0105914846FFF7BFFF0A90FF
:103A400040EA0749059949EA814949EA4869013C40
:103A50002C4494F8048000220023CDE916235FEA69
:103A6000D813029300F0B380746800913B4602467D
:103A700016A93046A047002800F0C78149463046C5
:103A8000FFF7BEFC0446002800F0C281A368D4F80A
:103A90000CA0039A0693D21A0792049860EB0A00CE
:103AA00008906A7B0B92A07E0C9094F81790C9F353
:103AB000840908F01F0B59464846FFF7CFF80D90D0
:103AC00049465846FFF7CAF86268069B53EA0A0A55
:103AD00017D0974B07998B424FF0000308998B4101
:103AE0000FD30B9B0C998B427CD0924B079A93423D
:103AF0004FF00003089A934114D2029B93B10F2810
:103B000010DCE37D68F38603E375DBB223F080030A
:103B1000E37521463046FFF759FB6B7BA376029B8A
:103B2000002B69D06A7BA37E9A4240F07481029B8D
:103B300013B118F0400F69D1C8F34013E27DB3EB25
:103B4000D21F40F06C81C2F384039B4540F06A8130
:103B5000029B002B00F0948018F0400F40F09380FF
:103B60002B7B032B40F26181039BA360049BE360EA
:103B7000E38A6FF30903E382AF1D2B7B033BDBB2C8
:103B80003A46214606F10C00FFF778FA00286DDB73
:103B90002B796A7943EA02232383DDE916234FF662
:103BA000FF70FFF703FAA0822A7B033AD2B23946AC
:103BB000FFF716FAA082E37DDA43C2F3C01262F384
:103BC000C713E375002027E14FF000081AE74946C4
:103BD0003046FFF7E7F8044600287FF457AF6FF050
:103BE0000C0019E1029B002B3FF47FAF0D9B012BD2
:103BF00087DC002A85D178E7E37DC3F384020132B4
:103C000062F38603E3756FF00C0005E1039BA3608C
:103C1000049AE260202200210EA8FDF713FB039B0B
:103C20000E93049A0F922B1D10932B7B013BDBB25A
:103C3000ADF84C300A9BADF84E308DF850708DF8D1
:103C400051B0099B8DF85230059B8DF8533096F892
:103C50002C3083F001038DF85430B3680EA9304640
:103C600098472046FFF78EF80020D5E021463046E1
:103C7000FFF7ACFA2046FFF785F86FF00200CBE0C3
:103C800018F0400F1ED095F80C9009F1FF395FFA3B
:103C900089F9B4F81680C8F30908B8F1040F30D8D0
:103CA00043464FF00008042B54D8C84552D205EBC8
:103CB00008021179E218D176013308F101085FFAA0
:103CC00088F8F0E72F1D2B7B013BDBB23A462146FB
:103CD00006F10C00FFF7D2F9002808DB2A7B013A35
:103CE000D2B23946A08AFFF77BF9A08263E721466A
:103CF0003046FFF76BFA2046FFF744F86FF00200FA
:103D00008AE0616806F10C00FEF7A0FF024608B1E8
:103D1000052104E04FF000081CE01C311A4613682E
:103D2000002BFAD1A8EB01034FF000080EE000BF12
:103D300080841E0040420F0005EB08010879D1186D
:103D40000871013308F101085FFA88F81B2B01D8CC
:103D5000C845F1D3039B0E93049B0F9304F11B03FF
:103D60001093616806F10C00FEF770FF1190C845D2
:103D700036D2A84408F104031293E38AC3F309037B
:103D80009944ADF84C900A9BADF84E308DF85070C8
:103D90008DF851B0099B8DF85230059B8DF853304A
:103DA00096F82C3083F001038DF8543000236360C3
:103DB0002A7B013A291DA08AFFF712F9A082238BE2
:103DC00098420FD00EA93046FFF7D8FD2046FEF7E7
:103DD000D9FFA28A238B9A4209D06FF010001BE012
:103DE0000023C9E7B3680EA930469847EAE70020E8
:103DF00012E06FF009000FE06FF009000CE06FF0C7
:103E0000090009E06FF00A0006E06FF00B0003E024
:103E10006FF0020000E0002019B0BDE8F08F6FF0F5
:103E20000D00F9E76FF00E00F6E76FF00F00F3E713
:103E3000EFF30983683305494A6B22F001024A63B4
:103E400083F30988002383F31188704700EF00E0B3
:103E5000302080F3118862B60C4BD96821F4E06100
:103E60000904090C0A4A0A43DA60D3F8FC2042F03C
:103E70008072C3F8FC2007490A6842F001020A6018
:103E80002022DA7783F82200704700BF00ED00E0BF
:103E90000003FA05001000E0302383F31188104B73
:103EA0005B6813F4006F03D1002383F3118870471C
:103EB00010B5F1EE103AEFF30984683C4FF08073CF
:103EC000E361084BDB6B236684F3098800F0AEF8EE
:103ED00010B1054BA36110BD044BA361FBE700BF0C
:103EE00000ED00E000EF00E0FF0200080203000820
:103EF00010B44FF0E0235C6800230BE0084A03F1A4
:103F000020004FF0FF3142F8201003F1600042F82A
:103F100020100133A342F1D95DF8044B704700BF74
:103F200000E100E00901C9B2074A131883F8001341
:103F300000F01F01400901238B4000F1600142F8AD
:103F4000213042F82030704700E100E00023037583
:103F500003691B68996882689142FAD203605A68C3
:103F6000426010605860704708B50846302383F3FC
:103F700011880B7D032B05D0042B0FD02BB983F3B5
:103F800011880AE08B6900221A604FF0FF338361C9
:103F9000FFF7DCFF002383F3118808BD4A680B6834
:103FA00013604A685A60F0E70023037503691B68D1
:103FB000996882689142FAD803605A68426010603A
:103FC0005860704708B5FFF7C1FF08BD08B5064B3C
:103FD000D9680875186802681A6053600122027572
:103FE000D860FCF777F908BD303A002030B587B0CB
:103FF00004460C4BDD68B1F1FF3F0FD02B460A4A57
:10400000684600F025F92046FFF7E0FF009B13B15A
:10401000684600F02BF9A86907B030BDFFF7D6FF5E
:10402000F9E700BF303A0020693F0008044BDA6826
:104030001B6898689368984294BF002001207047DD
:10404000303A002010B5084BD8681C6822681A6006
:10405000536001222275DC60FFF7A6FF014620466F
:10406000FCF738F910BD00BF303A002008B50B4B03
:1040700001221A70002353B109490A4800F030FCAC
:10408000064B02221A70002383F3118808BD034AED
:1040900002EB8302002151600133ECE7883A0020F3
:1040A00070500008303A002008B572B6044B18650D
:1040B00000F0BAFA00F098FB024B03221A70FEE7F8
:1040C000303A0020883A002008B500F009F908BD10
:1040D0008B6002230B7500234B75086108467047FF
:1040E00008B58168A1F1840341F8143C026941F8E4
:1040F000442C426941F8402C044A41F8242CC368FE
:10410000026820390248FFF7E3FF08BDED0200080E
:10411000303A002008B5FFF7E3FFFFF753FF08BD73
:1041200008B5034BDB6898610F20FFF74FFF08BD10
:10413000303A002008B5302383F31188FFF7F0FFF1
:1041400008BD00BF08B50146302383F3118808205D
:10415000FFF74CFF002383F3118808BD10B40368F8
:1041600001E0121B1B689C68A242FAD88A600B60AF
:104170005C684C60216059609968891A99604FF0B9
:10418000FF3383605DF8044B704700BFF8B51546F8
:104190001C46C2608B60486003680B605960016018
:1041A000092C00D80A24C068204400F085FB0A27A7
:1041B00000F07EFB0646431B9C4202D90A2F07D81B
:1041C000F8BD7C1C281900F085FB27463546EFE733
:1041D000012000F0C5FBF3E770B504460D46092940
:1041E00000D80A250A26601900F074FB00F060FB75
:1041F000041BA54202D90A2E04D870BD01363546EB
:104200000446F0E7012000F0ABFBF6E7F8B5054601
:104210000F46164600F04CFB2B689D420DD0EC6813
:10422000041B341900D334469B68A3420CD82246A1
:1042300039462846FFF792FFF8BD33460246394615
:104240002846FFF7A3FFF7E73146FFF7C5FFEEE784
:1042500008B50361C260002343610A460146024873
:10426000FFF7D4FF08BD00BF403A002008B51B4B44
:104270001B69984210D042680368136042685A6014
:104280000268936881680B44936000230360134BBA
:104290004FF0FF329A6108BD1968104A134643F87F
:1042A000101F4B600021016012699A4212D093687E
:1042B00081680B44936000F0FBFA084AD369A0EBD5
:1042C000030C126991686145E5D91B1A1944FFF77F
:1042D00083FFE0E700F0F8FADDE700BF303A0020A6
:1042E000F8B50BE0002383F31188E36821692046C9
:1042F0009847302383F311886369CBB9244D2C6927
:1043000000F0D6FAED69411BA2688A4232D8154402
:104310001F4BDD61616822680A606168516000229C
:10432000226053F8102F9A42DCD100F0CDFAD9E781
:1043300000F0BEFA0746461B6269B2420ED32B1A42
:104340001A44134B53F8101F99420CD0961900D2FF
:10435000324621460F48FFF701FFCFE7022000F069
:10436000FFFA0022EDE713463A4621460948FFF7D7
:104370000DFF0CE0064A52F8101F914207D0044A84
:10438000D061A2682B1A9918A160FFF725FFF8BD2C
:10439000303A0020403A002038B500F089FA054A4A
:1043A000D2E90845031B181945F10001C2E90801CB
:1043B00038BD00BF303A002000207047FEE700BF44
:1043C000704700BF4FF0FF30704700BFBFF34F8F03
:1043D000024B1B6913F4803FFAD170470020024062
:1043E000014BF3221A6170470020024008B50B4BC5
:1043F0001B7803B108BDFFF7E9FF094B5B69002B90
:1044000005DB074A136823F480631360F2E7044B6B
:10441000044A9A6002F188329A60F2E7A03A0020DA
:10442000002002402301674508B50C4B1B7803B1FF
:1044300008BDFFF7CBFF0A4B5A6942F000425A61B0
:104440001A6842F480521A601A6822F480521A6084
:104450001A6842F480621A60EAE700BFA03A0020BE
:10446000002002402DE9F04112F0070F0FD1054660
:104470000C46164610F0070F09D102442D4B9A4204
:104480000FD92D4B40F287321A60002004E02A4BEE
:1044900040F282321A600020BDE8F081083E083503
:1044A0000834072E08D92B6822689A4204D12B1DA4
:1044B0001B6862689A42F1D00EB90120ECE7FFF761
:1044C00095FFFFF783FF012E2FD9DFF87C800123B2
:1044D000C8F8143023682F4647F8043B63686B60C4
:1044E000FFF774FFD8F8103043F00103C8F810301C
:1044F0000023C8F814302B6822689A4207D13F681D
:104500006368BB4203D1083E08340835DBE70A4B39
:1045100040F2AF321A60094B1D60094B1E60094B17
:104520001C60FFF781FF0020B6E7FFF77DFF012049
:10453000B2E700BF000004089C3A0020983A00202F
:10454000943A0020903A0020002002407F2803D8AF
:1045500000F58030C0027047002070474FF40060C3
:10456000704700BF802070477F2811D838B50546B6
:10457000FFF7ECFF04462846FFF7F0FF30B1236851
:10458000B3F1FF3F06D104380434F7E7012038BD0A
:10459000002070470020FAE77F2801D900207047EB
:1045A00038B50446FFF712FFFFF720FFFFF718FFAB
:1045B0000E4B02225A615A6942EAC4025A615A6990
:1045C00042F480325A61FFF701FF2046FFF7BEFF39
:1045D00005462046FFF7C2FF0146284600F000F9D5
:1045E000FFF722FF2046FFF7BFFF38BD0020024043
:1045F00008B5FFF737FF08BD08B548B1094B1B7870
:1046000003B108BDFFF7F2FE064B01221A70F8E76E
:10461000044B1B78002BF4D0024B00221A70FFF7DA
:1046200003FFEEE7A03A002010B5002404B110BD4E
:10463000064804EB44039A00134603445968805823
:1046400000F0D0F80134E4B2F0E700BF7C5000087D
:1046500008B50846114600F03BFC08BD08B5084601
:1046600000F03EFC08BD00BF302383F31188704783
:10467000002383F311887047302383F31188704738
:10468000002383F311887047FFF786BE38B5EFF338
:104690001183D3B9EFF30583C3F3080353B9FFF7CD
:1046A000E3FFFFF7F1FF05460C46FFF7E1FF284661
:1046B000214638BDFFF7E0FFFFF7E6FF05460C4651
:1046C000FFF7DEFF2846214638BDBDE83840FFF73A
:1046D000DBBF00BF38B5FFF7D9FF104C104AC00848
:1046E00040EA4170A0FB025EC908A0FB040C1CEB71
:1046F00005004FF00003A1FB04455B410019A1FB3D
:10470000021043EB050311EB0E0140F100005B18B2
:1047100040F100001B0943EA007038BDCFF753E3B6
:10472000A59BC42009E000F1010C064A52F82020A4
:1047300041F8042B1A465FFA8CF0531EDBB2002AB4
:10474000F1D170475028004010B4144BD3F890308A
:1047500013F4004F0AD1114BD3F89040C3F89040A6
:10476000D3F8904044F40044C3F890400C4C2368C4
:1047700043F48073236009E000F1010C51F8044B0D
:10478000084A42F820401A465FFA8CF0531EDBB20A
:10479000002AF1D15DF8044B704700BF00100240C1
:1047A000007000405028004000B583B0012201A9EC
:1047B0000020FFF7B7FF019803B05DF804FB00BFCE
:1047C00010B582B00446FFF7EFFFA04201D102B05E
:1047D00010BD0194012201A90020FFF7B5FFF6E703
:1047E000704700BF704700BF704700BF074B45F2DE
:1047F00055521A6003225A6040F2FF729A604CF6DA
:10480000CC421A60024B01221A70704700300040FF
:10481000A13A0020034B1B781BB1034B4AF6AA2296
:104820001A607047A13A002000300040054B1B6819
:104830003BB903F1804303F50433D3F89420014BD3
:104840001A607047A43A0020024B4FF40002C3F8EC
:10485000942070470010024008B5FFF7E7FF024BB5
:104860001868C0F3407008BDA43A0020704700BF2C
:10487000FEE700BF084B094903E051F8042B43F859
:10488000042B074A9342F8D302E0002243F8042B9A
:10489000044A9342F9D37047283B0020485100084E
:1048A000283B0020283B002008B500F0AFF808BDE9
:1048B0004FF08043586A70474FF08043586300229E
:1048C0001A610222DA6070474FF080430022DA60FA
:1048D000704700BF4FF0804358637047FEE700BF4A
:1048E00070B586B004460E46194B586000258562A7
:1048F0000163FFF7ADFA24606460A560E56204F12E
:104900001003236163614FF0FF33A361E561FFF79B
:10491000CFFF02462B46C4E90823256580230D4AB4
:1049200004F134012046FFF7D3FBE0600123037557
:10493000094A009272680192B26802920393074B8F
:10494000049305956846FFF7E5FB06B070BD00BF10
:10495000883A0020B84F0008C04F0008DD48000822
:10496000024AD36A0343D362704700BF303A002043
:104970004B6843608B688360CB68C3600B6943619D
:104980004B6903628B6943620B680360704700BF29
:1049900010B5124BDA6A42F00702DA62DA6A22F0E4
:1049A0000702DA62DA6ADA6C42F00702DA64DA6E77
:1049B00042F00702DA66DB6E094C21464FF0904068
:1049C000FFF7D6FF04F11C010648FFF7D1FF04F101
:1049D00038010548FFF7CCFF10BD00BF00100240B2
:1049E00088500008000400480008004808B5FFF798
:1049F000CFFF00F0A9F808BD08B500F049FAFFF7AD
:104A000035FBFFF713FF08BD704700BF0F4B9A6DD2
:104A100042F001029A659A6F42F001029A679B6F19
:104A20000B4A936843F0010393604FF080434F2299
:104A30009A624FF0FF32DA6200229A615A63DA60BA
:104A40005A6001225A611A60704700BF001002408C
:104A5000002004E008B54FF080421369D168C9B264
:104A60000B40D943116113F0020F00D108BD302370
:104A700083F31188FFF728FB002383F31188F5E700
:104A80000C4A136823F0F00343F0600313601368CB
:104A900043F001031360074B1B6813F0020FFAD0B9
:104AA000044B00229A60034B9B6813F00C0FFAD161
:104AB000704700BF001002400D4B61221A600C4B82
:104AC0001B6813F0020FFAD0094B00229A60084BC2
:104AD0009B6813F00C0FFAD1054A69231360D2F8D2
:104AE000943023F4706343F4C063C2F89430704789
:104AF00000100240064B074ADA601A6842F08072E2
:104B00001A60034B1B6813F0007FFAD0704700BF98
:104B10000010024023140001064B074A1A611A686C
:104B200042F080621A60034B1B6813F0006FFAD0EA
:104B3000704700BF00100240200C100008B5FFF7BE
:104B4000D7F900F083F908BD10B5484B9A6A4FF0C9
:104B5000FF3199629A6A00229A62986AD86A60F074
:104B60000700D862D86A00F00700D862D86A186BCC
:104B70001963186B1A63186B986B9963986B9A6337
:104B8000986BD86BD963D86BDA63D86B186C1964DF
:104B9000196C1A641A6C364A4FF4E06111601A6E8F
:104BA00042F001021A66D3F8802022F00102C3F815
:104BB0008020D3F880209A6D42F080529A659A6FD7
:104BC00022F080529A679B6F2A4B4FF440721A6012
:104BD000284B5B6913F4806FFAD1264B00225A6090
:104BE000FFF74EFF214BD3F8903013F4407F07D0EE
:104BF0001E4B4FF48032C3F890200022C3F890205F
:104C0000FFF75AFF194A136843F4A0231360174BA8
:104C10001B6813F4003FFAD0144CD4F8903023F002
:104C20000323C4F89030FFF765FFFFF775FF0023FB
:104C3000A360114BC4F888300D4A136823F00703B2
:104C400043F0040313600A4B1B6803F00703042BB3
:104C5000F9D1064A936843F003039360034B9B68C2
:104C600003F00C030C2BF9D110BD00BF0010024063
:104C700000200240007000405555013408B5074A35
:104C8000536903F0010353612BB1054B1B6813B14A
:104C9000034A50689847FFF7FFF808BD0004014039
:104CA000A83A002008B5074A536903F0020353618C
:104CB0002BB1054B9B6813B1034AD0689847FFF7A7
:104CC000EBF808BD00040140A83A002008B5074AE7
:104CD000536903F0040353612BB1054B1B6913B1F6
:104CE000034A50699847FFF7D7F808BD0004014010
:104CF000A83A002008B5074A536903F00803536136
:104D00002BB1054B9B6913B1034AD0699847FFF754
:104D1000C3F808BD00040140A83A002008B5074ABE
:104D2000536903F0100353612BB1054B1B6A13B198
:104D3000034A506A9847FFF7AFF808BD00040140E6
:104D4000A83A002010B51A4B5C6904F478725A61D5
:104D500014F0200F05D0174B9B6A13B1154AD06A87
:104D6000984714F0400F05D0124B1B6B13B1114A3A
:104D7000506B984714F0800F05D00E4B9B6B13B10E
:104D80000C4AD06B984714F4807F05D0094B1B6CFC
:104D900013B1084A506C984714F4007F05D0054BB6
:104DA0009B6C13B1034AD06C9847FFF775F810BDA0
:104DB00000040140A83A002010B51F4B5C6904F4C0
:104DC0007C425A6114F4806F05D01C4B1B6D13B1EB
:104DD0001A4A506D984714F4006F05D0174B9B6D1D
:104DE00013B1164AD06D984714F4805F05D0134B69
:104DF0001B6E13B1114A506E984714F4005F05D032
:104E00000E4B9B6E13B10D4AD06E984714F4804F31
:104E100005D00A4B1B6F13B1084A506F984714F422
:104E2000004F05D0054B9B6F13B1044AD06F9847D4
:104E3000FFF732F810BD00BF00040140A83A00207F
:104E400008B5FFF707FEFFF727F808BD08B50621EC
:104E50000846FFF767F806210720FFF763F80621E9
:104E60000820FFF75FF806210920FFF75BF806210D
:104E70000A20FFF757F806211720FFF753F80621FD
:104E80002820FFF74FF807211C20FFF74BF808BD3B
:104E900008B5FFF753FE00F005F8FFF7B5FDFFF783
:104EA00003FD08BD002307E0054A002142F8331046
:104EB00002EBC302516001330F2BF5D9704700BFDD
:104EC000A83A00200B460146184600F043B80000FF
:104ED000024B0A4601461868FFF7BABB18110020BA
:104EE000024B01461868FFF7B9BB00BF181100203C
:104EF00010B501390244904201D1002005E0037849
:104F000011F8014FA34201D0181B10BD0130F2E788
:104F10002DE9F041A3B1C91A17780144044603F101
:104F2000FF3C8C42204601D9002009E00578BD42B3
:104F300004F10104F5D10CEB0405D618A54201D10A
:104F4000BDE8F08115F8018D16F801EDF045F5D0BA
:104F5000E7E7000010B504460448134620B10A46AE
:104F600002202146AFF3008010BD00BF000000000A
:104F7000636F6D2E76696D64726F6E65732E7065EA
:104F8000726970685F626C0040A2E4F16468910627
:104F90000000000041A3E5F26569920700000000EF
:104FA0004261642043414E496661636520696E64D5
:104FB00065782E00633000006D61696E00000000AE
:104FC00069646C6500000000000000000000000043
:104FD000691D000885260008D5250008A51D0008C4
:104FE000B11D000889290008751D0008851D0008ED
:104FF000791D0008811D00087D1D0008E11E0008C4
:10500000891D0008E52A0008312B0008991D0008B9
:10501000512900088000000000800000000080008E
:1050200000FFFF000000000000000000691D0008F4
:10503000552A0008792A00087D2A0008592B000803
:105040008D2A0008751D0008812A0008791D0008B6
:10505000852A00087D1D0008892A0008552A0008B5
:10506000E52A0008312B0008552A0008552A0008B7
:10507000B44F000820380020303A00200001002002
:1050800000FF0000010000000000802A0000000076
:10509000AAAAAAAA00000024FFFF00000000000046
:1050A000009009000000000000000000AAAAAAAABF
:1050B00000000000FFFF00000000000000000000F2
:1050C0000000000000000000AAAAAAAA0000000038
:1050D000FFFF0000000000000000000000000000D2
:1050E0007F050000000000000060030000000000D9
:1050F000FE2A0100D20400001C1100200000000064
:105100000000000068000000D00000000000000067
:10511000000000000000000000000000000000008F
:10512000000000000000000000000000000000007F
:10513000000000000000000000000000000000006F
:105140000000000000000000FFFFFFFFFFFFFFFF67
:10515000FFFFFFFFFFFFFFFFFFFFFFFFFFFFFFFF5F
:10516000FFFFFFFFFFFFFFFFFFFFFFFFFFFFFFFF4F
:10517000FFFFFFFFFFFFFFFFFFFFFFFFFFFFFFFF3F
:10518000FFFFFFFFFFFFFFFFFFFFFFFFFFFFFFFF2F
:10A00000000400203DB20008613B0208BD3A02088E
:10A01000293B0208BD3A0208F53A02083FB200089F
:10A020003FB200083FB200083FB2000869BF020813
:10A030003FB200083FB200083FB200083FB200083C
:10A040003FB200083FB200083FB200083FB200082C
:10A050003FB200083FB2000879EC0208A1EC020808
:10A06000C9EC0208F1EC020819ED0208D9C1020896
:10A07000EDC1020801C2020815C2020829C2020885
:10A080003DC2020851C202083FB200080D2E02086C
:10A09000392E0208492E02083FB2000841ED02089D
:10A0A0003DEE02083FB200083FB200083FB2000890
:10A0B0003FB200083FB200083FB200080DC50208D9
:10A0C00041C602083FB200083FB200083FB2000894
:10A0D0003FB2000815EE020829EE02083FB2000860
:10A0E000A5ED02083FB200083FB200083FB20008E9
:10A0F0003FB200083FB200083FB200083FB200087C
:10A100003FB200083FB200083FB200083FB200086B
:10A110003FB200083FB200083FB200083FB200085B
:10A1200065C2020879C202088DC20208A1C20208F3
:10A13000B5C202083FB200083FB200083FB20008B3
:10A140003FB200083FB200083FB200083FB200082B
:10A15000C9C20208DDC202083FB200083FB20008CF
:10A160003FB200083FB200083FB200083FB200080B
:10A170003FB200083FB200083FB200083FB20008FB
:10A180003FB200083FB200083FB200083FB20008EB
:10A190003FB200083FB200083FB200083FB20008DB
:10A1A00051B80008212A0108E10502080535020816
:10A1B000A53D0208F98B020881AD020800000000ED
:10A1C00040A2E4F164689106CE6E4334B0EF1FED17
:10A1D0000C14030003BEC59300007F05FFFFFFFFC3
:10A1E000FFFFFFFF81F0004102E000BF83F000436A
:10A1F00030B54FEA41044FEA430594EA050F08BF22
:10A2000090EA020F1FBF54EA000C55EA020C7FEAE5
:10A21000645C7FEA655C00F0E2804FEA5454D4EB62
:10A220005555B8BF6D420CDD2C4480EA020281EA2C
:10A23000030382EA000083EA010180EA020281EA64
:10A240000303362D88BF30BD11F0004F4FEA0131B6
:10A250004FF4801C4CEA113102D0404261EB4101C5
:10A2600013F0004F4FEA03334CEA133302D052424B
:10A2700063EB430394EA050F00F0A780A4F1010407
:10A28000D5F1200E0DDB02FA0EFC22FA05F2801841
:10A2900041F1000103FA0EF2801843FA05F3594127
:10A2A0000EE0A5F120050EF1200E012A03FA0EFCA6
:10A2B00028BF4CF0020C43FA05F3C01851EBE371D0
:10A2C00001F0004507D54FF0000EDCF1000C7EEBED
:10A2D00000006EEB0101B1F5801F1BD3B1F5001F2B
:10A2E0000CD349085FEA30004FEA3C0C04F101044A
:10A2F0004FEA445212F5800F80F09A80BCF1004F73
:10A3000008BF5FEA500C50F1000041EB045141EAF4
:10A31000050130BD5FEA4C0C404141EB0101013CBD
:10A3200028BFB1F5801FE9D291F0000F04BF0146AC
:10A330000020B1FA81F308BF2033A3F10B03B3F17E
:10A3400020020CDA0C3208DD02F1140CC2F10C020E
:10A3500001FA0CF021FA02F10CE002F11402D8BF6C
:10A36000C2F1200C01FA02F120FA0CFCDCBF41EA38
:10A370000C019040E41AA2BF01EB0451294330BD07
:10A380006FEA04041F3C1CDA0C340EDC04F11404E4
:10A39000C4F1200220FA04F001FA02F340EA0300BB
:10A3A00021FA04F345EA030130BDC4F10C04C4F101
:10A3B000200220FA02F001FA04F340EA03002946E1
:10A3C00030BD21FA04F0294630BD94F0000F83F42B
:10A3D000801306BF81F480110134013D4EE77FEA0E
:10A3E000645C18BF7FEA655C29D094EA050F08BF5A
:10A3F00090EA020F05D054EA000C04BF194610463B
:10A4000030BD91EA030F1EBF0021002030BD5FEA7E
:10A41000545C05D14000494128BF41F0004130BDA6
:10A4200014F580043CBF01F5801130BD01F00045FA
:10A4300045F0FE4141F470014FF0000030BD7FEA6D
:10A44000645C1ABF194610467FEA655C1CBF0B4668
:10A45000024650EA013406BF52EA033591EA030F7F
:10A4600041F4002130BD00BF90F0000F04BF002177
:10A47000704730B54FF4806404F132044FF00005AA
:10A480004FF0000150E700BF90F0000F04BF002123
:10A49000704730B54FF4806404F1320410F0004589
:10A4A00048BF40424FF000013EE700BF42004FEA84
:10A4B000E2014FEA31014FEA02701FBF12F07F4301
:10A4C00093F07F4F81F06051704732F07F4208BFB8
:10A4D000704793F07F4F04BF41F40021704730B5BF
:10A4E0004FF4607401F0004521F000411CE700BF0B
:10A4F00050EA010208BF704730B54FF000050AE08E
:10A5000050EA010208BF704730B511F0004502D58E
:10A51000404261EB41014FF4806404F132045FEA90
:10A52000915C3FF4D8AE4FF003025FEADC0C18BF39
:10A5300003325FEADC0C18BF033202EBDC02C2F12B
:10A54000200300FA03FC20FA02F001FA03FE40EABD
:10A550000E0021FA02F11444BDE600BF70B54FF0C1
:10A56000FF0C4CF4E06C1CEA11541DBF1CEA13559F
:10A5700094EA0C0F95EA0C0F00F0DEF82C4481EA07
:10A58000030621EA4C5123EA4C5350EA013518BF27
:10A5900052EA033541F4801143F4801338D0A0FB14
:10A5A00002CE4FF00005E1FB02E506F00042E0FBC1
:10A5B00003E54FF00006E1FB03569CF0000F18BFC7
:10A5C0004EF0010EA4F1FF04B6F5007F64F540746F
:10A5D00004D25FEA4E0E6D4146EB060642EAC62102
:10A5E00041EA55514FEAC52040EA5E504FEACE2E6F
:10A5F000B4F1FD0C88BFBCF5E06F1ED8BEF1004F72
:10A6000008BF5FEA500E50F1000041EB045170BDED
:10A6100006F0004646EA010140EA020081EA030131
:10A62000B4EB5C04C2BFD4EB0C0541EA045170BD2D
:10A6300041F480114FF0000E013C00F3AB8014F1A7
:10A64000360FDEBF002001F0004170BDC4F10004F0
:10A65000203C35DA0C341BDC04F11404C4F1200571
:10A6600000FA05F320FA04F001FA05F240EA0200CC
:10A6700001F0004221F0004110EBD37021FA04F602
:10A6800042EB06015EEA430E08BF20EAD37070BDBC
:10A69000C4F10C04C4F1200500FA04F320FA05F01B
:10A6A00001FA04F240EA020001F0004110EBD3701D
:10A6B00041F100015EEA430E08BF20EAD37070BD8D
:10A6C000C4F1200500FA05F24EEA020E20FA04F366
:10A6D00001FA05F243EA020321FA04F001F0004115
:10A6E00021FA04F220EA020000EBD3705EEA430E86
:10A6F00008BF20EAD37070BD94F0000F0FD101F0B5
:10A700000046400041EB010111F4801F08BF013CED
:10A71000F7D041EA060195F0000F18BF704703F02B
:10A720000046520043EB030313F4801F08BF013DB2
:10A73000F7D043EA0603704794EA0C0F0CEA13556E
:10A7400018BF95EA0C0F0CD050EA410618BF52EA28
:10A750004306D1D181EA030101F000414FF000002E
:10A7600070BD50EA410606BF1046194652EA43063C
:10A7700019D094EA0C0F02D150EA013613D195EAB0
:10A780000C0F05D152EA03361CBF104619460AD1F8
:10A7900081EA030101F0004141F0FE4141F4700102
:10A7A0004FF0000070BD41F0FE4141F4780170BDF2
:10A7B00070B54FF0FF0C4CF4E06C1CEA11541DBF57
:10A7C0001CEA135594EA0C0F95EA0C0F00F0A7F859
:10A7D000A4EB050481EA030E52EA03354FEA013186
:10A7E00000F088804FEA03334FF0805545EA131399
:10A7F00043EA12634FEA022245EA111545EA106561
:10A800004FEA00260EF000419D4208BF964244F1F7
:10A81000FD0404F5407402D25B084FEA3202B61A16
:10A8200065EB03055B084FEA32024FF480104FF4EA
:10A83000002CB6EB020E75EB030E22BFB61A75465E
:10A8400040EA0C005B084FEA3202B6EB020E75EBF1
:10A85000030E22BFB61A754640EA5C005B084FEA59
:10A860003202B6EB020E75EB030E22BFB61A754626
:10A8700040EA9C005B084FEA3202B6EB020E75EB31
:10A88000030E22BFB61A754640EADC0055EA060EF2
:10A8900018D04FEA051545EA16754FEA06164FEA35
:10A8A000C30343EA52734FEAC2025FEA1C1CC0D1E1
:10A8B00011F4801F0BD141EA00014FF000004FF06E
:10A8C000004CB6E711F4801F04BF01430020B4F12F
:10A8D000FD0C88BFBCF5E06F3FF6AFAEB5EB030CE7
:10A8E00004BFB6EB020C5FEA500C50F1000041EBE4
:10A8F000045170BD0EF0004E4EEA113114EB5C04B1
:10A90000C2BFD4EB0C0541EA045170BD41F4801183
:10A910004FF0000E013C90E645EA060E8DE60CEA8B
:10A92000135594EA0C0F08BF95EA0C0F3FF43BAFA8
:10A9300094EA0C0F0AD150EA01347FF434AF95EA5F
:10A940000C0F7FF425AF104619462CE795EA0C0F43
:10A9500006D152EA03353FF4FDAE1046194622E710
:10A9600050EA410618BF52EA43067FF4C5AE50EAEA
:10A9700041047FF40DAF52EA43057FF4EBAE12E7DA
:10A980004FF0FF3C06E000BF4FF0010C02E000BFBB
:10A990004FF0010C4DF804CD4FEA410C7FEA6C5C9E
:10A9A0004FEA430C18BF7FEA6C5C1BD001B050EA41
:10A9B000410C0CBF52EA430C91EA030F02BF90EA2C
:10A9C000020F0020704710F1000F91EA030F58BFEB
:10A9D000994208BF90422CBFD8176FEAE37040F04D
:10A9E000010070474FEA410C7FEA6C5C02D150EAEB
:10A9F000013C07D14FEA430C7FEA6C5CD6D152EAA6
:10AA0000033CD3D05DF8040B704700BF844610466A
:10AA100062468C461946634600E000BF01B5FFF769
:10AA2000B7FF002848BF10F1000F01BD4DF808ED39
:10AA3000FFF7F4FF0CBF012000205DF808FB00BF0A
:10AA40004DF808EDFFF7EAFF34BF012000205DF864
:10AA500008FB00BF4DF808EDFFF7E0FF94BF0120B1
:10AA600000205DF808FB00BF4DF808EDFFF7CEFFB2
:10AA700094BF012000205DF808FB00BF4DF808EDF1
:10AA8000FFF7C4FF34BF012000205DF808FB00BFC2
:10AA90004FEA410C7FEA6C5C02D150EA013C0AD1DA
:10AAA0004FEA430C7FEA6C5C02D152EA033C02D1CC
:10AAB0004FF0000070474FF0010070474FEA41022D
:10AAC00012F5001215D211D56FF47873B3EB625200
:10AAD00012D94FEAC12343F0004343EA505311F027
:10AAE000004F23FA02F018BF404270474FF00000B9
:10AAF000704750EA013005D111F0004008BF6FF0F7
:10AB0000004070474FF00000704700BF4A0011D26C
:10AB100012F5001211D20DD56FF47873B3EB6252B7
:10AB20000ED44FEAC12343F0004343EA505323FAC3
:10AB300002F070474FF00000704750EA013002D138
:10AB40004FF0FF3070474FF0000070474FEA41026E
:10AB5000B2F1E04324BFB3F5001CDCF1FE5C0DD97B
:10AB600001F0004C4FEAC0024CEA5070B2F1004FC5
:10AB700040EB830008BF20F00100704711F0804FC8
:10AB800021D113F13872BCBF01F00040704741F48D
:10AB900080114FEA5252C2F11802C2F1200C10FA91
:10ABA0000CF320FA02F018BF40F001004FEAC12375
:10ABB0004FEAD32303FA0CFC40EA0C0023FA02F319
:10ABC0004FEA4303CCE77FEA625307D150EA0133EF
:10ABD0001EBF4FF0FE4040F44000704701F00040BF
:10ABE00040F0FE4040F40000704700BF80F000409D
:10ABF00002E000BF81F0004142001FBF5FEA410355
:10AC000092EA030F7FEA226C7FEA236C6AD04FEA54
:10AC10001262D2EB1363C1BFD21841404840414099
:10AC2000B8BF5B42192B88BF704710F0004F40F44B
:10AC3000000020F07F4018BF404211F0004F41F467
:10AC4000000121F07F4118BF494292EA030F3FD033
:10AC5000A2F1010241FA03FC10EB0C00C3F1200346
:10AC600001FA03F100F0004302D5494260EB4000D5
:10AC7000B0F5000F13D3B0F1807F06D340084FEA40
:10AC8000310102F10102FE2A51D2B1F1004F40EB35
:10AC9000C25008BF20F0010040EA0300704749009D
:10ACA00040EB0000013A28BFB0F5000FEDD2B0FA3A
:10ACB00080FCACF1080CB2EB0C0200FA0CF0AABF5D
:10ACC00000EBC25052421843BCBFD04018437047FB
:10ACD00092F0000F81F4000106BF80F40000013201
:10ACE000013BB5E74FEA41037FEA226C18BF7FEAD8
:10ACF000236C21D092EA030F04D092F0000F08BF1A
:10AD00000846704790EA010F1CBF0020704712F000
:10AD10007F4F04D1400028BF40F00040704712F13F
:10AD200000723CBF00F50000704700F0004343F0A4
:10AD3000FE4040F4000070477FEA226216BF0846DA
:10AD40007FEA23630146420206BF5FEA412390EA9D
:10AD5000010F40F4800070474FF0000304E000BF93
:10AD600010F0004348BF40425FEA000C08BF704744
:10AD700043F0964301464FF000001CE050EA010208
:10AD800008BF70474FF000030AE000BF50EA01021D
:10AD900008BF704711F0004302D5404261EB41010A
:10ADA0005FEA010C02BF84460146002043F0B6432F
:10ADB00008BFA3F18053A3F50003BCFA8CF2083A54
:10ADC000A3EBC25310DB01FA02FC634400FA02FC5D
:10ADD000C2F12002BCF1004F20FA02F243EB020064
:10ADE00008BF20F00100704702F1200201FA02FCC6
:10ADF000C2F1200250EA4C0021FA02F243EB0200B9
:10AE000008BF20EADC7070477BB972B90029BEBF69
:10AE100000204FF0004106E008BF00281CBF6FF083
:10AE200000414FF0FF3000F007BAADF1080C6DE9BA
:10AE300004CE002909DB002B1ADB00F095F8DDF8C1
:10AE400004E0DDE9022304B07047404261EB4101B8
:10AE5000002B1BDB00F088F8DDF804E0DDE90223BD
:10AE600004B0404261EB4101524263EB430370473F
:10AE7000524263EB430300F077F8DDF804E0DDE9CC
:10AE8000022304B0404261EB41017047524263EB40
:10AE9000430300F069F8DDF804E0DDE9022304B0C3
:10AEA000524263EB4303704753B94AB9002908BFC4
:10AEB00000281CBF4FF0FF314FF0FF3000F0BCB94D
:10AEC000ADF1080C6DE904CE00F04EF8DDF804E0B9
:10AED000DDE9022304B07047430803F05533C01A7C
:10AEE000830803F0333300F03330184400EB1010C4
:10AEF00000F00F3000EB002000EB0040000E704728
:10AF000007EE900AF5EEC07AF1EE10FA01D400F0E7
:10AF10000BB8F1EE677A08B517EE900A00F004F866
:10AF2000404261EB410108BDD0B5FFF7BFFA0C4BC1
:10AF3000002206460F46FFF711FBFFF7E7FD044628
:10AF4000FFF792FA074B0022FFF708FB02460B4679
:10AF500030463946FFF74AF9FFF7D8FD2146D0BD04
:10AF60000000F03D0000F0412DE9F047089D044647
:10AF70008E46002B4DD18A42944669D9B2FA82F2AC
:10AF800052B101FA02F3C2F1200120FA01F10CFAE8
:10AF900002FC41EA030E94404FEA1C48210CBEFB20
:10AFA000F8F61FFA8CF708FB16E341EA034306FBA9
:10AFB00007F199420AD91CEB030306F1FF3080F038
:10AFC0001F81994240F21C81023E63445B1AA4B285
:10AFD000B3FBF8F008FB103344EA034400FB07F727
:10AFE000A7420AD91CEB040400F1FF3380F00A8168
:10AFF000A74240F207816444023840EA0640E41B5D
:10B0000000261DB1D4400023C5E900433146BDE808
:10B01000F0878B4209D9002D00F0EF800026C5E9AA
:10B02000000130463146BDE8F087B3FA83F6002EC2
:10B030004AD18B4202D3824200F2F980841A61EB3A
:10B04000030301209E46002DE0D0C5E9004EDDE758
:10B0500002B9FFDEB2FA82F2002A40F09280A1EB40
:10B060000C014FEA1C471FFA8CFE0126200CB1FB95
:10B07000F7F307FB131140EA01410EFB03F088428E
:10B0800008D91CEB010103F1FF3802D2884200F21B
:10B09000CB804346091AA4B2B1FBF7F007FB1011AD
:10B0A00044EA01440EFB00FEA64508D91CEB04044B
:10B0B00000F1FF3102D2A64500F2BB800846A4EBA6
:10B0C0000E0440EA03409CE7C6F12007B34022FA91
:10B0D00007FC4CEA030C20FA07F401FA06F31C43C0
:10B0E000F9404FEA1C4900FA06F3B1FBF9F8200CCD
:10B0F0001FFA8CFE09FB181140EA014108FB0EF013
:10B10000884202FA06F20BD91CEB010108F1FF3A62
:10B1100080F08880884240F28580A8F1020861446E
:10B12000091AA4B2B1FBF9F009FB101144EA01417C
:10B1300000FB0EFE8E4508D91CEB010100F1FF3427
:10B140006CD28E456AD90238614440EA0840A0FBBF
:10B150000294A1EB0E01A142C846A64656D353D095
:10B160005DB1B3EB080261EB0E0101FA07F722FAB9
:10B1700006F3F1401F43C5E9007100263146BDE8E2
:10B18000F087C2F12003D8400CFA02FC21FA03F345
:10B19000914001434FEA1C471FFA8CFEB3FBF7F0C6
:10B1A00007FB10360B0C43EA064300FB0EF69E42EB
:10B1B00004FA02F408D91CEB030300F1FF382FD284
:10B1C0009E422DD9023863449B1B89B2B3FBF7F62C
:10B1D00007FB163341EA034106FB0EF38B4208D905
:10B1E0001CEB010106F1FF3816D28B4214D9023E46
:10B1F0006144C91A46EA004638E72E46284605E764
:10B200000646E3E61846F8E64B45A9D2B9EB020834
:10B2100064EB0C0E0138A3E74646EAE7204694E7C4
:10B220004046D1E7D0467BE7023B614432E73046F7
:10B2300009E76444023842E7704700BF02E000F0CB
:10B2400000F8FEE772B6374880F30888364880F386
:10B25000098836483649086040F20000CCF2000008
:10B260004EF63471CEF200010860BFF34F8FBFF38A
:10B270006F8F40F20000C0F2F0004EF68851CEF21F
:10B2800000010860BFF34F8FBFF36F8F4FF00000D6
:10B29000E1EE100A4EF63C71CEF200010860062085
:10B2A00080F31488BFF36F8F23F0A8FA23F0B0FB6C
:10B2B0004FF055301F491B4A91423CBF41F8040BE7
:10B2C000FAE71D49184A91423CBF41F8040BFAE7DE
:10B2D0001A491B4A1B4B9A423EBF51F8040B42F8D5
:10B2E000040BF8E700201849184A91423CBF41F886
:10B2F000040BFAE723F086FA23F0E2FB144C154D19
:10B30000AC4203DA54F8041B8847F9E700F090FADE
:10B31000114C124DAC4203DA54F8041B8847F9E78C
:10B3200023F06EBA00040020000E002000A00008E8
:10B3300008ED00E0000100200004002058B10308DF
:10B34000000E0020B4100020B8100020E05E0020A5
:10B35000A0A10008BCA10008BCA10008BCA1000875
:10B360002DE9F04F2DED108AC1F80CD0C3689D4631
:10B37000BDEC108ABDE8F08F002383F311882846C6
:10B38000A047002022F032FCFEE722F0A9FA00DFFD
:10B39000FEE7000010F8012B11F8013B012A28BF3D
:10B3A0009A42F7D0D01A7047034613F8012B002AAF
:10B3B000FBD1181A0138704701F0FF01102A2BDB6E
:10B3C00010F0070F08D010F8013B013A8B422DD046
:10B3D00010F0070F42B3F6D1F0B441EA012141EA7F
:10B3E000014122F007047FF000070023F0E8025635
:10B3F000083C85EA010586EA010685FA47F5A3FAC5
:10B4000087F586FA47F6A5FA87F68EB9EED1F0BC35
:10B4100001F0FF0102F0070232B110F8013B013ADE
:10B4200083EA010313B1F8D1002070470138704757
:10B43000002D06BF35460338073815F0010F07D138
:10B44000013015F4807F02BF013015F4C03F013098
:10B45000F0BC0138704700BF38B500220023044615
:10B460000D46FFF7EDFA28B920462946BDE83840D9
:10B4700000F00AB8204605F1004100F005F840420E
:10B4800061EB410138BD00BFD0B50C4B0022064630
:10B490000F46FFF763F8FFF739FB0446FEF7E4FFBA
:10B4A000074B0022FFF75AF802460B463046394652
:10B4B000FEF79CFEFFF72AFB2146D0BD0000F03DC1
:10B4C0000000F0417047000070B5044628300BF0D2
:10B4D0003DFD04F1500007F007FC04F5C8700BF0C7
:10B4E00097FF04F526700FF0B7FD04F55C7014F0BB
:10B4F0007FFE04F5D66010F0C3F904F2347002F058
:10B500004DF9154B1549196004F24C7000231426AF
:10B510009DB206FB05120133127C002AF8D1104BB4
:10B520001D80104B1A6812B10F4818F01DFB1860EF
:10B5300004F58053012104F5F950C3F82C2F83F84A
:10B540002A1F103017F018FD084B1A680AB1084876
:10B55000EBE71C60204670BDEC300020BC520308B5
:10B56000EA300020AC30002068510308B8100020F9
:10B5700083510308F7B5454D044623F0F3F823F053
:10B5800005F9286820231A46006C4FF4E13103F0D6
:10B59000C5FD28684FF4807380224FF4E131C06C00
:10B5A00003F0BCFD204600F077F904F1280623F0F3
:10B5B000EDF8204601F040FA30460BF0E5FD23F0AF
:10B5C000E5F816F007F92B68D86A03685B689847B6
:10B5D00010B12F4817F04CFD04F2347004F15007FD
:10B5E00002F0F0F801230DF1070138468DF807301D
:10B5F00007F07CFA94F950306BB194F919100029D6
:10B6000009DB30464FF461330522C9B20BF084FEEA
:10B61000384607F0DBFB04F5C8700CF0FDFD04F5BF
:10B6200026700FF0DFFE204600F05EF994F9D03668
:10B63000C3B194F91030002B14DB092B2A6811DCFC
:10B64000103352F8230068B1E16803F071FD217CEA
:10B65000E368304609220BF05FFE002104F5D66056
:10B6600010F08EFC94F91A30002B09DB092B2A68A4
:10B67000D6BF1033002152F82310204601F030FECF
:10B6800003B0BDE8F04018F097BA00BFD810002012
:10B69000A45103080148FFF76DBF00BFE010002070
:10B6A0002DE9F341144C154EDFF86080144F20460D
:10B6B00022F0C0FF134A0146121B134801F064FA3E
:10B6C00022F030F80446A4B1206AE1690191B04249
:10B6D00014BF251AA8EB060522F0ACFF019902461B
:10B6E0002B46384601F050FA204622F02BF804464B
:10B6F000E9E702B0BDE8F08100010020000400206D
:10B70000CE51030800040020C4510308000E00209D
:10B7100010B50F4C05F000FF2368986A03680522F6
:10B72000DB69002198472368986A036864211B69D4
:10B7300098472368986A036828215B6898472368BC
:10B74000986A0368BDE810401B690021184700BFD4
:10B75000D810002038B5054618F02EFA284A13688C
:10B76000C31AB3F57A7F88BF106004460FF01AFF42
:10B77000244A136841F28831E31A8B4206D90168E2
:10B7800021B114600289204801F0FEF9EB7EDA074E
:10B790000AD51E4A136841F28831E31A8B4203D955
:10B7A00028461460FFF77CFFEB7E9B070CD4184AF9
:10B7B0001368E31A132B20D8284601F069FA2846AB
:10B7C000BDE8384000F06EB918F0F6F943F698235A
:10B7D0009842ECD90F48FFF79BFF0F4822F0D6FEA6
:10B7E000BFF34F8F0D490E4BCA6802F4E06213435A
:10B7F000CB60BFF34F8F00BFFDE71460DCE700BFF5
:10B80000BC100020C4100020E0510308C01000202C
:10B81000C8100020E0100020010007B000ED00E09B
:10B820000400FA050148FFF795BF00BFE0100020B3
:10B8300038B5054B1C6823680A461D68034B014652
:10B840002046A847002038BDD8100020CC1000208A
:10B8500010B50A4C2046FFF737FE094A0949204631
:10B8600023F030FB17F046FE074B084A1860BDE88E
:10B8700010400749074803F06BBB00BFE0100020F1
:10B88000E4400020C5B40008D810002025B8000806
:10B8900095B60008CC10002013B5044606F092FEC1
:10B8A00005F0B0FA204606F00DFE18B1B4F90030EC
:10B8B000022B0BD007F0BEF904F076FF02230DF146
:10B8C00006012046ADF8063007F060F902230DF1BD
:10B8D00006012046ADF8063007F04EF902B0BDE88B
:10B8E000104006F02DBD000010B54269002A14DD9D
:10B8F000037E092B11D809491033096851F82340F8
:10B900005CB110460BF044FB4FF4807301461A46BD
:10B910002046BDE8104003F001BC10BDD810002047
:10B9200030B52DED048B0C46A5B04822002105460C
:10B930000DEB020025F01AFB2368149394F82530D0
:10B94000ADF8543063681693A3681793D4ED037A67
:10B95000238A9FED517A9FED519A08EE103AF8EE46
:10B96000E77AB8EEC88A67EE877A28EE098ACDEDC5
:10B97000187ADFED4B7A28EE278AB0EE480A8DED73
:10B98000198A23F0A5FA638A08EE903AF8EEE88A5D
:10B9900020EE280A20EE090A8DED1A0AB0EE480AB8
:10B9A00023F0CEFAB4F91430B4F916205B4207EE56
:10B9B000903A238BADF87430D4F81B30CDF8763044
:10B9C000D4F81F30CDF87A3028EE800A94F823306E
:10B9D0008DF87E30F8EEE77A002AE38AB8BF0122BC
:10B9E00020EE090A67EE897AB8BF8DF87F2094F8B7
:10B9F00024208DED1B0A9907CDED1C7A8DF880204F
:10BA000005D5A27E002A3CD101228DF8812003F0C9
:10BA100001028DF88220C3F380028DF88320C3F3E6
:10BA2000C0028DF88420C3F300128DF88520C3F383
:10BA300040128DF88620C3F380128DF8872006AC63
:10BA4000C3F3C0128DF88820C3F3002321460122DE
:10BA500012A88DF8893002F029F80023049380B2EF
:10BA600045F236131F22CDE90240CDE900322846C7
:10BA700007A3D3E9002300F055FA25B0BDEC048BF1
:10BA800030BD012AC3D10222BFE700BFAFF300805F
:10BA9000F881690BB65DE4686F12833A0AD7233CDC
:10BAA00035FA8E3C2DE9F04F4369002BD1B00446A6
:10BAB00075DD037E092B72D83A4A1033126852F8AA
:10BAC0002350002D6BD02B68DFF8DC805B692846A3
:10BAD0009847002687B204F5AE6B04F2946AB3B2BD
:10BAE0009F422BD92B6828469B699847CDF800A028
:10BAF000C2B25B465146584616F0C6F901281BD122
:10BB0000D4F87835C3F31723F62B15D194F8739531
:10BB1000B9F1260F28BF4FF0260926220021404602
:10BB200025F024FA04F27C514A46404625F0D4F927
:10BB300041462046FFF7F4FE0136D0E718F03CF806
:10BB4000D4F8AC36C31AB3F57A7F28D300274FF464
:10BB50004072CDE90472032204AB8DF81820C4F8BA
:10BB6000AC0693E807000AAE03C6092332703222FE
:10BB7000CDE9013200939E2204F29463012107A8CB
:10BB80008DF825708DF826708DF8277016F08AF8DC
:10BB90002B680246DB680DF11E012846984751B01C
:10BBA000BDE8F08FD81000202830002070B52DEDB2
:10BBB000028B324B93F908308CB00446002B51D0E5
:10BBC00000F5267007900FF0B3FA94F8A912D4F894
:10BBD0006027242505FB0143D3F8B4329A4241D0B3
:10BBE0000798C4F860370FF06FFB00283AD094F83C
:10BBF000A93205FB034308A9D3F8BC220A92002509
:10BC000001220AA893EDB08A0B9502F059F908AB0E
:10BC100080B20293182640F20443CDE90036039027
:10BC200012A3D3E900230495204600F07BF9DFED51
:10BC3000147A0B9578EE277A012208A90AA8CDED8F
:10BC40000A7A02F059F908AB80B2CDE9016340F2FB
:10BC5000054303900093049506A3D3E900232046EF
:10BC600000F060F90CB0BDEC028B70BD9AC8BD123B
:10BC700034C4C7CD7162D977642A2749E010002007
:10BC800033938843BFF34F8F0549064BCA6802F4CC
:10BC9000E0621343CB60BFF34F8F00BFFDE700BFEF
:10BCA00000ED00E00400FA0513B51022002104465F
:10BCB0008DF8072025F05AF9054B1B68D86A0368F0
:10BCC0000DF107021B6B2146984702B010BD00BF63
:10BCD000D8100020F0B58BB0174604460E4617F07A
:10BCE0006BFF054604F0ACF903464FF4C87005F548
:10BCF000167504F58054B3FBF0F202FB103315FA0D
:10BD000083F3C4F8243FFD7E35B91F4817F0B0F91E
:10BD100084F8285F0BB0F0BD384605A902F08EFC10
:10BD200007460028F6D101A8FFF7BEFF9DF8165080
:10BD300001A92A460DF1170025F0BEF828B11348D5
:10BD400017F096F984F8287FE4E70F2D0CD8D4F883
:10BD5000243F84F8285FA3F51673C4F8243F2946CE
:10BD60000B4817F085F9D5E79DF814100029D1D0BC
:10BD700030461FF00BFC9DF8142094F82A1F05484C
:10BD800017F076F9C6E700BF605403088B54030828
:10BD9000AC540308CE54030807B5104601A902F0BD
:10BDA000FBFA58B9074B9DF804101B68D86AA1F13B
:10BDB000FF02036851421B685141984703B05DF888
:10BDC00004FB00BFD810002038B5084615461C46B5
:10BDD0001FF0E4FB60B99DF81030022B07D1012C55
:10BDE00005D123A3D3E90023C5E90023012038BDF1
:10BDF000282C20D00DD8601E83B20A2B15D80A2813
:10BE000013D8DFE800F0141212121C1212121224BE
:10BE1000200040F24C439C421DD040F6B9339C4276
:10BE200021D040F226439C4219D00020DFE712A324
:10BE3000D3E90023D8E712A3D3E90023D4E712A360
:10BE4000D3E90023D0E712A3D3E90023CCE712A360
:10BE5000D3E90023C8E712A3D3E90023C4E712A360
:10BE6000D3E90023C0E712A3D3E90023BCE700BF56
:10BE7000401DA12026812A0B9E6AC421818A46EE9C
:10BE800026417272DF25D7B7F017304A39059E5622
:10BE9000D5A4D139F922B6A7CDD269EBC51A133B87
:10BEA00003806A5575F30087011517CB0E03561FE3
:10BEB000E9A2A272EAE738B113B59DF81040CDE9C6
:10BEC000003413460A460146806AFFF77DFF02B040
:10BED00010BD000070B500F580560D46D6F8204F15
:10BEE0007CB90C21012022F00BFAC6F8200F08B90A
:10BEF000002070BD056084600430FAE72646A4681F
:10BF000024B12368AB42F9D1201DF2E70C210120B6
:10BF100022F0F6F9B0600028EAD00560B3689C60B2
:10BF2000B068E9E72DE9F04190B000F5F951BDF8AE
:10BF3000587004461646103140F2434201A8984614
:10BF400003F044F8012F0ED146EA07412046FFF7DF
:10BF5000C1FF054670B9002401A803F059F8204636
:10BF600010B0BDE8F08104F5F0601FF017FB002869
:10BF7000EAD1F0E73822002102A824F0F7FF0223DB
:10BF80008DF808309DF85C308DF82030189B0993AF
:10BF9000BDF86430ADF82830CDE90468ADF818700C
:10BFA000079517F00BFE0D4BC01841F10001CDE9CC
:10BFB0000C0104F5F06002A91FF0F2FA084B00280A
:10BFC000D5BF9A881A6801321218D4BF9A801A60B5
:10BFD0000028D4BF00240124BEE700BF40420F0068
:10BFE0005C30002030B58FB014460D463822002159
:10BFF000684624F0BBFFDDE91223CDE90223BDF83A
:10C000005030ADF8103004F119030593A37E8DF87C
:10C010001830159B0793BDF85830ADF8203017F055
:10C02000CDFD0D4BC31841F100016A46CDE90A313F
:10C030002846E17E1FF0F8FA084B0028D5BF9A8801
:10C040001A6801321218D4BF9A801A600028D4BF2F
:10C05000002001200FB030BD40420F005C300020B6
:10C06000F0B591B004460E46104608A9154602F0F8
:10C07000ADFB00283BD19DF82030012B1BD106F0F1
:10C08000D9FD04F091FB06F05BF906F09BFA1C4920
:10C0900004F1500006F0CAF91A4904F5C87006F018
:10C0A000C5F9194904F5267006F0C0F9174904F5D9
:10C0B000D66006F0BBF91022002106AF0CA824F0D0
:10C0C00055FF012239460CA88DF8382002F0A2FB5A
:10C0D0000A23029308A3D3E9002380B2CDE90370B9
:10C0E000CDE9002331462A462046FFF77BFF11B0F9
:10C0F000F0BD00BFAFF30080CDD269EBC51A133B92
:10C10000805C030824680308786D0308E86F03085F
:10C110002DE9F041ADF5487D66AC05460E46174663
:10C1200000214FF4C472204624F020FF17F044FD94
:10C130002F4B4FF47A72B0FBF2F0186093E80700CF
:10C1400084E8070002F0AAFD037C237402F0A6FD38
:10C15000437C63740323A374264B5A6962610DF513
:10C16000DD709A68DB68A261E361FFF79DFD47F629
:10C170000573EA692384204B002A18681F4B29DDC8
:10C18000CDE900320DF2CB211D4BC06A502203F0E5
:10C19000A7F850210DF2CB2025F0D4FB0DF11C089F
:10C1A00084F8320141460122204602F00FF90123B2
:10C1B00002930DA3D3E9002380B2CDE90380CDE93A
:10C1C000002331463A462846FFF70CFF0DF5487D1F
:10C1D000BDE8F081009350220A4BC06A0DF2CB21DA
:10C1E00003F07EF8D5E700BF9E6AC421818A46EE3F
:10C1F00050300020C0A10008D8100020F3540308DC
:10C20000EC540308A26303082DE9F0411546ADF58F
:10C21000866D06460F4622F0B9FA08A9284602F0B4
:10C220000FFB0446002840F09F8001464FF4D07277
:10C23000A4A824F09BFE9DF8B880B8F1100F7ED81A
:10C2400008F1FF330F2B2BD842460DF1B9010DF247
:10C25000D13024F041FE424651490DF1B90025F09C
:10C2600049FB0246B0B94F480DF11F0104F0B8FF79
:10C270000446002C63D09DF8B83073B39DF8283085
:10C280005BB39DF81F20013A032A6DD8DFE802F066
:10C290001C2E384122460DF11F010DF2D130E5E789
:10C2A000BDF82000479447AA0DF11F0105F0AAFB35
:10C2B0000446002843D0012300930DF2D13211230C
:10C2C00047A904F0C9FED4E7012B4DD10C9B8DF892
:10C2D0001C3147A9204606F03BFC9DF81F30013B6E
:10C2E000032B41D8DFE803F01C444A4F012B3BD11C
:10C2F0000C9BADF81C3147A9204606F061FCECE729
:10C30000012B31D10C9B479347A9204606F082FCB4
:10C31000E3E7022B28D10CA9204606F0D3FBDCE78B
:10C3200001238DF8903294F90030DA17CDE9A63266
:10C330005C210DF2D13025F005FB8DF8D00347AC20
:10C3400001222146A4A802F0A3FB0B23029312A30F
:10C35000D3E9002380B2CDE90340CDE9002339467B
:10C360002A463046FFF73EFE0DF5866DBDE8F081AA
:10C3700001238DF89032B4F90030D6E701238DF80F
:10C3800090322368D1E702238DF890322368A69378
:10C39000CEE700BFAFF30080D5A4D139F922B6A70C
:10C3A00010550308195503082DE9F04FDFF8D8A000
:10C3B0008BB0804608F5F06948461FF071F90546D4
:10C3C000002858D00024007E0694CDE90744ADF83B
:10C3D000244002F081FD2A7E8DF8240005F1100131
:10C3E00007A824F079FD2B6843F00043069317F06B
:10C3F000E5FB224B0390C218DAF804000E4641F127
:10C40000000308F5805760B30168009409690D4680
:10C4100006A9A847A04224DCDAF8040003689B6A56
:10C420009847D0E90A23CDE9042317F0C7FBDDE9DB
:10C430000423801A61EB0301114B834274EB010367
:10C440000FD397F8293F072B12D90E4A87F8294FA7
:10C450009388013393804846039A33461FF02EF9A0
:10C4600009E048461FF020F9002387F8293FA1E79B
:10C47000013387F8293F0BB0BDE8F08F40420F0031
:10C480007F841E005C3000207C3000202DE9F041CC
:10C490004FF00053DFF8E0801B684345FCB00546D1
:10C4A0000C46164604D03148DC22002124F05EFD03
:10C4B0004FF0005749A9C7F80080304602F00AF94A
:10C4C000002849D19DF824313B750BB9F37E3B75AB
:10C4D0009DF8252126480DF5937124F0FDFC20469A
:10C4E0001FF05CF84FF0005307AF58758122002110
:10C4F00028A824F03BFD3946012228A802F030F993
:10C500002823029317A3D3E9002380B2CDE9037057
:10C51000CDE90023214632462846FFF763FD154F3B
:10C520003326013E16F0FF06284608D0FFF73CFFF1
:10C530003B68986A036801215B689847F1E7FFF759
:10C54000E7F820461FF02AF840F0304040F4002081
:10C5500022F01CF8FFF796FB7CB0BDE8F08100BF2D
:10C56000AFF3008026417272DF25D7B704000020A8
:10C5700016000020D81000209AAD44C5F0B504463E
:10C5800089B008460E4615461FF008F868B92B7E9C
:10C59000022B28D1EB8A012B25D12A463146204691
:10C5A00009B0BDE8F040FFF795BBEB8A282B24D0FB
:10C5B0000DD8013B9AB20A2A15D80A2B13D8DFE806
:10C5C00003F01412121224121212124D450040F2FE
:10C5D0004C4293424AD040F6B932934256D040F290
:10C5E000264293424AD009B0F0BD2A463146204641
:10C5F00009B0BDE8F040FFF78BBD2A463146204622
:10C6000009B0BDE8F040FFF741BF07AF254816F07D
:10C610002FFD0122394606A88DF8182001F0B0FF41
:10C62000052302931DA3D3E9002380B2CDE90023A3
:10C63000CDE903702A4631462046FFF7D3FC17F0B8
:10C64000BBFA04F58054C4F82C0FCCE72A463146D7
:10C65000204609B0BDE8F040FFF7D6BD2A46314676
:10C66000204609B0BDE8F040FFF7FABC2A46314643
:10C67000204609B0BDE8F040FFF78EBB2A463146A0
:10C68000204609B0BDE8F04000F000BC2A46314623
:10C69000204609B0BDE8F04001F0CAB8F017304AB2
:10C6A00039059E56245503080A460146806AFFF75D
:10C6B00065BF000049421B4B112912D8DFE801F089
:10C6C0000911110D1111111111111519151D212526
:10C6D000292D9A6801329A6070479A8901329A81AD
:10C6E0007047DA890132DA8170475A8B01325A83F6
:10C6F00070471A8B01321A8370471A8A01321A82E4
:10C7000070475A8A01325A8270479A8B01329A8353
:10C7100070479A8A01329A827047DA8A0132DA8245
:10C72000704700BF5C3000202DE9F04F374E97B0C6
:10C730000023CDE90B330A93ADF834307368044617
:10C74000002B5FD0324D01274FF0000A4FF0000B55
:10C7500070688DF814704FF000088DF8158003682C
:10C76000CDE900AB0DF11502D3F8089005A94346B9
:10C77000C8479DF81430002B44D0414620220EA813
:10C7800024F0F4FB7068036806AAD3F814800AA9A1
:10C790000DF11603C047002834DD9DF8340002F087
:10C7A000B7FB0BA902468DF8500012A824F094FBA9
:10C7B00004F5F0680A9B0E930EA9DDE906234046B6
:10C7C0001FF0AAF910F10D0F014603D02046FFF724
:10C7D00071FFBDE70E981FF08FF903900E981FF0C0
:10C7E00085F9039BCDE9000708AA41462046FFF7DB
:10C7F000EBFA18B12B8A01332B82A9E76B8B01333B
:10C800006B83A5E717B0BDE8F08F00BF7C30002038
:10C810005C30002007B500F5F06168461FF030F984
:10C82000BDF8040064235843BDF80030B0FBF3F0BA
:10C8300080B203B05DF804FBF0B597B0044617F082
:10C84000BBF94FF47A73B0FBF3F0434B434D1B68D5
:10C850002860D86A03685B6D98474FF6FF7398426B
:10C8600028BF184628810EA90122284601F060FE43
:10C870000EAB80B20293182240F255130025CDE989
:10C88000003203902EA3D3E9002304952046FFF73E
:10C8900049FBE37E59074ED501220EA93048314F9E
:10C8A00001F068FA0EAB80B202931F264FF4AB730F
:10C8B000CDE90036039024A3D3E900230495204654
:10C8C000FFF730FB786803689B6A9847002832D0EE
:10C8D0003A788DF8382002680F924268ADF840200F
:10C8E0008268ADF84220C268ADF844200269ADF814
:10C8F00046204269ADF8482082691392C269ADF8BA
:10C900005020026AADF8522007AF436AADF85430A8
:10C91000012239460EA801F0D7F940F2571380B230
:10C92000CDE902700093049509A3D3E90023019691
:10C930002046FFF7F7FA17B0F0BD00BFAFF3008055
:10C94000F1C6A7C1D068080FD1F886A9B8E33A7636
:10C95000753CA33CAE0C08CED8100020503000200F
:10C960005C3000207C300020F0B506468DB000F52C
:10C97000F0601EF013FE2E4D20B100232B7001201D
:10C980000DB0F0BD17F018F92B7804463BB13046D6
:10C99000FFF740FF01210246264816F069FB03F02D
:10C9A0004FFB4FF4C87306F58057B0FBF3F202FB60
:10C9B000130304F5167010FA83F000238DF8183075
:10C9C00097F8283FC7F8240F23B901228DF81820C3
:10C9D00087F82A3F08A8FFF767F997F8281FC1F1E1
:10C9E0001004E4B2062C28BF062408AB22461944E2
:10C9F0000DF1190024F070FA013406AB0025029302
:10CA000018220123E4B2CDE90032049506A3D3E94C
:10CA1000002303943046FFF785FA87F8285F2846FD
:10CA2000AEE700BFAFF30080401DA12026812A0B96
:10CA3000000E00203455030870B5244D244E4FF4E9
:10CA4000807386B0AB80044617F0B6F84FF47A7363
:10CA5000B0FBF3F028606288B4F902307F2A98BFF7
:10CA600033700DF11701002304F109008DF8173020
:10CA700006F06EF841F2381002F014F9054608B1DC
:10CA800015F01CFE134B1D60134B00225D601A70E5
:10CA90002DB12B6861685B680122284698470F4BCF
:10CAA000009304F5F06004F5F6610D4B019441F23A
:10CAB000707203901EF03EFD3178039821B106B0EC
:10CAC000BDE870401EF062BD06B070BD5030002061
:10CAD00091300020843000207C300020B9BE000856
:10CAE000A9C6000830B50628134698BF1D4AC7B02E
:10CAF00098BF155C07930C464FF07C024FF0000185
:10CB000027A888BF002524F031FA079B22465A2126
:10CB10000DF1BE0016F068FA5A2828BF5A2008AC5A
:10CB20008DF8BD002146012227A88DF89C5001F008
:10CB300031FD0023049380B243F6FF731822CDE940
:10CB40000240CDE90032084804A3D3E90023FFF7EF
:10CB5000E9F947B030BD00BFAFF30080759D040C0C
:10CB60008EA454D6F0550308E01000200EB403B58F
:10CB700003AA52F8041B0192FFF7B4FF02B05DF85C
:10CB800004EB03B0704700000FB407B504AA0720F8
:10CB900052F8041B0192FFF7A5FF03B05DF804EB08
:10CBA00004B0704737B5044600F5F0601EF086FD0E
:10CBB0002046FFF72FFE462802D92B4816F058FAD8
:10CBC0002046FFF739FE94F90950002D38D0002394
:10CBD00004F10900EDB201A98DF8043005F0B8FFA9
:10CBE0002A2D224C0AD1224D2846FFF7CDFF23687B
:10CBF000986A036864215B689847F5E72B2D04D198
:10CC00001C48FFF7C1FF1C4B98474FF4FA6101A87D
:10CC100002F0C2F92468A06A03684FF47A715B6875
:10CC20009847E06A03689B6A984718B1012816D0B4
:10CC3000124800E01248FFF7A7FF01A802F0B8F978
:10CC4000104B00225A7116F0B7FF47F2305398424A
:10CC500007D90D4803B0BDE8304021F097BC0B4820
:10CC6000E9E703B030BD00BF6C550308D8100020C1
:10CC70008A5503089B55030838ED00E0D655030894
:10CC8000AB55030850300020263A09B0C0550308C0
:10CC90002DE9F341044616F08FFF3A4A1368C31A90
:10CCA000322B054609D9384B1B7833B13749106010
:10CCB0000B78013303F01F030B7004F5805616F058
:10CCC0007BFFD6F8243F984202D92046FFF74CFE5E
:10CCD0002F4A1368EB1AB3F57A7F07D3156016F065
:10CCE0006DFF02460B462046FFF75CFF204600F032
:10CCF0005FF8204600F0DEF8204600F045FE2046B2
:10CD0000FEF754FF204600F0B9FC204600F0A6FCD8
:10CD100016F050FF04F5F955DFF878800746103516
:10CD200016F048FFC01BB0F57A7F17D2D8F8003054
:10CD3000986A03684FF480619B68984740F2D77205
:10CD4000294601A802F042F92046FFF72DFB2046B4
:10CD5000FFF7EAFC01A802F05BF9E1E7D6F82C3F07
:10CD600063B116F029FFD6F82C3FC01AB0F57A7FD0
:10CD700004D92046FEF7CCFCFEF784FF02B0BDE8E4
:10CD8000F08100BF8C300020000E00209030002089
:10CD900088300020D810002010B590F80611044605
:10CDA0000AF06EFB6423C0B203FB0044A06E10BD0A
:10CDB00070B52DED048B90F995319EB00446002B93
:10CDC00058D090F89432002B54D016F0F5FED4F8D9
:10CDD0005037C01A27284DD904F5C87528460AF0DF
:10CDE00077FB2846D4F85067FFF7D6FF864241D03C
:10CDF00094F8961228460AF065FB00283AD0284697
:10CE0000FFF7CAFF94F89612C4F8500728460AF0B4
:10CE100037FB6423C0B203FB00409FED1B0A00F503
:10CE2000F67003F069F90AAD2822002114A8B0EECB
:10CE3000409AF0EE608AB0EE418A24F097F8012221
:10CE4000294611A88DED119ACDED128A8DED138A28
:10CE500000F0ECFF002380B21822049340F2E93383
:10CE6000CDE90250CDE90032204605A3D3E90023E5
:10CE7000FFF758F81EB0BDEC048B70BDAFF3008017
:10CE8000F2C20B46A9D4A7E26F12833A10B5A2B042
:10CE900001A90446104601F0E3F9014638B99DF8AE
:10CEA00005300DF1060204F1500006F017FC22B027
:10CEB00010BD00002DE9F04390F95030ADF52D7D07
:10CEC0000446002B00F0EF8100F15005284606F0E3
:10CED0001BFB94F86061D4F8542704EB0613D3F8D5
:10CEE0009C309A4200F0DF81C4F854374FF4D0727E
:10CEF000002144A824F03AF894F8883133B9B023DB
:10CF000003FB064393F8A930012B0CD894F86477FF
:10CF10004FB916F053FE00220023CDE94401CDE9BC
:10CF20004623002313E0012384F864373146284662
:10CF300005F0ACFFCDE9440194F86011284606F0F5
:10CF400001F850EA0103CDE94601EAD00223B022FC
:10CF500002FB06428DF82031D2F8C0100A2381FB73
:10CF60000310CDE94A10D2F8BC10D2F8B82081FBEA
:10CF70000310CDE94C10534394F8601108AA2846D9
:10CF8000CDE94E3306F074FB78B14E9BDDED086AB7
:10CF90009FED4F7A079307EE903AF8EEE77AE6EEC8
:10CFA000C77AFDEEE77ACDED4E7AB02303FB065249
:10CFB00003FB06468C32D6F8DC1050915168519133
:10CFC00094F860119268529203FB014393F8DA20BF
:10CFD0008DF84C2193F8A92094F888313BB9062AA2
:10CFE0000AD8DFE802F004045D6163696E00002383
:10CFF0008DF84D31ADF84E31062309AA28468DF83B
:10D00000503105F02FFF38B1DDED097A67EEA77AD0
:10D01000CDED567ACDED557A94F860110AAA2846DE
:10D0200005F02AFF28B1DDED0A7A67EEA77ACDED8B
:10D03000577A0BAF94F860113A46284605F008FF7E
:10D0400048B1D7ED007A67EEA77ACDED5A7ACDEDEB
:10D05000597ACDED587A9DF850119FED1E7A1E48F1
:10D06000DFED1E6A9FED1E6A55AB0022D6B2B142BB
:10D0700038D9D3ED007AF0EEE75AF4EE475AF1EEE4
:10D0800010FA09DCF4EEE67AF1EE10FA04D9F4EEC7
:10D09000C67AF1EE10FA00DB186001320433E5E7DE
:10D0A00002228DF84D21A5E70322FAE703238DF82C
:10D0B0004D3140F201139DE703238DF84D310223DA
:10D0C00098E703238DF84D314FF4817392E700BF49
:10D0D00000007A44FFFF7F7F0000C07F00EF7FC722
:10D0E00000EF7F470CAE3146012244A800F09CFFC0
:10D0F0004FF0000880B240F227434FF01809CDE905
:10D100000260CDE90039CDF8108073A3D3E9002384
:10D110002046FEF707FF2022414644A823F026FFC1
:10D1200094F86031DFED696AB02202FB03433146B7
:10D13000B3F8D620B3F8D83007EE102A07EE903AAD
:10D14000B8EEC77AF8EEE77A27EE267A67EEA67A87
:10D15000012244A88DED467ACDED477A00F0EEFE2F
:10D1600040F2254380B2CDE902600093CDF81080F3
:10D1700050A3D3E90023CDF804902046FEF7D2FE59
:10D1800094F86011CDF818812846CDE9448806F05E
:10D190003DFA94F972308DF814013BB1284606F03F
:10D1A00045FA18B9469B43F0010346939DF81431A4
:10D1B00043B10AA9284606F0CFF918B9469B43F0B7
:10D1C0000203469394F860113A46284606F046FA60
:10D1D00008B13B6844930122314644A800F058FD51
:10D1E0000023049380B244F623634FF01809CDE97D
:10D1F0000260CDE90039204630A3D3E90023FEF7D1
:10D2000091FE94F88931002B4DD194F86011B02330
:10D2100003FB014393F8FC30002B44D0D4F85C8727
:10D22000B8F1000F3FD100970AAB09AA284606F0D3
:10D23000EBFAC0B33B68D4F858279A4233D0DDEDFF
:10D240000A7A9FED237ADFED236AC4F85837F4EEAB
:10D25000C77A9DED097AADF812810122F1EE10FA3C
:10D2600027EE267A67EEA67AACBF13460023314636
:10D2700044A88DF810218DF811318DED457ACDED52
:10D28000467A00F0D7FC44F6226380B2CDE9026012
:10D290000093CDF810800BA3D3E90023CDF80490C0
:10D2A0002046FEF73FFE0DF52D7DBDE8F08300BF63
:10D2B000AFF30080D2BFDBC3C4BDE89B697F00BB76
:10D2C000ABB43CBA1234EDEC39AE5C310AD7233C36
:10D2D0000000003435FA8E3C5F43370F00E741CA47
:10D2E0000346084659B10222C3F8881483F858252A
:10D2F0004FF400731A464FF4E13101F00FBF70474D
:10D300002DE9F0431C4685B003F110051733904614
:10D31000DB086A46A2EBC30300AF9D46064689467A
:10D320002A460021684623F021FE6D440023224650
:10D3300041463846C7E90233C7F800D07D60A7F8F8
:10D34000089013F087F86946384613F07FF839469D
:10D350000123022206F5916012F094FF1437BD46B6
:10D36000BDE8F08370B52DED028B90F95030A0B080
:10D370000446002B00F0D780D0F89C30D0F8602510
:10D380009A4200F0D08000F15005C0F860350021CD
:10D39000B0F8B030ADF84D3028468DF84C1006F09E
:10D3A00055F994F8882194F8A930CDF84F0012B1BE
:10D3B000012B88BF012300268DF8533002AA94F870
:10D3C000DA308DF8543000212846029603960496F0
:10D3D00005F048FD03AA0021284605F04DFD04AAEA
:10D3E0000021284605F034FD9FED548ADDED047AD6
:10D3F00094ED320A67EE887A20EE080AFCEEE77AAE
:10D4000017EE903ADDED027AADF8593067EE887A82
:10D41000FCEEE77A17EE903ADDED037AADF8553081
:10D4200067EE887AFCEEE77A17EE903AD4ED377A19
:10D43000ADF8573067EE887AB4F8D630ADF85B3087
:10D44000D4F8C030CDF85D30FDEEE77AD4F8BC30CA
:10D45000CDF86130D4F8B830CDF8653017EE903A99
:10D46000D4ED387ACDF8693067EE887AFDEEE77A48
:10D4700017EE903AD4ED397ACDF86D3067EE887AB0
:10D48000FDEEE77A17EE903ACDF8713002F084FDA8
:10D49000BCEEC00A05AA10EE103AADF8753007AB25
:10D4A0000093002106AB2846059606F0ADF900284A
:10D4B0003DD09DED050A20EE080A02F06DFDBCEEA0
:10D4C000C00A10EE103AADF877300021284605F07A
:10D4D000DDFC00231A4AFDF7E7FC2422CDE9080110
:10D4E00000210AA823F042FD0AA908A823F028FC7D
:10D4F000436903F26C73ADF8793003698DF87B30C2
:10D50000C3688DF87C3083688DF87D3043688DF872
:10D510007E3003688DF87F3013AA342341F60371FF
:10D520002046FFF7EDFE20B0BDEC028B70BD4FF042
:10D53000FF338DF877308DF87830C6E70000C842A9
:10D5400040420F001FB5D0F86425D0F8B4329A429B
:10D5500004462BD090F8A91200F526700DF0B4FE09
:10D5600020B3D4F8B432C4F864350022CDF80530C5
:10D5700094F8A9328DF80420242202FB0343D3ED52
:10D58000B07A9FED0B7AD3F8BC22CDF8092067EE74
:10D59000877A01AAFDEEE77A41F6057117EE903A17
:10D5A0002046ADF80D300B23FFF7AAFE04B010BDE6
:10D5B0000000C8422DE9FF4100F5C8770025D0F8EA
:10D5C000688504462946384609F05AFF6426C0B2E9
:10D5D00006FB0040D0F8F83198453CD094F89612FC
:10D5E000384609F06FFFB0B32946384609F048FFC6
:10D5F000C0B206FB00402946D0F8F831C4F86835BF
:10D60000384609F03DFFC0B206FB0040D0ED7B7A02
:10D61000D4F86835CDF80530FDEEE77A01AA17EEAB
:10D62000903AD0ED7C7AADF80930FDEEE77A41F61C
:10D63000047117EE903AD0ED7D7AADF80B30FDEE27
:10D64000E77A204617EE903AADF80D300B238DF8AF
:10D650000450FFF755FE04B0BDE8F08110B5D0F8D6
:10D66000883404464BB1FFF77DFE2046FFF76AFF82
:10D670002046BDE81040FFF79DBF10BD2DE9F047E3
:10D6800090F9D03692B00546002B73D016F094FA7C
:10D69000B5F91210002908DDD5F82C27821A4FF4AD
:10D6A0007A73B3FBF1F39A4264D305F5D668C5F8F3
:10D6B0002C0740460EF002F936A7D7E900674FF075
:10D6C000000995F9D036002B4ED0002140460EF0CF
:10D6D0003BF90446002843D00EF024FE0128824680
:10D6E0003EDD6368D5F830271B699A4238D0C5F80B
:10D6F0003037202200210AA823F038FC95F8DC36C8
:10D700008DF83030BAF1030F05D0BAF1040F34D0E0
:10D71000BAF1020F01D18DF83DA020460EF0F8FDC0
:10D7200001282ED003282CD070BB02238DF83C306A
:10D73000636806AC1B681093012221460AA800F01A
:10D74000D5FD40F21A4380B21822CDE90032CDE96E
:10D750000240CDF8109032463B462846FEF7E2FBE9
:10D76000002301E0002BACD095F8FC260133DBB29E
:10D770009A42F7D212B0BDE8F08701238DF83D3010
:10D78000CBE78DF83C00D3E78DF83C90D0E700BFA5
:10D79000AFF30080521977FC70FEFF6810B50446A5
:10D7A00000F030F804F1080000F02CF804F110004B
:10D7B00000F028F82046024904F038FE204610BD4B
:10D7C000005603080E4B2DE9F0411F680646002461
:10D7D00000F1040804F1100357F823505DB12B68E1
:10D7E00036F834105B6B284698472B6818F83410CD
:10D7F000DB6B284698470134032CEBD1BDE8F08160
:10D80000D810002010B50349044604F00FFE20464E
:10D8100010BD00BF38560308034690F91900411C9B
:10D8200005D193F91000421C08BF93F91800704706
:10D83000F0B5A5B004460E46104603A9154601F002
:10D84000C7F9002840F0918030469DF80D701DF01A
:10D85000A5FE874240F08980D4F86837002B76D047
:10D860009DF90E00431C02D12046FFF7D5FF00288A
:10D870007BDB434B0928196877DC00F1100351F872
:10D880002360002E71D094F9743783420BD0D4F802
:10D89000702742B1DBB2092B4FF000026DD8103374
:10D8A00051F823301A61D4F8703784F87407B34202
:10D8B00008D0D4F8680701F0E1FD0023C4F87067D0
:10D8C000C4F87837D4F8700700284ED09DF80F20A0
:10D8D00094F87C6702F0010284F87C2702B1294A9F
:10D8E000114601F029FCEB7E84F875379DF80C3069
:10D8F000049984F87637D4F87837994200D17EB904
:10D9000094F87C374BB141B11E4B00934FF4006348
:10D91000D4F870071A4601F01FFC049BC4F878374E
:10D92000D4F87037D4F868271A6116F045F99DF8D5
:10D930001420C4F86C07C2B194F87C37D4F870078F
:10D94000ABB1104B0DF1150101F014FC0DE01420EA
:10D9500001F0A8F9064618B14FF4806101F03EFDD0
:10D96000C4F86867002E7FF47BAF25B0F0BD036874
:10D970000DF11501DB689847F7E71261FFDE00BF84
:10D98000D8100020E460E4F22DE9F043D0F87037BD
:10D99000C9B00446D3B190F87537BBB1D0F8683739
:10D9A000A3B1D0F86C5716F007F940F6B733401B17
:10D9B000984294F87C370CD92BB10022D4F8700728
:10D9C000114601F0B9FB0023C4F8703749B0BDE837
:10D9D000F08373B1344E0825D4F8700733467822AB
:10D9E00027A901F0D7FB002803DD013D15F0FF0555
:10D9F000F2D12BA7D7E900674FF00908D4F86807E0
:10DA000001F04EFD0028E1D008F1FF3818F0FF08C2
:10DA1000DCD0D4F8680706A901F0F2FD069D814626
:10DA2000002DD3D08422002127A823F09FFA94F858
:10DA300075378DF89D3094F876378DF89C30782DB9
:10DA4000D4F8783728932A4694F874378DF89E30A6
:10DA500028BF7822494607AD0DF1A50006928DF842
:10DA6000A42023F039FA0122294627A801F064F8FE
:10DA7000002380B21022049340F6B933CDE900327E
:10DA8000CDE9025032463B462046FEF74BFA0028CD
:10DA90009CD00699D4F8680701F036FDAEE700BFC8
:10DAA000E9A2A272EAE738B1E460E4F2F7B50C4605
:10DAB00005462F220021204623F058FA2B46382213
:10DAC000002120461DF094FF05F108032022382193
:10DAD00020461DF08DFF05F10C0310225821204631
:10DAE0001DF086FF05F110032022682120461DF05D
:10DAF0007FFF05F114032022882120461DF078FFC6
:10DB000005F118032022A82120461DF071FF95ED94
:10DB1000070A1DF0BDFF0DF10603ADF80600102247
:10DB2000C82120461DF064FF05F12007D826B7EC78
:10DB3000010A1DF0ADFF3146ADF806000DF10603F8
:10DB40001022204610361DF053FFB6F5847FEED12B
:10DB5000314605F12C03102220461DF049FF05F146
:10DB60002E074FF48C763B46314608222046083675
:10DB70001DF03EFFB6F5B07F07F10107F3D105F1C7
:10DB800037033146204603221DF032FF05F13803EA
:10DB90002046052240F263111DF02AFF05F13903EA
:10DBA000204607224FF4B4711DF022FF05F13A031D
:10DBB0002046012240F26F111DF01AFF05F13B03D0
:10DBC000204601224FF4B8711DF012FF05F13C030D
:10DBD0002046012240F271111DF00AFF05F13D03BC
:10DBE000204601224FF4B9711DF002FF05F13E03FA
:10DBF0002046012240F273111DF0FAFE05F13F03A9
:10DC0000204601224FF4BA711DF0F2FE05F14003E7
:10DC10002046012240F275111DF0EAFE204605F172
:10DC2000410301224FF4BB711DF0E2FE2F2003B02F
:10DC3000F0BD000037B50C4600210546216021717A
:10DC40000346012220461DF0D3FE01226B1C114623
:10DC500020461DF0CDFE95ED010A1DF019FF0DF1D6
:10DC60000603ADF806001022022120461DF0C0FE7A
:10DC700095ED020A1DF00CFF0DF10603ADF806004C
:10DC80001022204612211DF0B3FE052003B030BD46
:10DC900013B504460846002101602346C0F803106E
:10DCA000202201901DF0A4FE0198231D01222021B5
:10DCB0001DF09EFE019804F10803172221211DF09A
:10DCC00097FE072002B010BD70B50C461926054618
:10DCD00032460021204623F049F92B4620460822EF
:10DCE00000211DF085FE2B1D2046202208211DF05D
:10DCF0007FFE05F108032046102228211DF078FE42
:10DD000005F10A032046102238211DF071FE05F1AD
:10DD10000C032046102248211DF06AFE05F10E0377
:10DD20002046102258211DF063FE05F11003204605
:10DD3000102268211DF05CFE05F11403204620220C
:10DD400078211DF055FE05F1180320461022982178
:10DD50001DF04EFE05F11A0320461022A8211DF0E9
:10DD600047FE204605F11C031022B8211DF040FE9D
:10DD7000304670BD70B50C461C2605463246002163
:10DD8000204623F0F3F82B462046202200211DF0E8
:10DD90002FFE2B1D2046102220211DF029FE05F10B
:10DDA00008032046202230211DF022FE05F10C033D
:10DDB0002046102250211DF01BFE05F10E032046C7
:10DDC000102260211DF014FE05F1100320461022E0
:10DDD00070211DF00DFE05F1120320461022802156
:10DDE0001DF006FE05F114032046102290211DF0BF
:10DDF000FFFD05F1160320461022A0211DF0F8FDBD
:10DE000005F1180320461022B0211DF0F1FD05F1A7
:10DE10001A0320461022C0211DF0EAFD2046AB194E
:10DE20001022D0211DF0E4FD304670BD2DE9F341F4
:10DE30000E460446174600211922304623F096F874
:10DE4000A0460025B8EC010A1DF022FE2946ADF8D7
:10DE500006000DF106031022304610351DF0C8FDF6
:10DE6000302DEFD1237B092B28BF09238DF80530F6
:10DE70003FB929460DF10503042230461DF0B8FDD7
:10DE8000342510344FF000089DF80530984505EB17
:10DE9000081704D3F81DC00802B0BDE8F081B4EC47
:10DEA000010A1DF0F5FD0DF10603ADF80600102284
:10DEB000394630461DF09CFD08F10108E4E70000FA
:10DEC00037B50C4600212160A1800346054620227B
:10DED00020461DF08DFD95ED010A1DF0D9FD0DF1D7
:10DEE0000603ADF806001022204620211DF080FD1B
:10DEF000062003B030BD000073B500260E6090ED23
:10DF0000000A0C4605461DF0C3FD0DF1060331461F
:10DF1000ADF80600102220461DF06AFD95ED010ABD
:10DF20001DF0B6FD1022ADF806000DF106032046E7
:10DF300011461DF05DFD042002B070BD73B50C46A6
:10DF40001026054632460021204623F00FF895EDB5
:10DF5000000A1DF09DFD0DF106033246ADF80600E6
:10DF6000002120461DF044FD95ED010A1DF090FDB5
:10DF70000DF1060332463146ADF8060020461DF08D
:10DF800037FD95ED020A1DF083FD0DF106033246C3
:10DF9000ADF80600202120461DF02AFD95ED030A6C
:10DFA0001DF076FD0DF106033246ADF80600302176
:10DFB00020461DF01DFD95ED040A1DF069FD0DF1D3
:10DFC00006033246ADF80600402120461DF010FD44
:10DFD00095ED050A1DF05CFD0DF106033246ADF826
:10DFE0000600502120461DF003FD95ED060A1DF0A8
:10DFF0004FFD0DF10603ADF80600324620466021C4
:10E000001DF0F6FC05F11C032046072270211DF0CF
:10E01000EFFC204605F11D03062277211DF0E8FCE8
:10E02000304602B070BD00002DE9F3470D460446AE
:10E03000002190462846DE2222F098FF234638220F
:10E04000002128461DF0D4FC3822114604F10803B3
:10E0500028461DF0CDFC04F1100303227021284650
:10E060001DF0C6FC04F111030822802128461DF092
:10E07000BFFC04F118032522882128461DF0B8FCB6
:10E0800004F120032522AD2128461DF0B1FC04F146
:10E0900028031B22D22128461DF0AAFC04F12C03E0
:10E0A0001B22ED2128461DF0A3FC04F130032022A1
:10E0B0004FF4847128461DF09BFC04F134032022A8
:10E0C0004FF4947128461DF093FC04F1380320228C
:10E0D0004FF4A47128461DF08BFC04F13C0306228A
:10E0E0004FF4B47128461DF083FC04F13D03022275
:10E0F0004FF4B77128461DF07BFC04F13E03042267
:10E100004FF4B87128461DF073FC04F13F0306225A
:10E110004FF4BA7128461DF06BFC94F84030242B64
:10E1200028BF24238DF8033006220DF103034FF49A
:10E13000BD7128461DF05CFC04F1440A4FF4C07721
:10E140004FF000099DF80330994507F110062BD3D5
:10E1500094ED350A1DF09CFC0DF10603ADF80600A8
:10E160001022394628461DF043FC94F8D830012B84
:10E1700028BF01238DF80430B8F1000F07D13146D4
:10E1800001AB012228461DF033FC07F1110604F50E
:10E1900086744FF000099DF80430994515D3F01DA1
:10E1A000C00802B0BDE8F087BAEC010A1DF070FCAF
:10E1B0003946ADF806000DF10603102228461DF081
:10E1C00017FC09F101093746BCE7A4F12C0A06F156
:10E1D0006007B046534641462022284608F12008F1
:10E1E0001DF006FC47450AF1040AF3D1A4F11C080E
:10E1F00006F1CC0A434639462422284624371DF02E
:10E20000F7FBBA4508F10808F4D114F8043C242BB4
:10E2100028BF24238DF8053006F1D2010DF1050346
:10E22000062228461DF0E4FBD836A04600279DF8BC
:10E2300005309F4203D309F10109C034ABE7B8ECC4
:10E24000010A1DF025FC3146ADF806000DF106036C
:10E25000102228461DF0CCFB10360137E7E70000FE
:10E26000F7B5047F05460E462CB1838A822B02D96E
:10E27000012003B0F0BD002300960822194628466D
:10E280001DF078FADCB9731C08220093114623466E
:10E2900028461DF06FFA10247378802BE8D80123EC
:10E2A00072785F1C013B934210D32B7FA88A0734FE
:10E2B000E408B3B9844294BF00200120D9E7AB8AB7
:10E2C000DB00083BDB0873700824E5E7F3190093D3
:10E2D00021460023082228461DF04CFA08343B460C
:10E2E000DEE7201A18BF0120C3E70000F7B50C468F
:10E2F00005460F220021204622F038FE2B46382208
:10E30000002120461DF074FB05F108030822382186
:10E3100020461DF06DFB05F1090740263B463146BE
:10E320000522204605361DF063FB4F2E07F101073D
:10E33000F4D105F10C033146012220461DF058FBB3
:10E3400095ED040A1DF0A4FB0DF10603ADF80600DF
:10E350001022204650211DF04BFB05F114032046EE
:10E36000052260211DF044FB05F115030322652100
:10E3700020461DF03DFB95ED060A1DF089FB0DF1D1
:10E380000603ADF806001022204668211DF030FB80
:10E390000F2003B0F0BD000013B50446007F10B19C
:10E3A000A38A012B0CD8002300910822194620468D
:10E3B0001DF0E0F9237FA08A23B9B0FA80F040096C
:10E3C00002B010BD013818BF0120F9E72DE9F3476D
:10E3D0000D46044600219046284640F2791222F06C
:10E3E000C5FD23462022002128461DF001FB231DE8
:10E3F0000222202128461DF0FBFA631D0322222160
:10E4000028461DF0F5FAA31D0322252128461DF0FC
:10E41000EFFA04F108031022282128461DF0E8FA3B
:10E4200004F110030822382128461DF0E1FA04F116
:10E4300011030822402128461DF0DAFA04F11203E4
:10E440000822482128461DF0D3FA04F114032022A3
:10E45000502128461DF0CCFA04F118034022702107
:10E4600028461DF0C5FA04F120030822B0212846F1
:10E470001DF0BEFA04F121030822B82128461DF040
:10E48000B7FA04F12207C0263B4631460822284647
:10E4900008361DF0ADFAB6F5A07F07F10107F3D1FC
:10E4A00094F832308DF8073031460DF10703082219
:10E4B00028461DF09DFA002604F1330A9DF8073026
:10E4C0004FEAC6099E4209F5A47720D394F8323169
:10E4D000502B28BF50238DF80730B8F1000F08D11A
:10E4E00039460DF10703072228461DF081FA09F28B
:10E4F0004F17002604F233149DF807309E4207EBB5
:10E50000C6010DD30731C80802B0BDE8F0870AEB99
:10E5100006030822394628461DF06AFA0136CDE77F
:10E52000A319082228461DF063FA0136E4E700002B
:10E5300013B504460846002101602346C0F80310C5
:10E54000202201901DF054FA0198231D022220215F
:10E550001DF04EFA0198631D032222211DF048FA96
:10E560000198A31D032225211DF042FA019804F110
:10E570000803102228211DF03BFA072002B010BD2D
:10E5800008B5034608460021017001221DF030FA4B
:10E59000012008BD2DE9F3410D4604460021164631
:10E5A00028467B2222F0E2FC234603220021284653
:10E5B0001DF01EFA63781F2B28BF1F238DF806302D
:10E5C00005220DF10603032128461DF011FA01234F
:10E5D0009DF80620DF0003F10108013B9A421CD898
:10E5E00094F821305A2B28BF5A238DF807303EB9B2
:10E5F00039460DF10703072228461DF0F9F90737C0
:10E60000002622349DF807309E4207EBC6010DD349
:10E610000731C80802B0BDE8F08104EB0803082206
:10E62000394628461DF0E4F94346D1E7A3190822EC
:10E6300028461DF0DDF90136E4E70000F7B5047F58
:10E6400005460E462CB1838A122B02D9012003B055
:10E65000F0BD002319460722009628461DF08AF8CF
:10E66000731C009301220023072128461DF082F825
:10E67000D4B9B31C009305222346082128461DF077
:10E6800079F80D24B378102BE0D83746B278BB1B4D
:10E69000934210D32B7FA88A0734E408B3B984428D
:10E6A00094BF00200120D2E7AB8ADB00083BDB08E7
:10E6B000B3700824E6E7FB1C0093214600230822E0
:10E6C00028461DF057F808340137DFE7201A18BF35
:10E6D0000120BCE7F7B5047F05460E462CB1838ABE
:10E6E000CA2B02D9012003B0F0BD002319460096C1
:10E6F000082228461DF03EF8731CD4B90822009366
:10E700001146234628461DF035F810247378C82B8F
:10E71000E8D8012372785F1C013B934210D32B7F12
:10E72000A88A0734E408B3B9844294BF00200120CA
:10E73000D9E7AB8ADB00083BDB0873700824E5E708
:10E74000F319009321460023082228461DF012F8F1
:10E7500008343B46DEE7201A18BF0120C3E700005B
:10E76000F7B50D460446002116462846812222F0C0
:10E77000FDFB23460822002128461DF039F994F9B3
:10E7800001206378002AB8BF7F238DF807309EB937
:10E790000DF107030722082128461DF029F90F274C
:10E7A000002602349DF807309E4207EBC60105D3D0
:10E7B0000731C80803B0F0BD0827F1E7A319082204
:10E7C00028461DF015F90136ECE7000037B5044680
:10E7D000007F0D4610B1A38A072B15D800231946D8
:10E7E00000950822204608351CF0C4FF012300953F
:10E7F0003022082120461CF0BDFF237FA08A2BB9C0
:10E8000006288CBF0020012003B030BD073818BF98
:10E810000120F9E738B50C46002121600546C4F80F
:10E8200003100346302220461DF0E2F8204605F191
:10E830000803012230211DF0DBF8072038BD00005D
:10E840002DE9F04390F81C8085B006460D46B8F1DE
:10E85000000F06D0838AE02B03D9012005B0BDE864
:10E86000F083002319460D22009530461CF082FFEC
:10E870000DF10F030093032200230D2130461CF0FD
:10E8800079FF9DF80F30042BE7D82B72013B032B47
:10E8900003D8DFE803F025303B461024B8F1000F21
:10E8A0005FD105F198030093214643460722304685
:10E8B0001CF060FF073495F898305C2BCDD82F46BC
:10E8C00095F898207B1B934252D3337FB08A07344C
:10E8D000E408002B58D1844294BF00200120BDE7FA
:10E8E00005F11003009340220123102130461CF053
:10E8F00041FF5024D2E705F11003009320220123A9
:10E90000102130461CF036FF3024C7E705F1100314
:10E91000009308220023102130461CF02BFF1824FE
:10E92000BCE705F1100300930822002310213046B4
:10E930001CF020FF2B7C802B8FD8002705F11109BC
:10E940002B7CFC009F4204F11804A7D209EB0703BB
:10E95000009308220023214630461CF00BFF0137AC
:10E96000EEE7B38AC4EBC303DB0885F89830A2E76F
:10E9700007F19903009321460023082230461CF03A
:10E98000F9FE083401379BE7201A18BF012065E71C
:10E99000F7B50C46137809688DF8063015460DF169
:10E9A0000603032206461DF023F821680331216087
:10E9B0002B78013B032B0CD8DFE803F0020D161F68
:10E9C00005F10803402230461DF012F82368403359
:10E9D000236003B0F0BD05F10803202230461DF08E
:10E9E00007F823682033F3E705F1080308223046CF
:10E9F0001CF0FEFF23680833EAE72B7A802B28BF40
:10EA000080238DF8073008220DF1070330461CF0F3
:10EA1000EFFF236808332360002709359DF807308E
:10EA20009F42D6D2EB192168082230461CF0E0FF45
:10EA30002368083323600137F0E7000073B50C4604
:10EA4000137809688DF8073015460DF10703022287
:10EA500006461CF0CDFF2168023121602B78012B86
:10EA600003D0022B0BD002B070BD05F10803402289
:10EA700030461CF0BDFF236840332360F3E705F107
:10EA80000803202230461CF0B3FF23682033F4E74C
:10EA900073B50D46044600211646284640F273120F
:10EAA00022F064FA0523224601A928460193FFF7C4
:10EAB0006FFF019B04F19002053301A928460193E1
:10EAC000FFF766FF019B04F59072063301A9284603
:10EAD0000193FFF7B3FF019B04F59872063301A978
:10EAE00028460193FFF7AAFF94F840315C2B28BF1A
:10EAF0005C238DF803304EB90DF103030199072211
:10EB000028461CF075FF019B07330193002604F291
:10EB100041149DF8033001999E4203D30731C80880
:10EB200002B070BDA319082228461CF061FF019BAA
:10EB3000083301930136ECE7F7B50D460446002192
:10EB4000164628467F2222F011FA23460822002189
:10EB500028461CF04DFF631C0722082128461CF0A4
:10EB600047FFA31C05220F2128461CF041FFE31C90
:10EB70000422142128461CF03BFF1822231D1146B5
:10EB800028461CF035FF237A782B28BF78238DF890
:10EB900007309EB90DF107030722302128461CF0EB
:10EBA00027FF3727002609349DF807309E4207EBE0
:10EBB000C60105D30731C80803B0F0BD3027F1E71F
:10EBC000A319082228461CF013FF0136ECE70000C9
:10EBD000F7B5047F05460E462CB1838A7F2B02D9F8
:10EBE000012003B0F0BD00231946082200962846F4
:10EBF0001CF0C0FD731C0093072200230821284647
:10EC00001CF0B8FDB31C0093052201230F212846F8
:10EC10001CF0B0FDF31C00930422002314212846AD
:10EC20001CF0A8FD331D182200931146002328462E
:10EC30001CF0A0FDDCB906F108030093072223466F
:10EC4000302128461CF096FD3724337A782BC7D81C
:10EC50003746327ABB1B934210D32B7FA88A0734E6
:10EC6000E408BBB9844294BF00200120B9E7AB8A15
:10EC7000DB00303BDB0833723024E6E707F10903A1
:10EC8000009321460023082228461CF073FD083417
:10EC90000137DEE7201A18BF0120A2E700487047BD
:10ECA000B05603080121884238BF08461FF028BB30
:10ECB000FFF7F8BF08B11FF027BB7047FFF7FABF97
:10ECC00010B4026854681A4623465DF8044B18478E
:10ECD00000207047012070470020704700207047D7
:10ECE00000207047704700000020704700207047E8
:10ECF000704700007047000037B505460C46832278
:10ED0000011D01A800F062F9611EC9B202299EBF6F
:10ED100005EBC1010023C1E9073301A800F078F930
:10ED200003B030BD2DE9F7431E461B885B0705463F
:10ED3000884620D4011D422201A800F047F92C4644
:10ED400005F118094C4513D0E3696BB12B682846CF
:10ED50005B6C98473388276AC1B243F00403E069CB
:10ED60004246B8470834EDE7236A002BEED1F9E7B5
:10ED700001A800F04DF9012003B0BDE8F0830000C8
:10ED80007FB56D4685E806000446011D712203A883
:10ED90001E4600F01BF921460022C869D3B288B98B
:10EDA000086A78B995E8030004EBC2021C3201330B
:10EDB00082E803000124337003A800F029F92046FB
:10EDC00004B070BD0132032A01F10801E5D100242D
:10EDD000F2E700002DE9F04F2DED028B8BB00446D9
:10EDE0008B465322011D01A8BDF858809FED258B4D
:10EDF00000F0ECF8254604F11809002708F0040A91
:10EE0000A94536D0EB690BB92B6A63B1BAF1000F93
:10EE10000BD1236820465B6C98474346C1B25A46E3
:10EE2000D5E90706B0470835EAE7002FFBD18DED9D
:10EE3000028BADF810705B4605AA0BF1080C186840
:10EE40005968174603C7083363453A46F7D118682F
:10EE500038609B88BB8014F0B1FE0423ADF81030FD
:10EE60002368CDE902019B6C02A92046984701273F
:10EE7000D9E701A800F0CCF801200BB0BDEC028B63
:10EE8000BDE8F08F000000000000000030B503680E
:10EE90000968DD0FB5EBD17F23F0604421F06042BB
:10EEA0004FEAD1700BD0002BB8BFA40C0029B8BF1B
:10EEB000920C944202D034BF0120002030BD944215
:10EEC00005D1C1F38070C3F380738342F6D19442BD
:10EED0002CBF00200120F1E7082817D90C280CD9F5
:10EEE00010280CD914280CD918280CD920280CD992
:10EEF00030288CBF0F200E207047092070470A2051
:10EF000070470B2070470C2070470D2070470000A1
:10EF1000082817D909280CD00A280CD00B280CD0A7
:10EF20000C280CD00D280CD00E2814BF4020302007
:10EF300070470C207047102070471420704718202D
:10EF400070472020704700004368184783681847BF
:10EF500010B5024C8260C0E9004110BD485703085B
:10EF6000007B00F0010070477047000081608280E4
:10EF700070470000826838B504465AB1037B13F02D
:10EF8000010507D143F0010303739047237B65F329
:10EF90000003237338BD000010B5044B1B68044602
:10EFA000986A03681B699847204610BDD810002056
:10EFB00010B5054B1B680446986A036800211B695D
:10EFC0009847204610BD00BFD8100020F8B50C4B64
:10EFD00001601E680446B06A03681B6C17469847B8
:10EFE000054610B1F36AA3F84270206803689B6875
:10EFF00098471DB1F36A0022A3F842202046F8BDCD
:10F00000D810002010B50446FFF7E0FF204610BDE1
:10F0100010B5044600680368DB689847204610BDB9
:10F02000C181B1FA81F0400970470000C089704782
:10F0300070470000002070477047000070470000D4
:10F040000020704700207047704700004FF4B45014
:10F050007047000000207047002070470020704774
:10F060000020704700207047007B70477047000009
:10F0700007B503688DF80710DB6801220DF1070161
:10F08000984703B05DF804FB08B5036801225B6A8A
:10F0900098470028D4BF0020012008BD07B50368A9
:10F0A0000DF10701DB69984720B19DF8070003B017
:10F0B0005DF804FB4FF0FF30F9E7000013B504469C
:10F0C00008460191FCF770F923680199DB68024654
:10F0D000204602B0BDE810401847000014F06EBD95
:10F0E00010B444682CB903685DF8044BD3F8803041
:10F0F000184700205DF8044B7047000082681AB979
:10F100000368D3F8903018470020704782681AB916
:10F110000368D3F8943018470020704730B445682E
:10F1200025B90468E46FA44630BC604730BC704722
:10F1300000231A46FFF7F2BF436813B18B4200D099
:10F1400041B9836813B1934200D01AB9C0E90112E2
:10F15000012070470020704730B44468029D0CB114
:10F16000AC4204D10468E46FA44630BC604730BCB4
:10F170007047000010B444680CB19C4205D103688C
:10F180005DF8044BD3F88030184700205DF8044B3D
:10F190007047000037B50546806808B1984212D123
:10F1A0002B680191D3F8843092B2284698470446E0
:10F1B000286928B1002C03DD0199224600F000FAED
:10F1C000204603B030BD0024FAE700000023FFF71B
:10F1D000E1BF000082682AB942681AB90368D3F80F
:10F1E0008830184770470000013901298CBF002082
:10F1F00001207047002070470020704700207047B2
:10F20000704700000320704700230B707047000018
:10F2100070470000704700000020704700207047D2
:10F2200000207047704700004368C26893423CBFAB
:10F230008268D15443680133436001207047000065
:10F24000F8B505460C468F180026BC4207D02B683F
:10F2500014F8011B9B68284698470644F5E730469A
:10F26000F8BD000000207047002070470020704764
:10F270000020704738B590F89C308B4204460D460C
:10F280000CD080F89C1014F097FC2368C4F8A00000
:10F290005B682046984708B984F84D5038BD000097
:10F2A0007FB50D461446194600267AB1531E0B4A07
:10F2B0006846CDE90026089ACDE9025300F00EFA1F
:10F2C0000198844204D92E5404B070BD1346EEE771
:10F2D000002CF9D02C4404F8016CF5E76C570308B6
:10F2E00008B410B585B007AC54F8043B00940394FF
:10F2F000FFF7D6FF05B0BDE8104001B07047000031
:10F3000070B504460CF04EF95E224FF400010CF08B
:10F3100035F90D4E0D4B1D6833783BB9E86A042270
:10F320002146483014F062FC01233370EB6A2A2234
:10F3300083F84620EB6A93F89C301BB904482146B9
:10F3400014F012FC70BD00BF92300020D8100020D5
:10F350005057030807B503680DF10701DB699847AB
:10F3600020B19DF8070003B05DF804FB4FF0FF30BB
:10F37000F9E70000F8B506460F4614460025AC42F2
:10F380000AD0336830469B699847431C01D1284610
:10F39000F8BD78550135F2E72046F9E70EB403B51C
:10F3A00003AA036852F8041B5B680192984702B0F5
:10F3B0005DF804EB03B0704700F090B913B5044654
:10F3C00008460191FBF7F0FF23680199DB680246CC
:10F3D000204602B0BDE810401847000070B5002676
:10F3E0000446C0E9026601200D461EF089FFB042C6
:10F3F00008BF3546206065602674204670BD000059
:10F4000010B5037C044613B900681EF07DFF20464A
:10F4100010BD000070B5057C04460E46DDB9BFF393
:10F420005B8FC560BFF35B8FBFF35B8F8560BFF3FE
:10F430005B8F43688B420CD000681EF065FF31463D
:10F4400001201EF05DFF206010B96560284670BD88
:10F4500066600125FAE70025F8E7000038B50546A3
:10F460000C4644B121462846FFF7D4FF20B904EBEF
:10F470004404A408F5E7204638BD00000023BFF38C
:10F480005B8FC360BFF35B8FBFF35B8F8360BFF3A2
:10F490005B8F7047BFF35B8F0068BFF35B8F704774
:10F4A00070B505460C30FFF7F5FF05F10806044678
:10F4B0003046FFF7EFFFA04206D930466D68FFF7F0
:10F4C000E9FF2544281A70BD3046FFF7E3FF201AF4
:10F4D000F9E7000070B50546406898B105F10800ED
:10F4E000FFF7D8FF05F10C0604463046FFF7D2FFC0
:10F4F0008442304694BF6D680025FFF7CBFF013C86
:10F500002C44201A70BD000038B50C460546FFF7A4
:10F51000C7FFA04210D305F10800FFF7BBFF04446A
:10F520006868B4FBF0F100FB1144BFF35B8F01206E
:10F53000AC60BFF35B8F38BD0020FCE72DE9F041E4
:10F54000144607460D46FFF7C5FF844228BF044610
:10F55000D4B1B84658F80C6B4046FFF79BFF3044D7
:10F56000286040467E68FFF795FF331A9C4203D817
:10F570006C600120BDE8F0816B60A41B3B68AB6050
:10F580002044E8600220F5E72046F3E738B50C4652
:10F590000546FFF79FFFA04210D305F10C00FFF7CF
:10F5A00079FF04446868B4FBF0F100FB1144BFF339
:10F5B0005B8F0120EC60BFF35B8F38BD0020FCE760
:10F5C0002DE9FF41884669460746FFF7B7FF6C46BD
:10F5D00006B204EBC6060025B44209D06268206872
:10F5E00008EB050121F078FC636808341D44F3E75B
:10F5F00029463846FFF7CAFF284604B0BDE8F08127
:10F60000F8B505460C300F46FFF744FF05F1080634
:10F6100004463046FFF73EFFA042304688BF6C6884
:10F62000FFF738FF201A386020B130462C68FFF70A
:10F6300031FF2044F8BD000073B5144606460D4660
:10F64000FFF72EFF844228BF04460190DCB101A9D8
:10F650003046FFF7D5FF019B33B93268C5E9023365
:10F66000C5E9002401200CE09C4238BF01942860C9
:10F67000019868608442F5D93368AB60241AEC6065
:10F68000022002B070BD2046FBE700002DE9FF41DB
:10F690000F466946FFF7D0FF6C4600B204EBC00589
:10F6A0000026AC4209D0D4F8048054F8081BB819DD
:10F6B000424621F011FC4644F3E7304604B0BDE871
:10F6C000F081000038B50546FFF7E0FF044601462B
:10F6D0002846FFF719FF204638BD00002DE9F04FFE
:10F6E0002DED028B06468DB0904691F80090B9F151
:10F6F000000F00F0DE82B9F1250F08D04B1C0393F8
:10F70000336849469B68304698470399EDE791F87E
:10F7100001908B1CB9F1250F0393F1D00025AA4667
:10F720002C461F2C3BD8B9F12B0F2DD01CD8B9F18A
:10F73000200F2BD0B9F1230F2ED0A9F13003DBB26B
:10F74000092B36D860064BBF05EB85050AEB8A0A04
:10F7500003EB450503EB4A0A4EBF05F0FF050AF02F
:10F76000FF0A44F0200407E0B9F12D0F11D0B9F1E0
:10F77000300FE2D144F00104039B13F8019B039383
:10F78000B9F1000FCDD126E044F0020444F00404A6
:10F79000F2E744F00804EFE744F01004ECE77F2CB4
:10F7A000CBD9230617D5B9F16C0F14D144F480746A
:10F7B000E2E7B9F12E0F05D1620600F17A8244F03A
:10F7C0004004D9E7B9F16C0F02D144F08004D3E7CB
:10F7D000B9F1680FD0D0A9F14503022B61D809F126
:10F7E000200944F010045FFA89F908F1070828F0AD
:10F7F0000708F8E80201FBF7A9F914F0400F08BF69
:10F80000062524F0C004B9F1650F08EE100AA4B271
:10F8100050D144F0400427060DD59FED977AF0EEC5
:10F82000C87AF4EEC77AF1EE10FAC2BF4FF63F7312
:10F83000234043F0400414F0800346D03B2DA946FA
:10F8400028BF4FF03B0909F101095FFA89F9072741
:10F850001722002106A8029321F088FB4A46394668
:10F8600006A8B0EE480A14F0B1FB9DF818300193D9
:10F8700003F00902012A029B83462FD0A0072FD450
:10F8800014F0040F0CBF00222022019911F00C0784
:10F8900058D0002A40F0AB82BAF1030F50D8174677
:10F8A00037E0A9F16503022B00F25B8124F010041C
:10F8B000A4B29AE7B9F1660F02D144F08004AAE736
:10F8C000002DA8D0013DEDB2A5E70A2D83BF0A2582
:10F8D00099462F462F4698BF9946B9E72D22D4E77F
:10F8E0002B22D2E70427AAEB07072107FFB20AD48D
:10F8F000336802929B6820213046013F984717F0F9
:10F90000FF07029AF4D122B1336811469B68304652
:10F910009847019B594D13F0080F594B08BF1D46DE
:10F92000013D04F0100415F8011F002900F0B58016
:10F930000CB12039C9B2336830469B689847F2E76A
:10F940000327D0E7CDF808B0002B36D0019BD9446F
:10F95000DB065FFA89F907D59DF81930312B04BF12
:10F9600009F1FF395FFA89F94FFA89F3002B44DD79
:10F97000B9F1080F28BF4FF0080914F08003049371
:10F980001ABF2BEAEB730133052302B101330DB12A
:10F99000691C0B449A45C4BFAAEB0303DFB214F001
:10F9A000090F2FD177B3336805929B682021304629
:10F9B000013F9847FFB2059AF4E76006DDD45D4544
:10F9C00004DB1BF1040FA8BF44F080046B1C06A9E4
:10F9D0000B4435B113F80119302902D1013DEDB2C4
:10F9E000F7E72106C9D505F101095D455FFA89F9F7
:10F9F00006DDA5EB0B05EDB2BFE74FF00109BCE753
:10FA00000025BAE722B1336811469B683046984713
:10FA1000220708D43FB1336830219B683046013F4C
:10FA20009847FFB2F6E7049B002B47D02BEAEB7414
:10FA3000ABEB040A06AB9A44ABEB09096D42A34554
:10FA400017DBA14515DA9AF80110013CA54219DC33
:10FA5000002900F0D281336830469B689847631CC8
:10FA600004D133682E219B68304698470AF1010A79
:10FA7000E5E73021E9E700BF7F96184B9C57030864
:10FA800098570308A34507D19DF81930352B0FD897
:10FA900002D1019BDD060BD559B9002F3FF435AEDD
:10FAA000336820219B683046013F9847FFB2F4E756
:10FAB000312133689B6830469847EEE79DF819106E
:10FAC00031291EBF019B03F0EF03019333683046D9
:10FAD0009B689847E5B9336814F0100F14BF4521AF
:10FAE00065219B6830469847BBF1000F29DACBF1BE
:10FAF000000302932D21336830469B6898473021DC
:10FB0000029B092B23DD01310A3BC9B20293F7E7BF
:10FB100033682E219B68304698470235EDB24FF08E
:10FB200002094B460CAA1A44336812F8181C9B6849
:10FB300009F101095FFA89F930469847A945F0D1E2
:10FB4000C9E702D1019BDC06D1D42B21D3E733686E
:10FB500030469B6898470299336830319B68C9B238
:10FB6000A9E7B9F1630F37D0B9F1730F4FD0B9F1ED
:10FB7000640F63D124F0900714F4807FBFB20DF1BD
:10FB800018097BD008F1070222F00702904651685D
:10FB900058F8080B002904DA404261EB410147F0B4
:10FBA00080070A234A4600F07BF9A0EB0900C4B2A3
:10FBB0007B0640F19F8027F00109AC421FFA89F9CA
:10FBC00080F0D28007F01403102B03D127F0110727
:10FBD0001FFA87F9AB468FE058F8043B8DF81830D0
:10FBE00001250DF11809200701D4AA451CD84D4460
:10FBF0005746A9453FF451AF336819F8011B9B687C
:10FC000030469847002FF4D0013FFFB2F1E758F893
:10FC1000049B14F0400F14BF29464FF0FF314846B3
:10FC200021F090FE0546DEE7336820219B683046D0
:10FC30000AF1FF3A98475FFA8AFAD6E7B9F1690FF5
:10FC400098D0B9F1750F27D124F01004A7B20A2378
:10FC500017F4807FDBB20DF1180944D008F10708D2
:10FC600028F00708F8E802014A4600F019F9A0EB6D
:10FC7000090027F08007C4B2BFB299E758F8040B17
:10FC80000028B8BF40424FF00A024946B8BF47F0CB
:10FC9000800700F0B7F888E724F00607B9F1700F85
:10FCA000BFB214D00AD8B9F1580F13D0B9F16F0F01
:10FCB00017D00DB0BDEC028BBDE8F08FB9F1780F15
:10FCC000F7D1F90601D547F004071023C0E747F044
:10FCD0001007F6E7E20601D547F006074FF4047374
:10FCE000B6E70823B4E758F8040B1A46494600F073
:10FCF00089F8BCE7A346B94619F0100F41D00CAB08
:10FD0000234413F8193C302B30D129F016091FFA7F
:10FD100089F919F0080744D119F0010F35D0DA45F7
:10FD200045D904EB0A05A5EB0B05EDB2336819F0D4
:10FD3000100F9B683FD030213046984719F0040FD0
:10FD400008D0336819F0020F9B6814BF582178213E
:10FD5000304698473368AC429B6839D230213046F0
:10FD6000013D9847EDB2F5E7A346C5E719F0040F4A
:10FD700002D10BF1010B01E00BF1020B5FFA8BFBDF
:10FD8000C7E719F0860FC4D0F3E73368DA459B68FC
:10FD90000FD9202130460BF1010B98475FFA8BFBFE
:10FDA000F3E7DA4505D9AAEB0B07FFB2BEE7254614
:10FDB000BCE70027BAE719F0860FCBD019F0020F85
:10FDC00014BF2B21202119F0800F18BF2D21BFE770
:10FDD000651E06AB53FA85F5336815F801199B6863
:10FDE000013CE4B230469847002CF5D155E6BAF113
:10FDF000040F3FF677AD002786E5A3457FF44DAEAF
:10FE000042E600BF082A30B505D10346C008FCD140
:10FE100030330B700DE0102A0DD100F00F0202F10B
:10FE20003003392B88BF02F13703000901F8013B89
:10FE3000F3D1084630BD03460022DCB223F00103B3
:10FE4000023342F10002580840EAC270C31842EB84
:10FE50005202180940EA0270C01842EB1212030A5B
:10FE600043EA0263181842EB1222030C43EA0243EE
:10FE70001B1842EB1242D31842F100001B0943EA5F
:10FE80000073C3EB4315C3EB85053034020904EB63
:10FE9000450453EA101001F8014BCED1C9E7000028
:10FEA000082B30B50AD10346C00840EA4170C908A2
:10FEB00050EA0104F7D13033137013E0102B13D143
:10FEC00000F00F0404F13003392B4FEA101088BF03
:10FED00004F1370340EA0170090902F8013B50EAD6
:10FEE0000103EDD1104630BD20F00104023441F190
:10FEF0000003610841EAC3710C1943EB5303210964
:10FF000041EA03710C1943EB1313210A41EA03611F
:10FF10000C1943EB1323210C41EA0341091943EB6C
:10FF20001343591843F10003C5B2080940EA0370AE
:10FF3000C0EB4014C0EB84043035190905EB4405CF
:10FF400050EA131302F8015BCED1CBE770EE600AE2
:10FF5000DFED057AF0EEE00AF4EEE70AF1EE10FAD2
:10FF60004CBF0120002070470000003408B52DED83
:10FF7000028B9FED088AF0EE480A1FF05BF8B5EEA1
:10FF8000C00AF1EE10FA48BF30EE080ABDEC028B51
:10FF900008BD00BF0000B44308B52DED028B9FEDF6
:10FFA000088AF0EE480A1FF045F8B5EEC00AF1EEF7
:10FFB00010FA48BF30EE080ABDEC028B08BD00BF46
:10FFC00000A00C4710B5B4EE400AF1EE10FA2DED8A
:10FFD000028B0446B0EE608AF0EE418A0FD70BF038
:10FFE000E1FAA2B24FF480610BF0C8FA38EE288A29
:10FFF000B6EE000A28EE000ABDEC028B10BDB4EE8E
:020000040801F1
:10000000E00AF1EE10FA07D4B4EE410AF1EE10FA6C
:10001000C8BFB0EE410AEFE7B0EE600AECE70000BF
:10002000884203DB90420146A8BF1146084670474C
:10003000884203DB90420146A8BF1146084670473C
:10004000094A136849F2690099B21B0C00FB01339D
:100050001360064B186844F2506182B2000C01FB39
:100060000200186080B27047080E0020040E0020C5
:10007000036800EE103A7047024682B0006851688B
:100080006B4603C39DED000B02B0704701234A1E6F
:1000900003FA02F202421CBF8B40C01A70470000F4
:1000A000D0ED010AD1ED016A90ED021A91ED027ACC
:1000B00090ED000AD1ED007A70EEA60A31EE071A33
:1000C00030EE270A88B008B0704700BFD0ED010AB3
:1000D000D1ED016A90ED021A91ED027A90ED000ADD
:1000E000D1ED007A70EEE60A31EE471A30EE670A7B
:1000F00088B008B0704700BFD0ED010A90ED021A39
:10010000D0ED007A60EE200A20EE011A27EE800A78
:1001100088B008B0704700BF91ED005AD1ED015A88
:1001200091ED026AD0ED006A90ED017AD0ED027A8D
:1001300076EE856A37EE257A77EE867AC0ED006A2C
:1001400080ED017AC0ED027A704700BFD0ED006A01
:1001500090ED017AD0ED027A66EE806A27EE007AA1
:1001600027EE800AC0ED006A80ED017A80ED020A78
:10017000704700BF90ED007AD0ED017A90ED026AF1
:10018000C7EE006A87EE807AC6EE007AC0ED006A9C
:1001900080ED017AC0ED027A704700BFD0ED007AA1
:1001A000F4EE677AF1EE10FA10D6D0ED017AF4EEA3
:1001B000677AF1EE10FA09D6D0ED027AF4EE677A9A
:1001C000F1EE10FA6CBF012000207047012070474B
:1001D000D0ED007A9FED0F7AF0EEE77AF4EE477AF1
:1001E000F1EE10FA14DCD0ED017AF0EEE77AF4EEDD
:1001F000477AF1EE10FA0BDCD0ED027AF0EEE77AF6
:10020000F4EE477AF1EE10FACCBF012000207047DF
:1002100001207047FFFF7F7F08B52B2900F2828203
:10022000DFE811F044004602400233022A021B02BA
:10023000680157014E016E0158003F0179018401A8
:100240004500D4000401EF003901290120010B0110
:1002500091010A02E501DF0145005800D101C40106
:10026000B901AA019F01C700BE00B700AA009B0008
:10027000700061002C006D0262025102D0ED016A33
:10028000D0ED007A9FEDDD6A36EEA77A77EEE67A5A
:10029000D0ED026A27EE067A67EE867AF1EE666A9C
:1002A000C0ED016A80ED027AC0ED007A08BD90EDE4
:1002B000007AD0ED016AD0ED027AF1EE666AB1EE15
:1002C000477AF1EE677AC0ED006A80ED017AC0ED01
:1002D000027A08BDD0ED027A036842680260F1EE4E
:1002E000677A4360F3E7D0ED007A90ED026ADFEDC4
:1002F000C36A37EE867A77EEC67A27EE267A67EEFD
:10030000A67ACFE7D0ED017ADFEDBD5ADFEDBD6A09
:100310009FEDBD7A90ED006ADFEDBC4A9FEDBC5ABF
:1003200067EEA66A27EE877A67EEA57ADFEDB95AFF
:10033000E6EE246AA6EE057AE6EE257ADFEDB64A09
:1003400090ED026A9FEDB55ADFEDB55AE6EE246AEC
:10035000A6EE057AE6EE257AB5E790ED027AD0EDC5
:10036000007A43688360B1EE477AF1EE677A80EDF8
:10037000007AC0ED017A08BD90ED017AD0ED007AE7
:100380008368B1EE477AF1EE677A80ED027A036016
:10039000EFE781680268436841608260036008BDDE
:1003A000D0ED017A83680268F1EE677AC0ED017AD8
:1003B000F3E790ED027AD0ED017A0368B1EE477A67
:1003C000F1EE677A80ED017A83606DE7D0ED007A17
:1003D00090ED017ADFED935A9FED886A77EE876A98
:1003E00077EEC77A90ED027A66EEA56A67EE867AB6
:1003F000B1EE477AC0ED016AC0ED007A80ED027A75
:1004000008BD90ED026AD0ED007ADFED7C6A4368AA
:1004100037EE867A77EEC67A67EEA67A27EE267AE8
:100420008360C0ED017A80ED007A08BDD0ED027ADC
:1004300043688360F1EE677A9BE7D0ED026AD0ED06
:10044000007A9FED6E6A37EEE67A77EEA67AD0ED07
:10045000016A67EE867AF1EE666A27EE067AC0EDEB
:10046000026ADEE7D0ED017A8368F1EE677AC0EDCB
:10047000027A436008BDD0ED026AD0ED007A9FEDAC
:100480005F6A436837EEE67A77EEA67ADFED656A53
:1004900067EE867AC2E7826841680368816002601D
:1004A000E7E7D0ED017A90ED007A9FED546A77EEA0
:1004B000876A77EEC77A90ED027A66EE866A95E7EC
:1004C00090ED017AD0ED027AB1EE477AF1EE677ADB
:1004D000FBE6D0ED007A90ED016ADFED486A36EE7A
:1004E000677A77EE867A27EE267A67EEA67A80ED2F
:1004F000017AD9E6D0ED007A4368F1EE677A46E7F3
:10050000D0ED007A90ED017A9FED3C6A77EEC76AF4
:1005100077EE877ACFE790ED007AD0ED027AB1EEF0
:10052000477AF1EE677A80ED007AD0E6D0ED007A76
:1005300090ED017ADFED315A9FED3A6A77EE676A06
:1005400077EE877A4EE790ED017AD0ED027A036874
:10055000B1EE477AF1EE677A80ED027AC0ED007A6B
:1005600087E7D0ED007A436882684260F1EE677AEF
:10057000C0ED007A836008BDD0ED026AD0ED017A4B
:1005800090ED007AF1EE666AB1EE477AF1EE677AA5
:10059000C0ED016AC7E7D0ED017A90ED007A83687B
:1005A0004360F1EE677AB1EE477A7BE6D0ED016AFF
:1005B000D0ED027A90ED007AF1EE666AF1EE677A9C
:1005C000B1EE477A6CE690ED027AD0ED007A43689E
:1005D000B1EE477AF1EE677A80ED017AC0ED027AEA
:1005E000DCE6D0ED027A0368F1EE677AECE6D0ED56
:1005F000007A8368F1EE677AF0E700BFF304353FD5
:10060000DB26B93E46D0BC3EC9355BBFCF78123E33
:100610004F0DAABEC6AC6EBF4D1F6BBFF184CABEE4
:10062000F63BCC23F30435BFF304353F81177E3FFF
:10063000A296F93DA296F9BDD0ED026AD0ED007AFE
:100640005FED075A1FED096A37EEA67A77EEE67A74
:10065000D0ED016A67EEA57AFDE6D0ED006AD0ED37
:10066000017A1FED106A37EEA67A77EEE67A5FED33
:10067000126A27EE067A38E790ED007AD0ED017A1B
:10068000B1EE477AF1EE677A71E6D0ED016AD0ED0E
:10069000007A1FED1B6A37EEE67A77EEA67A5FEDF9
:1006A0001F6AE6E7D0ED017A0368F1EE677A55E755
:1006B000D0ED007A90ED016A5FED256A37EE867A1B
:1006C00077EEC67A0FE7D0ED017A90ED026A5FED22
:1006D0002A6A36EE677A77EE867A27EE267A67EE12
:1006E000A67A80ED027A44E6D0ED017A90ED026AB6
:1006F0005FED336A37EE867A77EEC67AEDE7D0EDB6
:10070000027A1FED366A1FED367AD0ED006A5FED92
:10071000375A27EE877A67EE867AA6EE867AE6EE75
:10072000A57A00E70AF03EFFBDE8084040F211124A
:100730004FF480010AF022BF90ED020A90ED017A99
:10074000D0ED007A20EE000AA7EE070AA7EEA70A6E
:10075000B1EEC00A704700BF7047000038B50568A9
:1007600004462DB12846FEF74BFE2846FEF7A2FAB6
:10077000204638BD13460246014802F095BA00BF34
:10078000E630002013B50422054B019304460146D0
:100790000DEB0200FFF7EEFF024B1C8002B010BD14
:1007A000FFFF3F00D830002007B5502304228DF80A
:1007B0000430412300210DEB02008DF805300623A3
:1007C0008DF806308DF80710FFF7D4FF0420FFF7EF
:1007D000D9FF03B05DF804FB00EB0212907B20B957
:1007E0001BB19289120758BF3F20984008447047B8
:1007F000430608D4000A08D0054B1B88184214BFD2
:10080000012000207047002070470120704700BF82
:10081000DC30002010B50B4B1A880B4B01301B68E5
:1008200080B2142404FB0033824207D9DC898C4255
:1008300003F1140304D0013080B2F5E7002010BDAD
:100840000120FCE7EA300020EC3000208289836838
:10085000D20648BF1B68184670470000828983682B
:10086000D20648BF1B6818467047000007B504232E
:1008700000220DEB03010B48019202F0F5F99DF8FF
:100880000430502B07D19DF80530412B03D19DF842
:100890000630062B01D0FFF787FF012003B05DF87B
:1008A00004FB00BFE630002082894368920705D52B
:1008B0001B68181E18BF01200B6070470120FBE762
:1008C00037B58B891446DA070D4605D523684A6883
:1008D00013442360012012E09B07FBD50A4B1B68E1
:1008E000142201A902FB0030FFF7DEFF48B1019995
:1008F00022686B680A44D3581BB15B1A236003B0AB
:1009000030BD0020FBE700BFEC3000202DE9F04FA8
:100910008BB01F469DF854800691142353430593D2
:1009200008F10603DBB2054616464FF0000B0793AD
:100930005FFA8BFA07EB0A1999F80F40002C4CD09C
:10094000062C28D1B8F10B0F21D84846FFF77EFFBF
:100950000446C8B1169B099309AA49463046FFF7D9
:10096000AFFF88B11499434652463846FFF734FF2B
:10097000099B0293079B0699CDE900033246234663
:100980002846FFF7C3FF18B90BF1010BD0E7002091
:100990000BB0BDE8F08F1499434652463846FFF736
:1009A0001BFFB0EB953FEFD1C5F30423A342EBD17E
:1009B0000B4C059B206809A91844FFF775FF002818
:1009C000E2D0D9F80430099A1344169A1344069ACF
:1009D00013602068059B1844DAE72046D8E700BF7B
:1009E000EC3000202DE9F04F1F4B5FFA80F8B3F890
:1009F00000A0C0F3403348EA03281C4B1E680F4692
:100A000087B00546C0F3042B00211FFA81F9CA45BF
:100A100027D9F3894345344620D1337C062B0FD1A7
:100A20003046FFF71BFFC8B10023CDE90133009327
:100A30004A46034639462846FFF768FF044609E060
:100A40009B450BD105A93046FFF72EFF0028F5D0B6
:100A5000059B3B60204607B0BDE8F08F013114369E
:100A6000D3E70024F6E700BFEA300020EC30002096
:100A70002DE9F04F98468DB0142353430693484B0D
:100A80009DF85890DDF868B004461868069B0E463D
:100A900018440AA91746FFF707FF00287DD0002356
:100AA000079309F10603DBB209939DF81CA006EB3E
:100AB0000A15EB7B002B70D0062B3BD12846FFF7A5
:100AC000C5FE0890002831D0B9F10B0F65D8179BEF
:100AD0000B930BAA29463846FFF7F2FE30B39BF87A
:100AE0000030012B59D85A1C0BEB83038BF80020E4
:100AF00041465D6052464B463046FFF76DFE1B9AFD
:100B00000899CDE904B2199A0392189A02920B9AA5
:100B10000192099A009203463A462046FFF7A8FF41
:100B200000BB9BF80030013B8BF80030079B013382
:100B30000793BAE7179A686810440A9A1044A042CB
:100B400013D14B46524641463046FFF745FE189BAF
:100B50001B9A1860199B1D6000231370104B1868B6
:100B6000069B18440DB0BDE8F08F052BDED1031DA8
:100B70009C4203D000F108039C42D7D11B9B201A52
:100B80008008187052464B4641463046FFF724FE17
:100B9000189B1860199B1D60E0E70020E2E700BF8A
:100BA000EC3000202DE9F04F8BB00025DFF8A4A039
:100BB000079306460F4690461560254B1B881FFA83
:100BC00085FB5B4541D9DAF80000142303FB0B04D5
:100BD00009A9204694F81090FFF766FE98B3B9F182
:100BE000060F17D12046FFF739FE014658B3149B74
:100BF0000593079B0297CDE903830023CDE90033DA
:100C00005A463046FFF734FF0446E0B120460BB0A9
:100C1000BDE8F08F0998B04204D1149A00233B60DC
:100C20001370F3E7B9F1050F0DD1031D9E4203D0F8
:100C300000F108039E4206D1149B301A80081870F8
:100C400000233B60E2E70135B7E70024DEE700BFA1
:100C5000EA300020EC3000202DE9F04798460D885E
:100C6000234B0446C5F30809186809EB890588B0C9
:100C700000EB850507A92846119E95F810A0174698
:100C8000FFF712FE20B90025284608B0BDE8F0871E
:100C90000021BAF1060FC8F8001013D12846FFF75B
:100CA000DDFD0028EFD0109B0091CDE90383CDE955
:100CB00001170B46059601464A462046FFF7D8FE27
:100CC0000546E1E70798A04202D139603170DBE7C1
:100CD000BAF1050FD7D1031D9C4203D000F10803E0
:100CE0009C42D0D1241AA408002334703B60CBE787
:100CF000EC3000200138C0B204289ABF014B185CC8
:100D000000207047DC5803082DE9F04F2DED028BD1
:100D100083B000240093931DDBB208EE103A054621
:100D20000E461746A246A0464FF0010BE0B2010165
:100D300005EB001090F80F90B9F1000F5AD0837BAB
:100D40003F2B02D92E4812F00FFF17B1002B08BF1E
:100D50003F23C3F1200EA3F1200C2AFA03F208FA74
:100D60000EFE28FA0CFC42EA0E0242EA0C0212F0D5
:100D7000010FC3F1200CA3F12002E3D10BFA02F220
:100D80002BFA0CFC42EA0C020BFA03F3B9F1060F42
:100D900043EA0A0A42EA080813D10B2FD2D8FFF718
:100DA00055FD814658B16858FAF7FEFA009B184481
:100DB000C3B218EE102A31464846FFF7A5FF0134AA
:100DC000B4E74846FFF796FF01900028BAD068586C
:100DD000FAF7EAFA009B1844C0B2B9F1050F04BF54
:100DE0000230C0B21028019BACD8308804300344D4
:100DF0003380E4E703B0BDEC028BBDE8F08F00BFA9
:100E0000A05703082DE9F04F85B00423DFF8989030
:100E1000ADF80E3000244FF0140A214B1B881FFA46
:100E200084F8434539D9D9F800300AFB08F15D1838
:100E30002F7CB5F80EB0062F23D1B8F1000F02D1E8
:100E4000184812F091FE28460193FFF707FD064669
:100E5000A8B1019B5858FAF7A7FA0022C3B20DF1C6
:100E60000E013046FFF750FF59464046FFF7D2FCCF
:100E70000028E5D1062F02D0AB899B07E0D40134CE
:100E8000CBE73846FFF736FF0028D9D0BDF80E3043
:100E900004331844ADF80E00E6E705B0BDE8F08F66
:100EA000EA300020A0570308EC300020437803F01C
:100EB0001F021F2A0FD00278C3F3401342EA032314
:100EC00040F2FF12934206D000680138C31C94BF61
:100ED0000020012070470120704700002DE9F341F8
:100EE000224FDFF8908006460D4604247B88A342FB
:100EF00037D904230DEB03012246384601F0B4FE36
:100F00009DF80510737881EA0302D20618D196F88D
:100F100000C09DF80400C3F34013C1F340124CEA33
:100F2000032340EA022293420AD13268019B5340D4
:100F300013EA080F04D12C80012002B0BDE8F08133
:100F400001A8FFF7B3FF20B1094B2C801C800020C3
:100F5000F3E701F01F00FFF7CDFE031D1C44A4B210
:100F6000C4E74FF6FF732B80F1E700BFE6300020A7
:100F7000D830002000C0FFFF70B50C462046114657
:100F800015461E4620F0DEFC831CAB420AD85F22C9
:100F9000225422180330A84206F1580656709CBF0E
:100FA0000022E25470BD00002DE9F74FDDE90D5439
:100FB00007468A46164609689DF830809B462246B9
:100FC0009DF83C300093284620F0A8FC4FF0000923
:100FD0009BF800105FFA89F29142019212D92146E2
:100FE000284620F0AFFCC0B28442019A07D90BEB2F
:100FF00082025168221A0968284420F08FFC09F106
:101000000109E5E7E6B12146284620F09BFCC3B282
:101010009C4204D93168E21AE81820F07FFC009B5A
:1010200013B9B8F1000F13D0F37B052B10D1434651
:1010300022462946384603B0BDE8F04FFFF79CBF73
:10104000009B13B9B8F1000F02D09AF81030ECE70A
:1010500003B0BDE8F08F0000F0B58BB007AC1F46C1
:101060000023C4E9013307930DF11303CDE90043D5
:10107000154606AB05AA0646FFF7EEFD014610B978
:1010800028700BB0F0BD9DF84030069A0195CDE96F
:1010900002739DF81330009330462346FFF784FF18
:1010A000EFE700002DE9F04F984689B014234B4339
:1010B000DFF828A1039204460E4604934FF000097E
:1010C0005FFA89F52B0108EB0515059395F80FB02C
:1010D000BBF1000F7FD0BBF1060F58F803702AD187
:1010E0003846FAF761F939460246204620F0E0FB1F
:1010F000002869D12846FFF7A9FB0746002863D0DE
:10110000039B079307AA29463046FFF7D9FB00281F
:101110005AD0059B58F80300FAF746F9129B009342
:10112000079A3B4631462044FFF7BCFF00284BD0CE
:1011300009B0BDE8F08F3946204620F089FB88B918
:10114000DAF80000049B07A91844FFF7ADFB00285C
:101150003AD0129B83F800B06868079B1844039B41
:101160001844E5E7BBF1050F2ED11021384620F0D9
:10117000E9FB5FFA80FB5A463946204620F0BAFB6D
:1011800010BB14F90B305F2B1ED10BF1010B14F8BF
:101190000B30583B022B17D8DAF80000049B07A944
:1011A0001844FFF781FB78B16868079B129A1844CE
:1011B000039B18440423137014F90B30592B06D0E9
:1011C0005A2B06D0582BB3D009F1010978E7043027
:1011D000AEE70830ACE75846AAE700BFEC30002085
:1011E0002DE9F04F8BB0DFF8C8B0029104461746E6
:1011F00000252E4B1B881FFA85FA534552D914221D
:1012000053465343DBF8002002EB0309D35899F807
:101210001080B8F1060F33D110211846039320F047
:1012200091FB039B5FFA80F842461946204620F066
:1012300061FB0646002833D14846FFF70FFB034603
:1012400070B3029A009204EB080032465146FFF751
:1012500029FF804620B37FB10DF11303009306AA46
:1012600007AB05A9CDE9076605960996FFF79AFC35
:10127000069B0BB19B893B8040460BB0BDE8F08FCD
:101280001946204620F0E4FA50B9029B07A983F8DA
:1012900000804846FFF708FB20B1DDF81C80EBE733
:1012A0000135A6E74FF00008E6E700BFEA3000206E
:1012B000EC3000202DE9F04F87B01425DFF898B00E
:1012C000039206460F4698464D434FF00009039A95
:1012D0005FFA89F302EB031A9AF80F40ECB1062C7F
:1012E00037D1DBF8000004A92844FFF7DDFA0446F3
:1012F00078B30499DAF80420BAF80C000A4483079A
:1013000002EB08010DD552F80820B2420BD1DBF8F0
:101310000030109A1D44EB891380204607B0BDE8C9
:10132000F08F8E42F2E705AA51463846CDF8148078
:10133000FFF7C6FA68B15046FFF788FA024640B197
:10134000109B00933946059B3046FFF7B3FF0028FA
:10135000E3D109F10109BAE7EC3000202DE9F743A8
:10136000184FDFF8648004460D4600264FF014093C
:101370003B88B1B28B4222D9D8F8003009FB01304A
:10138000037C062B01D00136F2E783899B0709D540
:1013900043681B68A34205D1C3892B80012003B099
:1013A000BDE8F083FFF75AFA02460028EBD000951B
:1013B00000232046FFF77EFF0028E4D0EFE700205F
:1013C000EDE700BFEA300020EC30002030B50B4BD9
:1013D0001C880B4B1B68002295B2AC420CD91D7CBB
:1013E000062D06D15D68854203D1DB890B80012083
:1013F00030BD01321433EFE70020F9E7EA30002076
:10140000EC30002010B590B00023CDE908330693EE
:101410000A930DF11703009306A908AB07AA044627
:10142000FFF7C0FB014668B111230122CDE902326A
:101430000BAB01939DF817300093079A08AB204639
:10144000FFF7B2FD10B010BDF0B5304D87B040F2DF
:10145000A51202908DF80C1006460C4601A8291D15
:10146000FDF7B4FD052204A92868FEF70FF9074629
:1014700001A8FDF7CDFD052F06D1049BB34203D192
:101480009DF81430A3423ED0214E224F4FF4B0724B
:10149000314601A8FDF79AFD2868FEF71BF80428DD
:1014A00021D92868052202A9FEF78AF8431F5C4269
:1014B0005C4101A8FDF7ACFD2CBB3C68E36A93F8E6
:1014C0009C3093B9A06A036801211B699847A06A00
:1014D00003684FF4FA719B689847A06A036800217B
:1014E0001B699847D2E70024E3E7A06A03681B6CF6
:1014F00098470028E6D00AF055F840F2FA424FF437
:1015000080110AF03BF807B0F0BD00BFB0300020FA
:10151000B4300020D81000202DE9F341154E164FAD
:10152000C92406F10408013CA4B2FCB140F24B12FC
:10153000414601A8FDF74AFD3068FDF7B1FF0546B9
:1015400001A8FDF765FD042D10D93D68A86A036860
:101550000A211B699847A86A03680A215B689847B3
:10156000A86A036800211B699847DCE702B0BDE860
:10157000F08100BFB0300020D810002000B58BB043
:101580000023CDE90733049309930DF10D03009374
:1015900005AA07AB04A9FFF705FB10B3059B23B30E
:1015A000DB7BC2898DF8182003F01F03C2F30022F1
:1015B0001B0243EA4233049A43EA82339DF818201F
:1015C0000DF10E01134306A80693FFF787FC40B107
:1015D0009DF8193003F01F03052B03D09DF80D3043
:1015E00003B100200BB05DF804FB037CD9E70000D9
:1015F000F0B5144F3B8889B006460D46FBB10DF19E
:101600000B030024009304AA05AB03A9CDE905440C
:1016100003940794FFF7C6FA88B10B4B38881B6810
:10162000A2B290420BD91A46013411688E4203F1DE
:101630000C03F5D1137A2B70012009B0F0BD002006
:10164000FBE700BFE0300020D430002013B50DF1DF
:1016500007010446FFF7CCFF10B92046FFF78EFFC5
:1016600002B010BD07B5074B1B884BB10DF1070148
:10167000FFF7BEFF08B19DF8070003B05DF804FB5B
:101680001846FAE7D030002010B50C46FFF7EAFF05
:1016900040B9A30608D5054B1B6813B1186AC0F3FF
:1016A000800010BD0020FCE70120FAE7F840002090
:1016B0000138032816D8DFE800F002080E13FDEE0B
:1016C000C07A17EE903A0B707047BDEEC00A10EE6C
:1016D000103A0B807047BDEEC00A81ED000A7047DA
:1016E00081ED000A7047000037B5036803F000433E
:1016F00003600A4B1B880C4613B9002003B030BDB1
:10170000074D01A92868FFF7CFF80028F5D014B1DC
:101710002B681B7C23700198F0E700BFEA300020A3
:10172000EC3000202DE9F04F8FB09B469DF87030D3
:101730000B93142343439DF860901A9D0A93074628
:1017400088460892002307939DF81CA008EB0A1610
:10175000F47B002C00F0BC80B089FFF749F800282A
:1017600000F0B380062C2FD13046FFF76FF8044607
:10177000002800F0AA80199B0D930DAA3146384627
:10178000FFF79EF8002800F0A0804B4652465946CD
:101790004046FFF721F81D9A05920B9A04921B9A76
:1017A000CDE902520D9A019209F10602D2B2034626
:1017B00000922146089A3846FFF7B4FF002800F04F
:1017C00084800FB0BDE8F08F089B1B780993002B35
:1017D0003CD02B8867F308032B8052464B46594672
:1017E0004046FEF7F9FF3B4B03EA40302B6823F0FD
:1017F000FF4323F4FF0323F4FC4318431B9B28609F
:1018000003B11C70344B18680A9B0DA91844FFF7EC
:101810004BF8002859D00D9A73681344199A9818F8
:101820000B9A002ACDD02D4A1278002AC9D0F27B1B
:10183000012AC6D1B2895207C3D5199A9B56002BEB
:10184000BFD1EB7843F08003EB70BAE74B465246CA
:1018500059464046FEF7C0FF2B68C3F35133984208
:1018600033D1089A0123137095F90330002B06DA5F
:10187000EB78099A62F3C713EB701046A1E7052CC9
:1018800023D16B78C3F34302022A1ED8013262F3DC
:1018900044036B701B9B13B11B9A042313700E4BF4
:1018A00018680A9B0DA91844FEF7FEFF68B170681E
:1018B0000D9C95F801B0199B2044CBF3430B1844C1
:1018C0000BF1FF3B00EB8B007BE7079B01333AE713
:1018D000204676E700E0FF7FEC3000200C0E002071
:1018E0002DE9F04F8BB0DFF8EC90048807920022CE
:1018F0008DF82720B9F800201F46C4F308039A4248
:1019000005460E461C4662D9DFF8CC801BB2D8F8DB
:10191000001003EB83039A0001EB83031B7C052B70
:1019200018D14378C3F34301022915D8013161F37B
:10193000440343700EB104233370D8F80010687864
:101940000A44C0F34300431E506800EB83000BB011
:10195000BDE8F08F062B04D001340123A4B28DF82A
:1019600027304FF0140B4FF0000AB9F80030A342B3
:101970002DD9D8F800200BFB04229089FEF738FF00
:10198000B8B1117C062917D11046FEF767FF014652
:1019900078B1079B0597CDE90363CDE901A5CDF8A3
:1019A00000A000230DF127022046FFF7BBFE002810
:1019B000CDD10134A4B2D8E72B68C4F3080403F0F6
:1019C000004323432B6006B131705068BFE700200D
:1019D000BDE700BFEA300020EC30002073B50546BB
:1019E0000C461646334601220DF107012846FFF743
:1019F00077FF28B19DF80730042BF3D804B123708A
:101A000002B070BDF8B514460746002220460E46C7
:101A1000FFF76AFE002540B1BD4206D000223146E4
:101A20002046FFF7DBFF0135F5E7F8BD0139032953
:101A30000BD8DFE801F00204060801F095B801F0C8
:101A4000CBB801F0F1B801F04DB89FED010A704735
:101A50000000C07F37B5037A02888DF8042003F0B8
:101A60001F03C2F300221B0243EA4233426843EAE7
:101A700082339DF804200C4613430DF1020101A8A6
:101A80000193FFF72BFA054670B19DF8050000F0B1
:101A90001F00FFF72FF9BDF802200432034692B26F
:101AA0000348214601F0E0F8284603B030BD00BFEE
:101AB000E63000202DE9F0472DED028B82B0044680
:101AC00000AF007AFFF716F9C31D23F00703E946BC
:101AD000ADEB030D0E46804669462046F0EE408A87
:101AE000EA46FFF7B7FF88B3E0680022F91DFFF769
:101AF00077FB054640B9344BE2681B683349986967
:101B000003681B68984721E0B2071BD5227AFB794E
:101B10009A4222D1F7EE000AB0EE680AFEF716FAF2
:101B2000D8B1D6B94246514628461FF0C5F968B12A
:101B30005146424628461FF0CFF931462846FFF766
:101B400083FC03E0FFF71AFD0028DFD00837CD46FD
:101B5000BD46BDEC028BBDE8F087FB79042B07D9AD
:101B6000194BE2681B681A49986903681B68C9E742
:101B7000217A0429F4D85046FFF758FFF307B0EE56
:101B8000408A0BD5FFEE000AFEF7E0F99FED110A3F
:101B90000028B7EE008A08BFB0EE408AF9792846DF
:101BA000FFF744FFF0EE400AB0EE480AFEF7CEF928
:101BB00002460028CAD1294628EE280AF879FFF7FC
:101BC00077FD1146BAE700BFD8100020B4570308CC
:101BD000CD5703080000000070B515462DED028BAF
:101BE0000446B0EE408A00EB0116B44207D020460E
:101BF0002946B0EE480AFFF75DFF1034F5E7BDEC6B
:101C0000028BBDE87040FFF787BC0000B7EE000A0A
:101C1000FFF7E2BF2DE9F04F2DED028B8BB002AF45
:101C200005460E46B0EE408A9146FFF7A7FC0446F3
:101C300038B1002420462437BD46BDEC028BBDE8F8
:101C4000F08F7B1DC7E90500B860F861009307F1CC
:101C50000C0207F1140307F108012846FEF7A2FF62
:101C60000028E6D0FB68002B3DD093F80F80C38995
:101C70003B74C3F3002206F01F031B0243EA423306
:101C8000BA6843EA82333A7CB91D134307F1100066
:101C90003B61FFF723F982460028CAD03046FFF7A0
:101CA00029F8C31D23F00703FA88ADEB030D0DF1EE
:101CB000080B0432034692B21B48594600F0D4FF89
:101CC000B9F1000F12D131465846FFF7AFFE294651
:101CD00020EE080A4046FFF7EBFC01212846FFF7FB
:101CE000B3FB5446A6E790F81080C0E7022E10D050
:101CF000032E11D0012E9DD19BF80030B8F1020FB8
:101D00000DD0B8F1030F0CD0B8F1010F92D12B70A8
:101D1000E3E7BBF80030F1E7DBF80030EEE72B80BB
:101D2000DBE72B60D9E700BFE6300020B4EE400AC5
:101D3000F1EE10FA10B504460CD69FED327AF0EEB3
:101D4000C07AF4EE477AF1EE10FA03DC042902D1EE
:101D500080ED000A10BD032919D1B5EEC00A9FED30
:101D60002A7ADFED2A7A9FED2A1ADFED2A0AF1EEB0
:101D700010FA58BFF0EE477A30EE270A40F6C90055
:101D8000FEF720F9BDEEC00A84ED000AE2E7022961
:101D90001AD1B5EEC00A9FED1C7ADFED1C7A9FEDDB
:101DA0001E1ADFED1E0AF1EE10FA58BFF0EE477A68
:101DB00030EE270A40F6CE00FEF704F9BDEEC00A69
:101DC00010EE103A2380C5E70129C3D1B5EEC00A51
:101DD0009FED0D7ADFED0D7A9FED111ADFED110AFF
:101DE000F1EE10FA58BFF0EE477A30EE270A40F6CF
:101DF000D300FEF7E7F8FDEEC07A17EE903A2370B5
:101E0000A8E700BFFFFF7F7F0AD7233C0AD723BC88
:101E10000000004F000000CF00FEFF46000000C79A
:101E20000000FE42000000C32DE9F3411D4690F979
:101E30000030232B0F4690464FF000042CD017495A
:101E4000019401AA20F030FC064618B9002002B027
:101E5000BDE8F081F9F7A8FA1028F7D80F4901AAD0
:101E6000204620F021FC0028F0D0214620F098FBED
:101E70000A4988ED000A01AA3E60204620F014FCC1
:101E800030B10749F9F786FA10B901202870DEE76A
:101E900000232B700120DAE72046D8E7E857030833
:101EA000EF57030830B504469DB00D460EF094FB85
:101EB0000123214600220EF01DFB431C044624D0C2
:101EC0000EF08AFB2346632203A90EF04BFBA0B160
:101ED0000DF1020302AA01A903A8FFF7A5FF00283C
:101EE000EED0019800220DF10301FFF779F90028E7
:101EF000E6D02B8801332B80E2E70EF06DFB214604
:101F00000EF022FB01201DB030BD0020FBE70000D9
:101F10002DE9F0479EB0154601900EF05DFB0123C0
:101F2000019900220EF0E6FA431C064602D133481E
:101F300011F01AFEDFF8CCA0DFF8CC80DFF8CC90EF
:101F400001270EF049FB3346632205A90EF00AFB78
:101F5000F0B10DF10A0304AA03A905A8FFF764FF75
:101F60000028EED0039800220DF10B01FFF738F99D
:101F7000044600283FD02A88BAF80030934212D88D
:101F800009F010FB40F64C124FF4801109F0F6FAFC
:101F90000EF022FB31460EF0D7FA194B01201F70CC
:101FA0001EB0BDE8F0870C20D8F8001042438C50DA
:101FB0002A88D8F80030049900FB02325160298841
:101FC0009DF80A2000FB01331A7222B1B9F80030E3
:101FD0000133A9F800302B8801332B802046FFF70E
:101FE000CDFA0028ADD19DF80B109DED040A2046D6
:101FF000FFF79CFEA5E70746A3E700BFFC570308D1
:10200000E4300020E2300020D4300020D030002026
:102010002DE9F7430D46064600286DD01CF09CF9CB
:10202000074610B9354811F09FFD00233449ADF83B
:10203000003001AA019320F037FBDFF8C48088B19B
:102040006946FFF72FFF044630B938461CF05CF9AB
:10205000204603B0BDE8F08301AA4146002020F0ED
:1020600023FBECE7DFF8A89038461CF04DF9D9F8CF
:10207000000008B1FCF722FE224BDFF89880224FC7
:1020800000241C80BDF80030A8F800400C20584304
:102090003C80FCF70DFEC9F8000008B91B48C2E7F8
:1020A000BDF80030A8F8003023B3304601941CF08E
:1020B00053F906460028B5D01149ADF8024001AAEF
:1020C00020F0F2FADFF8388070B10DF102022946F3
:1020D000FFF71EFF044608B93046B7E701AA41469C
:1020E000002020F0E1FAEFE730461CF00DF9BDF8D2
:1020F00000303B800124ABE70446A9E728580308D9
:1021000054580308D0300020E0300020565803080F
:10211000D4300020E230002010B50446FFF778FFED
:1021200028B921460248BDE8104010F0A1BF10BDFB
:10213000805803082DE9F0434FF000089DB0054694
:102140000E461746A2F80080002E35DDB2B20023FD
:102150009CB2A24203F1010902D9EB5C0A2B29D1FE
:10216000632C28BF63242246294603A81EF0B4FE30
:102170001CAB1C44A6EB090604F8648C9DF90C30DA
:10218000232B4D44E0D0002BDED00DF1020302AA38
:1021900001A903A8FFF748FE0028D5D00198002226
:1021A0000DF10301FFF71CF80028CDD03B88013367
:1021B0003B80C9E74B46CBE701201DB0BDE8F0836B
:1021C0002DE9F04FDFF828810546D8F800009FB0D0
:1021D0000E4608B1FCF772FD434FDFF818A1DFF897
:1021E000189100240DF10A0231462846C8F8004033
:1021F0003C80AAF80040A9F80040ADF80A40FFF77B
:1022000099FF00286DD0BDF80A300C205843FCF728
:102210004FFDC8F8000010B9344811F0A5FCBDF816
:102220000A303B80A346BDF80A30A34257D9002E9E
:1022300055DDB1B2002297B2B94202F1010302D9D1
:10224000AA5C0A2A49D1632F28BF63273A46294648
:1022500005A801931EF040FE1EAB1F44019B07F82A
:1022600064BCF61A1D449DF91430232BDBD0002BDF
:10227000D9D002AB04AA03A905A8FFF7D5FD002811
:10228000D1D0039800220DF10901FEF7A9FF0746FE
:102290000028C8D00C2303FB04F2D8F80030985073
:1022A000D8F800301344049A5A609DF808201A7236
:1022B00022B1B9F800300133A9F8003001343846B2
:1022C000A4B2FFF75BF90028ADD19DF809109DED90
:1022D000040A3846FFF72AFDA5E71A46ABE7AAF835
:1022E00000301FB0BDE8F08FE230002056580308E0
:1022F000D4300020E0300020D030002002460248D8
:10230000418A1430FFF75CBFE458030810B50A4B4C
:102310001B680446D86A03685B69984710B1214678
:10232000FFF7FAFE054B5B8A23B12046BDE810405B
:10233000FFF7E4BF10BD00BFD8100020E458030829
:1023400030B5002085B0FFF7E1FF214B1A7872B954
:1023500001221A701F4B204A1B680292986A1F4A7A
:102360000368039204AA12E906009B6A98471C4D71
:1023700004246B88A34229D90423224669462846AF
:1023800000F072FC6846FEF791FD18B1154B1C80F9
:1023900005B030BD009801A9FEF724FB60B19DF89F
:1023A000010000F01F00FEF7A5FC221D0346019965
:1023B00092B2284600F058FC9DF8010000F01F0082
:1023C000FEF798FC04300444A4B2D2E70020DFE713
:1023D000E5300020D81000209330002009290108A2
:1023E000E6300020D830002070B50E4B1E880E4B12
:1023F0001B68002294B2A64209D91C460132256806
:10240000854203F10C03F5D194ED010A70BD8B896F
:102410001B0649BF8B6891ED020AC01A90ED000AB5
:10242000F4E700BFE0300020D43000202DE9F04177
:1024300005460F464FF000085FFA88F307EB0311DB
:10244000CC7BDCB1042C0BD84E682E443046FFF711
:10245000CBFF31462046FFF72BF908F10108EBE7E7
:10246000052CFAD14C682C442046FFF7BDFF84EDC3
:10247000000A84ED010A84ED020AEEE7BDE8F0816E
:1024800070B50E4B1E880E4B1B68002294B2A642FC
:1024900009D91C4601322568854203F10C03F5D1A8
:1024A00094ED010A70BD8B891B0649BF8B6891EDC5
:1024B000020AC01A90ED000AF4E700BFE0300020E5
:1024C000D43000202DE9F0418AB00023CDE9073354
:1024D000039309930DF10903009304AA07AB03A921
:1024E0000446FEF75FFB054620B9002630460AB0D9
:1024F000BDE8F081049B002B3AD0DB7BEA898DF8A4
:10250000142003F01F03C2F300221B0243EA4233EC
:10251000039A43EA82339DF814200DF10A01134314
:1025200005A80593FEF7DAFC064658BB06A928461F
:10253000FEF7BAF90028D9D09DF815700499DDF896
:10254000188007F01F07B9B19DF81C3093B1089AA5
:10255000012B556802D0099B5B681D442046FFF79C
:1025600043FF4968414429443846FFF7A1F8BDE7D5
:10257000037CC3E73546F1E729462046FFF780FF95
:102580004146F1E79DF815009DF8093000F01F0263
:10259000052A0FD0002BA8D100F01F00FEF7AAFBE0
:1025A000BDF80A200432034692B22146044800F0E6
:1025B0005BFB9BE7002BEFD0A4EB8304ECE700BFB1
:1025C000E63000202DE9F04385B0FEF74FF9134EB9
:1025D000134F00254FF014083288ABB29A4219D934
:1025E0001C463B6808FB043494F81090B9F1040FC2
:1025F0000ED803A92046FEF757F948B10398019079
:102600002146FFF73DFF019801464846FFF750F885
:102610000135E1E705B0BDE8F08300BFEA300020F6
:10262000EC3000202DE9F347DFF88C901F4940F68D
:1026300078226846FCF7CAFCB9F800702FB11C4B31
:102640001A881C4B1B889A4228D0194E194D052414
:102650004FF00008B9F800701FB132882B889A42F9
:102660001CD0013C14F0FF0418D00022114601A830
:102670003788CDF80480FFF737F84FF0000A1FFACB
:102680008AF30AF1010A28B10022114601A8FFF7D6
:10269000A5F9F4E7A9F800302F80DBE76846FCF7DE
:1026A000B7FC384602B0BDE8F08700BF9430002088
:1026B000CE300020DE300020DA300020024A1388BD
:1026C00001331380704700BFCE3000202DE9F04168
:1026D0002DED028B90B00023CDE9083305930A93CA
:1026E0000DF1110300930E4608AB06AA05A9044696
:1026F000FEF758FA0546D8B10699F1B1CA7BEB89C5
:102700008DF81C3002F01F02C3F300201302059A5B
:102710009DF8117043EA403343EA82339DF81C2050
:102720001A43C3F30423052B079200F0868037B1C8
:1027300010B0BDEC028BBDE8F081027CDFE7012B1D
:1027400005D121B18B895B0701D5FFF7B7FF27467C
:1027500077E0BDF812204FF6FF739A420AD14C4B36
:1027600083F800804B4B4C491B68986903681B68D1
:102770009847DDE79DF81D1001F01F01042925D9B8
:102780009DF81D00BDF81220444900F01F00FEF71F
:10279000B1FA4988131808338B424AD204321044E4
:1027A00080B2FDF7EFFF9DF81D0000F01F00FEF75F
:1027B000A1FABDF812100431024689B23846FDF77D
:1027C000D9FFBDF81210042207A85EE02046FFF7EB
:1027D0002DF90699F0EE408A71B12046FFF704FE0C
:1027E000B0EE408AF0EE400AB0EE680AFDF7AEFBAC
:1027F00038B1002EC4D19BE729462046FFF740FEA2
:10280000EEE7002EBCD19DF81D3003F01F03032B13
:10281000B6D09FED230A38EEC88AF0EEE88A68EE5B
:10282000808AB0EEC88AB4EEE88AF1EE10FAA7D535
:102830007EE7174B01221A7094E7002F87D0A4EB94
:10284000870711234FF00108CDE902380BAB019344
:102850009DF81130009329462046069A08ABFEF7F2
:10286000A3FB0DF1120107A8FEF738FB00283FF487
:1028700070AF9DF81D0000F01F00FEF73BFABDF899
:1028800012100431024689B23846FDF773FF4FE754
:10289000CC300020D8100020A4580308E6300020D7
:1028A00017B7D1387FB5164D2E1D40F27F12314635
:1028B00001A8FCF78BFB2868FCF7F2FD042812D96D
:1028C0002868052202A9FCF7FDFE431F5C425C411B
:1028D00001A8FCF79DFB44B19DF80C100298012261
:1028E000FFF7F4FEE1E70024F2E7064B1B68986A65
:1028F00003685B6B984708B1FFF794FE04B070BDA6
:10290000B0300020D8100020FFF7CCBF2DE9F043F5
:1029100085B088460DF106010646FEF71FFD48B951
:10292000374B38491B68986903681B68984705B09E
:10293000BDE8F083DFF8D8900027FDB208EB05155D
:10294000EB7B002B53D0062B11D10023BDF80600E2
:10295000039303AA2946FDF7B3FFC8B12846FDF744
:1029600075FF014618B103983044FFF7CFFF0424E8
:10297000B9F80230A3420BD90423224602A94846E3
:1029800000F072F902A8FEF791FA18B11E4B1C80F4
:102990000137D2E79DF80930BDF80610C3F34012A5
:1029A0009DF8083043EA0223994216D1029803A900
:1029B000FEF718F888B16B680399334499420CD13B
:1029C0009DF8090000F01F00FEF794F9221D034650
:1029D00092B2484600F048F9DAE79DF8090000F0A5
:1029E0001F00FEF787F9021D224494B2C0E7074B8F
:1029F000187808B9FFF78AFCFFF760FE97E700BF79
:102A0000D8100020B4580308D8300020E43000204B
:102A1000E630002010B50446FCF74CF9204610BD06
:102A200038B51148114D10F0A7FA114A11490E4856
:102A30001CF048FA2846002340F8043B10F09CFAAA
:102A40001420FCF72FF9044610B19B21FCF7C6FCBB
:102A50000949074A05482C601CF034FABDE83840A3
:102A60000648002100F0F8B894300020B030002073
:102A7000E4400020590701085D070108E630002006
:102A800038B504460D46FEF7E1FD08B92B68236012
:102A900038BD000091ED007AD0ED007ADFED086AD4
:102AA00080ED007A77EEC77AF0EEE77AF4EEE67A18
:102AB000F1EE10FA4CBF01210021FEF7C5BC00BFAA
:102AC00000000034D1ED007A90ED007AF4EE477A00
:102AD000F1EE10FA04D0C0ED007A0121FEF7B4BC8B
:102AE0007047000090ED000A7047000038B50446BA
:102AF0000D46FEF7ABFD10B995F90030237038BDD7
:102B000091F900300370704791F9002090F900109E
:102B1000914202D00270FEF775BC704791F9001027
:102B200090F900309FED097A01705B1A07EE903A38
:102B3000F8EEE77AF0EEE77AF4EEC77AF1EE10FA03
:102B40004CBF01210021FEF77FBC00BF0000003414
:102B500091F9002090F90010914203D002700121F8
:102B6000FEF772BC7047000090F9003000EE103A9A
:102B7000B8EEC00A7047000038B504460D46FEF7AF
:102B800065FD10B9B5F90030238038BDB1F90010EA
:102B9000B0F900309FED097A01805B1A07EE903A98
:102BA000F8EEE77AF0EEE77AF4EEC77AF1EE10FA93
:102BB0004CBF01210021FEF747BC00BF00000034DC
:102BC000B1F90020B0F90010914203D00280012138
:102BD000FEF73ABC70470000B0F9003000EE103A42
:102BE000B8EEC00A7047000038B504460D46FEF73F
:102BF0002DFD08B92B68236038BD00000B68036009
:102C0000704700000A6801688A4202D00260FEF73D
:102C1000F9BB70470A6801688A4203D0026001214B
:102C2000FEF712BC7047000090ED000AB8EEC00A33
:102C30007047000008B5064B1B68586903685B685D
:102C4000984720B9BDE80840024810F011BA08BD05
:102C5000D8100020F85A0308017011B100234380F6
:102C600070474FF44873FAE770B51C460378A3B970
:102C7000B2F5487F11D212FA84F3B3F5487F094BBD
:102C80001B685869C8BFC2F548750368D4BFA5B2B0
:102C9000ADB29E682B46B047641BB4FA84F040097D
:102CA00070BD00BFD810002070B51C460378A3B9D2
:102CB000B1F5487F11D211FA84F3B3F5487F094B7F
:102CC0001B685869C8BFC1F548750368D4BFA5B271
:102CD000ADB2DE682B46B047641BB4FA84F04009FD
:102CE00070BD00BFD810002010B5044601F02AFBCB
:102CF0004FF0FF33E36204F1300010F03DF904F1CE
:102D0000640011F021F80023C4F88C30C4F890302E
:102D1000C4F8943006492046FFF788FB054B1A6833
:102D200012B1054810F020FF1C60204610BD00BF06
:102D3000805C0308F4300020185B0308084699B152
:102D4000C81FC3B2102B0ED810280CD8DFE800F033
:102D5000090B090B0B0B0B090B0B0B0B090B0909CF
:102D600009000020704701207047000007B50DF1F1
:102D70000601FEF72BFB08B312490B68DB0718D4DA
:102D8000114BBDF806201A801A821A841A86A3F8FD
:102D90004020A3F85020A3F86020A3F87020A3F8E7
:102DA0008020A3F89020A3F8A020A3F8B02001234E
:102DB0000B60054800220C21FEF728FF03B05DF8E8
:102DC00004FB00BFF0300020100E0020F7B50446D1
:102DD0000DF1070101278DF80770FFF787FE2046E8
:102DE000FFF7C4FF94F91530032B15D104F1280621
:102DF0003046FEF72BFC054670B90DF10701304651
:102E00008DF80770FFF78AFE0DF1070104F1150038
:102E10008DF80750FFF782FE04F092FA21780546FC
:102E20002046FFF78BFF30B100220521284604F031
:102E300061F9C4F80C010023E36184F85830638819
:102E4000013B9BB2C72B84BFC823638003B0F0BD96
:102E5000B02303FB010191F8A90010B1D1F898301B
:102E600013607047B02303FB010191F8AA0010B171
:102E7000D1F89C3013607047B02303FB010191F837
:102E8000AB0010B1D1F8A030136070472DE9F843C2
:102E9000B02303FB01038446D3F8B8200F4622B9C0
:102EA000D3E9300150EA01032CD0B02606FB07C657
:102EB000B6F8600000283FD0D6E930231F4DDFF878
:102EC00080901343A0FB05451ED042375CF82700D5
:102ED00003F0AAFD074610F071FE14EB090245F15C
:102EE0004904D3194FF47A7544F10004A3FB053269
:102EF00005FB0422D6E93045001B61EB05011818DB
:102F000042EB0101BDE8F883F06D492310EB0900A5
:102F100043F10003071945EB030410F04DFED6F80A
:102F2000B810401AC0194FF47A7344F10004A0FBA2
:102F3000030103FB0411E5E70146E3E700840C24E9
:102F4000B0F5F79010B5B02303FB0103B3F8604070
:102F5000ACB1423150F8210003F066FD094BA4FBEF
:102F60000313094C091943F149034FF47A72081805
:102F700043F10003A0FB020102FB031110BD204638
:102F80002146FBE700840C24B0F5F79000EBC1016B
:102F9000C1F82821A1F82C317047000001EB810312
:102FA00010F92330022B0BD1C38C5B0718D500EB33
:102FB000C1000D4BC0F828312E23A0F82C317047EA
:102FC000DBB21A2B0CD8012202FA03F3074A1A408B
:102FD00032B100231A4600EBC100C0F82821ECE70B
:102FE000034A2E23F7E700BF205D0308008C00048E
:102FF000505C030838B50446F9B9D0F80C01E0B1CB
:10300000B4F82C31CBB103689B6A9847D4F80C31E3
:10301000B4F82C2119688242CD68D4F8281128BF51
:1030200002461846A847D4F828310344C4F828318A
:10303000B4F82C31181AA4F82C0138BD2DE9FF473B
:1030400001EB8103044610F923500F4600EB83087F
:10305000002940F01D81A5F10903D0F80C610E2B69
:1030600029D8DFE813F029002800100028002800E4
:10307000290028002800280028001B01280028001B
:10308000290029000026142303FB0743002283F8AC
:1030900020214FF4FC70FBF705FE0546002800F0E8
:1030A0001381B02303FB0743009658334246214661
:1030B00000F050FC08E10EB9002505E1012380F87D
:1030C000203110F079FDD4F81431C31AB3F5966F9E
:1030D000074625D9D4F81C31002B3FD13368304640
:1030E0001B6E9847C4F81C01122D48D0112D4FF0CB
:1030F000000348D14FF40062D4F81C113046FCF7AD
:103100000DF833680021DB6B3046984794F9243082
:10311000C4F81471002B0BDD00212046FFF73EFFA1
:1031200094F92430002B03DD00212046FFF762FFD5
:103130000F2D2AD025F010030A2B36D14FF4D07072
:10314000FBF7B0FD0546002800F0BE80009604F1B4
:1031500058034246214601F07FF9B5E094F8183152
:103160000133DBB2082B08BF002384F8183194F830
:103170001821574B53F82230C4F81C31B4E74FF4F0
:1031800000630022B8E71A46B6E74FF4CC70FBF7AD
:1031900089FD0546002800F09780009604F1580349
:1031A0004246214600F0B4FE8EE0B4F82C31002BEC
:1031B00082D1336830465B6998475FFA85FAB0F58B
:1031C000005F28BF4FF400500AF1FF3987B25FFA61
:1031D00089F9002F3FF470AF336830469B699847F8
:1031E000B9F1010FC1B20AD894F81821384B53F83D
:1031F000223094F9242052BBB3F5164F30D2E38C21
:10320000AAF1110213F0010F14BF4FF461334FF410
:10321000E123012A18D894F818012D4A52F82020E9
:103220009A4211D104F2211002F0B8F860B1112DC8
:103230004FF4BF600CBF01270227FBF733FD0546A3
:10324000002841D001971BE0013FBFB2C1E7B3F5B1
:10325000E13FD4D3E28C520702D4B3F5613FCED123
:1032600004F22110039102F099F803990028C6D0C6
:103270004FF4BF60FBF716FD054628B3002301930A
:10328000009604F158034246214602F017FC1BE069
:103290000B2D3FF4F7AE132D7FF40EAF142303FB79
:1032A0000743002683F820616820FBF7FBFC0546F6
:1032B00050B1B02303FB07435833009642462146E2
:1032C00003F094FB034B2B60284604B0BDE8F08765
:1032D000305C0308045E0308F8B504460D46B026CA
:1032E00010F06AFC06FB0546002386F859304FF6BD
:1032F000FF730746A6F88630A6F888302946204690
:10330000FFF79CFE90B1012286F8592004EB0513CB
:1033100005F14202194644F82200DF644FF47A6353
:10332000A1F85030BDE8F84003F00EBCF8BD000035
:103330002DE9F74F01EB8103044610F923A0BAF100
:10334000070F0D460FB24FEA81090DD0BAF1000FF9
:103350000DD1B02101FB05044FF6FF7384F859A08D
:10336000A4F88630A4F8883003B0BDE8F08F90F858
:103370001231CB40DA07F7D48144D9F8083123B9A8
:1033800003B0BDE8F04FFFF7A7BF90F92430002B42
:1033900001DDFFF72FFED9F8080103689B68984705
:1033A000019010F009FC019906464FEA0518002922
:1033B00062D1A044D8F84C30C31AB3F57A6FD3D990
:1033C0004FF0B00B0BFB05405A4658301DF0CEFDB8
:1033D0000BFB05424FF6FF73A2F88630A2F8883047
:1033E0005FFA8AF34FF47A61172B82F85850C8F8C5
:1033F0004C60A8F8501004D83F4921FA03F3DB07CA
:103400000BD4D9F8080198BBB02101FB0545002376
:10341000C9F8083185F8593002E0012382F85930A3
:1034200004EB0714B4F85030F52B61D994F852200E
:10343000B3F5FA6F02F1010284F8522094D294EDB0
:10344000157A07EE903AB5EEC07AF1EE10FA81BF28
:10345000F8EEE77ADFED296A67EEA67ADFED286AF3
:103460008CBFE7EE267AF8EE677AC4ED157A7BE733
:1034700003685B689847C7E74FF0B00A0AFB054A44
:103480009AF8C83053B10023DAE930014FF47A7268
:10349000F7F70AFD002306468AF8C830B02303FB7D
:1034A000054393F8BC206AB9012283F8BC20D9F8FF
:1034B00008010368DB6A9847124903466A1C062024
:1034C000F9F754FB04EB080304EB0511DA6CB21AAC
:1034D000A1F85020B02101FB0545DE6495F8592084
:1034E000012A9DD994F83821002A99D19E6497E742
:1034F000002284F85220A2E70042C0000AD7A33C71
:1035000048E17A3F345B030813B540F21E4204469B
:1035100000F1300101A8FBF759FD00212046FFF71B
:1035200007FFD4F8083113B1012384F8113101A841
:10353000FBF76EFD02B010BD10B40C4611461A46E2
:103540003CB9D0F8080120B103685DF8044B5B6911
:1035500018475DF8044B704710B590F900300C46E1
:103560000BB9002010BDD0F8080118B90023237052
:103570000120F7E703681B6998470028F1D1F5E7B8
:10358000174B136010B449BBB0F91030002B0DDDA0
:1035900007EE903A9FED137AF8EEE77A67EE877AB6
:1035A000C2ED007A01205DF8044B7047D0F8083175
:1035B00013B190F8591049B990F9000010B90023DF
:1035C0001360EFE7431E58425841ECE719680C6A54
:1035D0001846114623465DF8044B18470020E2E7E1
:1035E000CDCCCC3D6F12833A90F811318B420BD980
:1035F000142303FB0100B0F90200002804DDC828F1
:10360000A8BFC82080B27047C820704759B990F948
:10361000283043B990F900302BB1D0F8080110B12F
:1036200003685B6A184700207047000008B503462E
:1036300090F9220040B1D3F8080128B103689B6AD1
:10364000984780F00100C0B208BD000021B9D0F851
:10365000080108B103F0E8B90020704731B9D0F88B
:10366000080118B103681146DB6B1847002070474A
:10367000B02301FB030191F8B40010B1D1F8B030D0
:103680001360704741B990F90000122806D0A0F1EC
:103690001703584258417047002070470120704777
:1036A00070B50D4690F918107F29044613460ED0C8
:1036B0002A46C9B2BDE87040FFF73EBFD4F8080102
:1036C00050B1036829465B69BDE870401847002186
:1036D000FFF7D8FF0028F1D070BD000011F0010FF6
:1036E0002DE9F84F0446884691461E4605D11A46F4
:1036F0004946BDE8F84FFFF7D3BFD0F83031002B73
:103700004BD0D4F830A1C8F34105B4279AF8003063
:1037100007FB05A74FEAD8080637002B48D1D4F895
:10372000303183F80180D4F83011012303FA05F217
:103730000B7813430B703246494638461DF0CCFBDC
:10374000B32ED4F8303153D86A1C9A7005EB450576
:10375000D4F83031C5EB051506EB85059D80D4F80E
:103760003051AA7812B3012328789340013B984244
:103770001CD1F7F7B1FBB4F834311844A4F8340184
:10378000AA88A91D2046FFF78BFFD4F8302100231B
:103790009370D4F83021137008E040F2D621012054
:1037A0001AF0AEFDC4F830010028AAD1BDE8F88FA8
:1037B0009AF80120424509D1EB40DB07AFD53246EC
:1037C000494638461DF078FB0028EFD04FF0000B3B
:1037D0008AF802B0D4F830A19AF80000F7F77CFB21
:1037E000B4F836311844A4F836018AF800B096E7E8
:1037F0001A780F2AB3D104229A70D4F830314FF4DA
:1038000034729A80ABE700002DE9F743984690F8B0
:103810003931DDF8289004460E4673BBB02505FB10
:10382000010595F8AC7017B3EB6F1360D5F88030D5
:10383000C9F8003001AAFFF7A3FE70B1DDED017AEF
:103840009FED0F7AD9F8003067EE877AFCEEE77AC1
:1038500017EE902A9B1AC9F80030B02101FB0644EC
:1038600094F8AD303BB1D4F8A430C8F800303846F5
:1038700003B0BDE8F083034BF7E70027F7E700BF8D
:1038800000007A440000204101207047704700008A
:1038900070470000014B0B6001207047CDCC4C3EBF
:1038A00001207047012070470120704700207047B9
:1038B00070470000002070477047000006207047E6
:1038C00000487047505D03087047000010B504467B
:1038D000FBF7F0F9204610BD70B586B001AD044687
:1038E0000E461222002128461DF040FB0221032231
:1038F00064238DF804108DF806308DF80B200D230D
:103900008DF80F108DF81620042194F8DC218DF825
:1039100007308DF81010012307218DF81210D118EF
:103920008DF808208DF80D308DF8116084F8DC11C9
:103930000022E95C01330A44122BD2B2F9D160684B
:103940008DF8152003681322DB682946984706B0D6
:1039500070BD0000F0B589B004460E9D009503F0DF
:1039600045F8314A226062680023C4F8D03004F57B
:10397000F475C4F8E831C4F8EC31C4F8F03142B958
:10398000E3682A491A780320F9F7F0F8204609B0CD
:10399000F0BD274E07933068716802AA03C2CDE9D3
:1039A00005333189118002A8012630F8022B462AFE
:1039B0000CD8510908AF07EB810102F01F0251F842
:1039C0000C7C06FA02F23A4341F80C2C0133052B29
:1039D000EBD105AB03CBC4F8E80118686960A860B7
:1039E0002069012305A912308DF81430FFF77EF805
:1039F000226992F91230927C012A0ED8A26892F9BB
:103A00002420002A03DD19462046FFF765FF10F049
:103A1000D3F86E30C4F8E001B8E7E26805491278DF
:103A20000320F9F7A3F8B1E7B45D0308585D030874
:103A300040510308755D03082DE9F04186B0054645
:103A40000E4690460021142268461F461DF08EFA4D
:103A500002238DF8003064238DF802300F230722F3
:103A60008DF8033003238DF807308DF80B208DF887
:103A70001430062295F8DC318DF80C2001240A223E
:103A80008DF80D201A1985F8DC218DF804308DF899
:103A900009408DF80E808DF80F708DF81160234667
:103AA00000221DF8031001330A44142BD2B2F8D1BE
:103AB00068688DF8132003681522DB68694698470B
:103AC00006B0BDE8F081000070B5044610F074F84F
:103AD0000646D4F8E801F7F7FFF90546D4F8EC01FB
:103AE000F7F7FAF90544D4F8F001F7F7F5F9ADB2B4
:103AF00094F8E4310544ADB2AB422EDA236993F970
:103B000012209B7C012B2DD8D4F8E031B34224D273
:103B1000B4F8E6310125462B0CD8580904EB800097
:103B200003F01F01D0F8E80105FA01F1014216D0B7
:103B3000A4F8E631012394F8E6112046FFF77CFF54
:103B400094F8E431013384F8E431B4F8E6316E36A8
:103B50000133C4F8E061A4F8E631012003E0013349
:103B60009BB2D8E7002070BD38B5C368426E5A607A
:103B7000C368B0F868201A81C368B0F86A2083F877
:103B8000322090F86C3013F0010F0446C36800F047
:103B9000978003225A7090F86D30D8070CD5E368EF
:103BA00004225A7094F86D20910705D55207E368F6
:103BB0004CBF062205225A70D4F86F00D4F8731057
:103BC000E56844A3D3E90023F6F7C8FC43A3D3E98F
:103BD0000023F6F7C3FCF6F771FF6861D4F87700AD
:103BE000D4F87B10E5683BA3D3E90023F6F7B6FCD5
:103BF0003AA3D3E90023F6F7B1FCF6F75FFFA8611B
:103C0000314BD4F87F00D4F88310E5680022F6F732
:103C1000A5FCF6F753FF2861E5680FF0CDFF286695
:103C200094F88730DB071CD5E368D4F88820DA6184
:103C3000DFED267A94ED230AE56820EE270AFCF7EB
:103C400095F9204685ED080A02F002FFD4ED247AAA
:103C5000E368F1EE677AC3ED0F7AE368012283F837
:103C6000502094ED277ADFED1A6AE36827EE267A72
:103C7000BCEEC77A17EE102ADA85D4ED287AE3680D
:103C800067EEA67AFCEEE77A17EE902A1A8694ED94
:103C90002C7AD4ED2B7AE36877EE877AB6EE007A49
:103CA00067EE877AC3ED117AE368D4F8B8209A6496
:103CB000E268012382F85230E26882F8533038BD5E
:103CC000012278E7AFF3008000005940E02E654202
:103CD0000000C842F8C1631ADCA54C400000000097
:103CE000D0126341F0B5836893F92430002B85B07E
:103CF000054628DC002605F16407686803685B69EF
:103D0000984720B3686803689B69984701AAC1B2C5
:103D10003846CDE90166039603F0C6F8012804464B
:103D2000EBD1019B03F00602062AE6D103F44072B0
:103D3000B2F5407FE1D1DB04DFD52846FFF714FF61
:103D4000204605B0F0BDFFF7BFFE0028D2D100200D
:103D5000F7E700000320704700487047F85D03084C
:103D600090F8623013B1002280F862201846704744
:103D7000014B0B6001207047AE47E13D70470000EA
:103D80002DE9F0412DED028B04460D4686B0D1F8A9
:103D900003109FED548A342202F0E6FEE368B5F882
:103DA00001201A81E368D5F803205A60E368EA79B4
:103DB0005A70E3682A7A83F8322002AF0023D5F8DC
:103DC0001120D5F8151000933846D5F819300FF0AA
:103DD000D9FF97E80F00E6680C3686E80F00E36825
:103DE000B5F80F20DA85E3684FF6FF771F86E368A2
:103DF000012683F85060D5F82130D5F81D2007EE54
:103E0000103AD5F8253006EE902A07EE903AB8EE33
:103E1000C77AF8EEE77AF8EEE66AE36827EE087A02
:103E200067EE887A66EE886A83ED0E7AC3ED0D6AD6
:103E3000C3ED0F7AE168204602F036FEE36883F8AE
:103E40005160E36883F85260E36883F85360E36885
:103E500083F85060B5F80920E36807EE902AF8EE81
:103E6000E77A67EE887AC3ED117AB5F80B20E3683C
:103E700007EE902AF8EEE77A67EE887AC3ED127AB9
:103E8000B5F80D20E36807EE902AF8EEE77A67EEC2
:103E9000887AC3ED107AD4F80C800FF08DFEC8F844
:103EA0006000B5F82B30BB4210D007EE903AB8EE68
:103EB000E70AE76820EE080AFCF758F887ED090AD8
:103EC000E36883F85460E3681A6E9A62EB79003B0A
:103ED00018BF012384F8623006B0BDEC028BBDE848
:103EE000F08100BF0AD7233C10B50446FAF7E2FE82
:103EF000204610BD0620704700487047485E030802
:103F00007047000010B50446FAF7D4FE204610BDF5
:103F100037B5069D0095044602F068FD114B2360FD
:103F20000023C4E91B3384F8683084F87430AA2372
:103F300084F8793141F24423A4F87A31A36893F9E3
:103F400024305BB16068084903680E22DB6898473B
:103F50006068064903682222DB689847204603B060
:103F600030BD00BFE45E0308505E03085F5E0308D7
:103F700070B5B0F8812190F87C31B0F87D51D0F85F
:103F800089111A44044602F0EFFD632D00F0BC8055
:103F9000AE2D00F0E5802A2D40F09F80E368B4F854
:103FA00087211A81E368D4F889215A60E5680FF007
:103FB00003FE2866D4F87D00D4F88110E66879A362
:103FC000D3E90023F6F7CAFAF6F778FD7061D4F862
:103FD0008500D4F88910E66872A3D3E90023F6F7C8
:103FE000BDFAF6F76BFDB061E368012683F85C600B
:103FF000D4F89530E26807EE903AF1EE677AC2EDB8
:10400000167A654BD4F88D00D4F891100022F6F79B
:10401000A5FAF6F753FDE1680246204602F02EFEAF
:10402000E36894F8B62083F83220D4F89D3007EE88
:10403000103AD4F8A13007EE903A67EEA77AE36819
:10404000E7EE077AB1EEE77A83ED117AE368D4F808
:10405000A5209A64E3689FED517A83F85260E36883
:1040600083F85360D4F8AD20E36807EE902A67EE3A
:10407000877AFCEEE77AC3ED207AE36894F8B620FD
:1040800083F88420D4F87530E268DBBBD4F879304B
:10409000222B0FD81F2B33D8102B16D00F2B07D95C
:1040A000122B03D8102B03D004230FE0142BFBD0CA
:1040B00001230BE0322B02D003D8302BF8D106239A
:1040C00004E0443B012BEFD9F2E70323537094F84B
:1040D000623043F0010384F8623094F8623013F0E8
:1040E00001000CD09A07C3F3400008D5E268616E66
:1040F000526891424ED123F0030384F8623070BDC0
:104100000523E3E75670E2E7D4F88910D4F8850078
:10411000E668F6F71BFDF061D4F89110D4F88D0035
:10412000E668F6F713FD3062204602F091FCD4F801
:104130009500D4F89910E668F6F708FD07EE900AA6
:10414000F1EE677AC6ED0F7AE368012283F850201A
:10415000D4F88931636694F8623043F00203BAE719
:10416000D4F87D20DFED0E6AE36807EE102A27EE13
:10417000267ABCEEC77A17EE102ADA85D4F88120A9
:10418000E36807EE902A67EEA67AFCEEE77A17EE70
:10419000902A1A860020B2E70000594000007A44B5
:1041A0000000C84200000000D012634110B590F832
:1041B0007430013B0446082B06D8DFE803F01019E1
:1041C0001D26374C50586000AA2904BF012380F8EF
:1041D0007430002380F8953184F8963104E0442946
:1041E00004D1022384F87430002010BD0023F9E7C5
:1041F0001229FBD10323F5E7042380F8743080F8FB
:10420000953180F87C110023E6E7B0F895311B2B3F
:10421000ECD8C218013382F879119AB2A0F895311E
:1042200090F87C319342DFD80523DBE7B0F8953175
:10423000FF2BDBD890F87C011A1A2244013382F854
:1042400075109AB2A4F89531B4F8813103449A42BA
:10425000CADB0623C6E7C0F875110723C2E7D0F80A
:10426000753103EB0121C0F875110823BAE7D0F8C6
:10427000753103EB0141C0F875110923B2E7D0F89D
:10428000753103EB0161C0F87511002094F87C21B1
:1042900084F8740004F2791110F0B2F8B4F88121B6
:1042A00004F1750110F0ACF8D4F87531834204D1F3
:1042B0002046BDE81040FFF75BBE236F0133236744
:1042C00092E700007FB5836893F924300446F3B188
:1042D0000FF072FC94F86830032B054617D8E26E95
:1042E000824214D2164A666852F823100191084699
:1042F000F7F75AF833680199DB6802463046984769
:1043000094F86830C8350133E56684F868304FF4B6
:1043100000560025606803680DF10F01DB699847BE
:1043200050B19DF80F102046FFF740FF013E284393
:10433000B6B2C5B2002EEDD1284604B070BD00BFA4
:10434000CC5E030810B50023044643608360C3605D
:104350000249FEF76BF8204610BD00BF285F030836
:104360000620704700487047985F0308014B0B60B8
:10437000012070470AD7A33DD0F880300B600120A0
:1043800070470000836893F9243023B1806E831F47
:10439000584258417047012070470000D0F88030E3
:1043A00013F4746F0CBF01200020704710B5044651
:1043B000C06E19F0A9FF204610BD000010B50446DC
:1043C000FFF7F4FF2046FAF775FC204610BD000009
:1043D0008268C36F92F92220022A03F4207304D06A
:1043E000A3F52073584258417047B3F5207F08D099
:1043F000064B1B68DB6A93F89C3023B990F8840065
:104400007047012070470020704700BFD81000207F
:104410001FB5836893F924308BB1836E062B0ED0C1
:10442000C26804214FF0030C1278CDE9011C90F80A
:1044300062100091013203490620F8F797FB05B09E
:104440005DF804FB9C5F0308C3681B7813B983689D
:10445000187870470020704737B5069D00950446D0
:1044600002F0C4FA0F4B23600F4B63670023A3676E
:1044700084F886300FF0A0FBE3682067012283F800
:104480008520A368DB8C9B0704D42046FFF7DCFF64
:104490001A2803D1E368012283F82C20204603B0B8
:1044A00030BD00BFC8620308D05F03082DE9F341A7
:1044B000B0F88C3040F6BC72C3F30C039342044650
:1044C00000F0C8810FD840F6A77293423BD040F667
:1044D000AE72934200F04B8140F6A172934200F01D
:1044E000378100201FE141F21472934200F0628193
:1044F00041F233729342F4D1FFF7A6FF1A28F0D1AC
:104500002046B4F88E20D4F8901002F02DFB94F8D9
:104510009700E36810F08F0040F08181D4F8982074
:104520009FEDC67A07EE902AF4EE477AF1EE10FA84
:1045300000F07581B1EEE77A012283ED137AE3682A
:1045400083F85520EFE0B0F894304FF6FF7299B23F
:10455000914205D0C2681381C368D0F890205A6098
:10456000B4F88E20D4F89010204602F0FDFAE568E9
:104570000FF022FB2866D4F8B430DFEDB17A07EEF5
:10458000103AB4EEE77AF1EE10FA3BDDE2685363DD
:10459000E368D4F8B8209A63D4F8BC30E26807EE38
:1045A000903AF1EE677AC2ED0F7AE368012583F85D
:1045B0005050E168204602F077FAB4F8D630E2684D
:1045C000DFEDA06A0A214B43C2F88030B4F8E22044
:1045D000E36807EE102AB8EE477A27EE267A83EDD5
:1045E000117AB4F8E420E36807EE902AF8EE677ACF
:1045F00067EEA67AC3ED127AE36883F85250E36857
:1046000083F85350D4F89860D4F89C7085A3D3E90C
:10461000002330463946F6F731FA00285FD083A3ED
:10462000D3E9002330463946F5F798FF81A3D3E953
:104630000023F5F793FFF6F741FAE5686861D4F8CF
:10464000A000D4F8A410E56878A3D3E90023F5F717
:1046500085FF78A3D3E90023F5F780FFF6F72EFA5C
:10466000A861D4F8B020DFED757AE36807EE102A70
:10467000B4EE677AF1EE10FA0CBF0122002283F843
:104680005C20D4F80C80D4F8A86098F85C30D4F89A
:10469000AC7093B1D4F8B0502846F5F707FF024646
:1046A0000B4630463946F5F7A1FD07EE905AF1EE7C
:1046B000677A06460F46C8ED167A39463046F6F751
:1046C00045FADFED617AE16807EE100A67EE277AB6
:1046D0002046FDEEE77A17EE902A02F0CFFA94F822
:1046E000D230E268FF2B82F8323002BFE36800224A
:1046F00083F8322094F8963003F00F03082B09D882
:10470000DFE803F0051417141A1D171A1D00E368DB
:1047100001225A7094F8963013F0400F4FF00100C8
:1047200010D0E368587002B0BDE8F081E36803225E
:10473000EFE7E3680422ECE7E3680622E9E7E368D1
:104740000522E6E71A06EED5E36802225A70EAE788
:10475000B0F88E20D0F8901002F006FAE368B4F8B2
:104760009C20DA85E368B4F89E201A86B9E6B0F892
:104770008E20D0F8901002F0F7F9D4F89C30D4F8DD
:10478000A010E367D4F8803083EA010212F4746F5A
:104790000BD0E268127801F47461009103F4746341
:1047A0002A4901320620F8F7E1F9D4F8A030C4F81C
:1047B000803096E6B0F88E20D0F8901002F0D4F950
:1047C000D4F8983007EE103AD4F89C3006EE903AC0
:1047D000D4F8A03007EE903AF4EE676AF1EE10FAE2
:1047E000C8BFF0EE667AB4EE677AF1EE10FAC8BF91
:1047F000F0EE477A9FED167AE368F4EEC77AF1EEB1
:1048000010FA08DBB1EEE77A012283F85120E36861
:1048100083ED107A65E6002083F8510083E70022DB
:10482000DA645EE600000000006A08C1F8C1631A9D
:10483000DCA54C4000000000D0126341FFE65BAFF6
:10484000005043C80AD7A33B0000C842E05F0308FA
:1048500000000034B0F88E20D0F8901002F084F9F7
:1048600094F89600E36870B983F88400E368C3F8AD
:104870008000E368C3F88C00E368C3F88800E3684D
:10488000C3F890004FE794F8982083F88420B4F898
:10489000C5304FF6FF7293421CBF0A225343E268B1
:1048A00008BF0023C2F88030D4F89C60D4F8A07010
:1048B00031A3D3E9002330463946F6F7B7F800288C
:1048C00041D12DA3D3E90023D4F8A400D4F8A81033
:1048D000F6F7ACF8B8BB28A3D3E90023D4F8AC00B2
:1048E000D4F8B010F6F7A2F868BBB4F8C0204FF6C1
:1048F000FF739A4227D01F4BD4F80C800022304619
:104900003946F5F72BFEF6F7D9F8C8F88C00D4F83D
:10491000A400D4F8A810174BE6680022F5F71EFE95
:10492000F6F7CCF8C6F8880010A3D3E90023D4F832
:10493000AC00D4F8B010E668F5F710FEF6F7BEF854
:10494000C6F89000CDE5A368DB8C9B077FF5C9AD69
:10495000E3680020C3F88C00E368C3F88800E368CC
:10496000C3F89000E36883F85400DCE60000000020
:1049700000408FC000408F40BBBDD7D9DF7CEBBD6E
:104980002DE9F84F90F88630013B04460D46082B80
:1049900006D8DFE803F0404B4F575B63677FB400F6
:1049A000242908D1012380F886300023A0F8903113
:1049B0000020BDE8F88F90F89731DFF800925E1C78
:1049C000F6B203444FB2032E80F89761B24683F8E3
:1049D00092714FF00608A8BF4FF0030A00F5C97B9B
:1049E00059F8040B524659461CF084FF78B9042E3E
:1049F00006D1303F092FDBD9002384F89731D7E760
:104A0000D6D93E2DF8D1012384F89831F4E7B8F1D6
:104A10000108E5D1F0E7402903D1022384F886306C
:104A2000C6E7522940F09D800923F7E7A0F88A10D5
:104A30000323F3E7B0F88A1001EB0525A0F88A50AC
:104A40000423EBE7A0F88C100523E7E7B0F88C10FF
:104A500001EB0525A0F88C500623DFE7A0F88E10A7
:104A60000723DBE7B0F88E1001EB0525ADB2AB07ED
:104A7000A0F88E50A5F108050CBF08230023F82DDF
:104A800080F8863094D9002380F88630A36F0133F4
:104A9000A3678DE7B0F89031FF2B98BFC21803F1E0
:104AA000010398BF82F89010B0F88E209BB2083AAC
:104AB0009342A0F89031FFF67BAFB3F5807F50D8DA
:104AC000002202218C300FF0ADFC0221024604F1DD
:104AD0008E000FF0A7FCB4F88E100246083904F1DE
:104AE00090000FF09FFC002384F88630B4F88A30E1
:104AF0008342CBD12046BDE8F84FFFF7D7BCB0F8D2
:104B00009021FE2A2DD88318013292B20A2983F807
:104B10009010A0F890217FF44BAF8318002183F808
:104B2000901090F890303A2B1BD1C66ECEB100F1A8
:104B30009201053A30461CF0DDFE054688B9304644
:104B400019F0E2FBA36EE566062B07D8DFE803F059
:104B5000040B0F1D2B0D2D000123A3660FF02CF865
:104B6000206700235AE70523F7E70223F5E794F8C7
:104B700062300133DBB2032B84F86230EED90323B9
:104B8000A366002384F86230E8E794F86230A268F4
:104B90000133DBB284F8623092F920200AB1022B93
:104BA000DCD90423D9E70623D7E706F0FBFC4FF452
:104BB000CE724FF4801106F0E1FCCFE79862030853
:104BC0004068024903681122DB6818470C6003083B
:104BD00038B5836893F92230054653B3C06F10F49B
:104BE000007414D1EB6814491A7806200132F7F7E3
:104BF000BDFFEB6811491A7806200132F7F7B6FFBE
:104C00002846FFF7DDFF85F88440002038BDC30546
:104C100007D5EB680A491A7801320620F7F7A6FF94
:104C2000F3E710F0800404D1EB6806491A780132EA
:104C3000F3E70120EAE700BF2060030840600308B3
:104C4000616003087A60030810B50446054907202F
:104C5000F7F78CFF606804490368BDE81040DB6823
:104C600013221847A0600308B46003082DE9F0433D
:104C700004464068036887B05B699847002506468C
:104C80002F46B5420BD0606803689B699847C1B254
:104C90002046FFF775FE0743FFB20135F1E70EF03E
:104CA0008BFFA36893F924200546E2B1A26E062A81
:104CB00000F0FC80616E814215D2216F01F5FA612E
:104CC000814221D2606FF6F76FFB06466068036889
:104CD0009B6A9847B04206D36068616F03683246AA
:104CE000DB6898472567E268906A2D1AB5F5967FCC
:104CF00082BF002382F85430E268384688BF82F8C9
:104D0000553007B0BDE8F08394F898110029EAD037
:104D1000E16E09BB052A1FD8DFE802F003349AA030
:104D2000B7452369606893F91220036805921B6CEC
:104D300098477049704B059A012808BF0B4604F14B
:104D40006C066E49009330464FF461330EF080F9E3
:104D5000013001D10023E366E06E0028C3D0F6F7EE
:104D600023FB0646606803689B6A9847B042BAD343
:104D70006068E16E03683246DB689847002384F878
:104D80009831B0E72046FFF75FFB5D4B5D4A5E4917
:104D90001A2818BF1A46236904F16C0093F91230DF
:104DA00000920122D2E72369597893F9016011F04A
:104DB0006F0FD1D0524B554A16F0010F08BF1A465B
:104DC00016F0020F04F16C0006D0DFF870C1504BF2
:104DD00011F0010F08BF634616F0040F2DD0DFF865
:104DE00060E1DFF860C111F0030F08BFF44616F070
:104DF000080F25D0DFF85081DFF850E111F0070FE0
:104E000008BFC64616F0200F1DD0DFF84491DFF82A
:104E1000448111F00F0F18BFC846760616D53D4ED7
:104E200011F02F0F3C4918BF3146CDE90281CDE981
:104E300000CE3A490EF00CF98AE7DFF8C4C0D6E795
:104E4000DFF8BCE0DEE7DFF8B880E6E72C49ECE706
:104E500094F86220324B53F8222009E093F9203075
:104E6000012B0BD0022B0DD0002B7FF475AF2D4AF8
:104E70002D4904F16C000EF0EBF869E794F862201C
:104E80002A4BE8E70623A36666E72046FFF7DCFA2D
:104E90001949274A1A2818BF0A46264904F16C0006
:104EA0000EF0D6F800287FF455AF55E793F922307D
:104EB000022B7FF418AF204B1B68DB6A93F89C3001
:104EC0001BB1012384F884300DE794F88430002B63
:104ED0003FF409AFE36F9B057FF505AF636E834237
:104EE000BFF401AF2046FFF7AFFE05F57A736366A6
:104EF000F9E600BFCD600308C86003081F6103081E
:104F0000EE570308D5600308426103083B520308CB
:104F1000D9610308096103080A6103089D61030858
:104F2000B0620308B0610308C06103088C62030823
:104F300012610308BB610308D8100020DA6103087E
:104F4000F3600308F2600308FC600308FB600308D9
:104F5000036103080461030806207047836893F91E
:104F600024302BB1D0F8BC05B0FA80F0400970476E
:104F700001207047D0F8BC350B600120704700005D
:104F8000004870470C63030890F8C035822B08D89E
:104F90001A0611D4033B012B0ED9084B0B600120DC
:104FA0007047FF2BF9D1054B0B60836893F9240000
:104FB000B0FA80F040097047014BEFE7AE47613E21
:104FC0008FC2F53D002070477047000001207047F8
:104FD00010B5054B03600446D0F8F40508B1F9F7A5
:104FE00069FE204610BD00BF0466030810B50446E4
:104FF000FFF7EEFF2046F9F75DFE204610BD0000EA
:1050000013B5D0F8BC150023012202FA03F40C42B8
:105010000CD0C268127800910649013251F8233051
:1050200005490620F7F7A2FD02B010BD0133162B8B
:10503000EBD1F9E74C65030814630308C1F302716F
:105040000139C9B204299ABF014B585C002070474E
:105050004465030830B5D0F8DC357BB190F8E055F5
:105060000020C2B2954209D953F830208A4200F19B
:10507000010401D140B230BD2046F2E74FF0FF30CD
:10508000F9E7000030B5039C0A44914209D011F8B9
:10509000015B18782844C0B2187025782844207025
:1050A000F3E730BD2DE9F041044640681D46036832
:1050B00086B09B6ABDF8306088461746984706F16F
:1050C000080398424FF000003AD3B5238DF8103012
:1050D0008DF8137062230DF10F078DF80E008DF817
:1050E0000F008DF8113004220DF10E030DF11201A5
:1050F000204600978DF81280ADF81460FFF7C2FFCC
:105100003246294620460097FFF7BCFF60680368D7
:105110000622DB6804A99847606803683246DB68AA
:1051200029469847606803680122DB680DF10E018B
:105130009847606803680122DB6839469847012078
:1051400006B0BDE8F081000013B50446406803686E
:105150009B6A9847072806D9002300931A46062120
:105160002046FFF79FFF02B010BD00001FB590F86A
:105170009734052B05D9FFF7E7FF002005B05DF850
:1051800004FB02238DF80C108DF80D2000930122F2
:1051900003AB0621FFF786FFF0E70000F0B50446F9
:1051A00040681D46036885B09B6A0F4616469847BF
:1051B0000A280FD903230093012203AB06212046BE
:1051C0008DF80C708DF80D608DF80E50FFF76AFFAA
:1051D00005B0F0BD0020FBE790F8D2350133DBB21B
:1051E00080F8D2352BB990F8752490F87A14FFF72F
:1051F000D5BF7047022938B50546184641D00A295F
:1052000039D001291ED1122A1AD8012A1AD9931E7F
:10521000102B17D8DFE803F0171D0916233F1616C9
:105220001616161616161616290001232024834278
:105230003BD1D5F8BC3523EA0403C5F8BC3501E001
:10524000202A2CD038BD95F8D64584F001030224DD
:10525000EDE795F8D64584F001030424E7E795F8D7
:10526000D64584F001030824E1E795F8D64584F09B
:1052700001031024DBE7092A15D00B2AE2D1802490
:105280000FE0102A01D0152ADCD1AB684FF48074EE
:1052900093F82230CBE701234FF40054C7E74FF4D3
:1052A00000440523C3E74024FBE72846FFF776FFC9
:1052B000D5F8BC352343C5F8BC35012385F8D43572
:1052C000C0E700002DE9F04385B002AFC0F8E83533
:1052D00097F8283080F8EC3590F8F03580F8E02524
:1052E000541C83F001035B42A40080F8ED350026D6
:1052F000E31DC0F8DC15C0F8E4650546914640683A
:105300006A46DB08A2EBC3039D46026802AB926AC1
:105310007B60013C8846A4B2904704F1090292B236
:10532000904218D37B680296414603AA08EBC9094C
:10533000494504D051F8080B42F8040BF8E7013452
:10534000A4B200948B2206212846FFF7ABFE0C374F
:10535000BD46BDE8F0833046F9E7000013B50C23E5
:105360000446009309220B4B0621FFF79BFE0EF02B
:1053700023FC94F88834C4F88404013384F8883416
:10538000E36805491A780620013202B0BDE81040F2
:10539000F7F7ECBB486603083C63030810B500232D
:1053A00008248278082A0ED8DFE802F00B051217CD
:1053B000202B37474D00622902D10223837002E07F
:1053C0008370B52901D0002042E083780133F5E7EE
:1053D00003238370C1700171F5E704238370C378E0
:1053E00019440379C9B2C1701944F4E705238370E5
:1053F000C378027901700B44DBB2C37013440371AC
:10540000E1E706238370C37819440379C9B2C170F8
:105410001944002301714370D5E7C3780278194419
:105420000379C9B2C1701944437801710133DBB209
:105430009A424370C7D10723C0E7C27884708A427A
:10544000C1D08370ADE7027983708A42A9D101206F
:1054500010BD000007B50023009304220A21FFF7C6
:1054600021FE03B05DF804FB1FB5C368044619783C
:105470008068FEF7B9F80123ADF80A300621002351
:10548000ADF80800ADF80C30009102AB08222046C0
:10549000FFF708FE04B010BDB0F87624083201F022
:1054A00063BB00002DE9F74F0569D0F8BC35044611
:1054B00095F9010038B923F40023C4F8BC356B78A2
:1054C00084F8D7352EE013F4002000F08880D4F85B
:1054D000F435FBB128460DF1070110F8017F07F004
:1054E000EF0747F021078DF80770FDF717FB4FF026
:1054F000000C60466646312210214FF028080CF15E
:10550000FF3527FA0CF3052D64D8DFE805F00E2CE3
:105510006E6363A20821152018F0F2FEC4F8F405AA
:105520000028D7D103B0BDE8F08FD4F8F4954FF040
:10553000200A09EBC00509F830A003F001036E70E2
:10554000AA70E9706B6000F1010ED4F8F495023096
:105550005FFA8EFEC0B209EBCE054FF0050A09F8DE
:105560003EA06E7033E0D4F8F4E54FF021090EEB65
:10557000C0050EF8309003F001036E70AA70E97058
:105580006B60D4F8F49500F1010E5FFA8EFE09EB22
:10559000CE054FF0070A09F83EA06E70AA70E970B8
:1055A0006B6000F1020ED4F8F49594F8C1A55FFA8F
:1055B0008EFE4FEACE050330C0B24D44BAF1000F63
:1055C00010D14FF00A0B09F83EB085F801A0AA707F
:1055D000E9706B600CF1010CBCF1070F8FD12369EE
:1055E0005B786DE74FF0090AB9E7D4F8F4E54FF0BE
:1055F00022090EEBC0050EF8309003F001036E7027
:10560000AA70E9706B60D4F8F49500F1010E5FFAAE
:105610008EFE09EBCE054FF00D0A09F83EA06E7024
:10562000AA70E9706B6000F1020ED4F8F49594F85A
:10563000C1A55FFA8EFE4FEACE050330C0B24D44DD
:10564000BAF1000F02D14FF00E0BBCE709F83E8013
:1056500087E7D4F8F4E54FF025090EEBC0050EF806
:10566000309003F001036E70AA70E9706B60D4F89B
:10567000F4A500F101095FFA89F90AEBC90E4FF0B0
:10568000180B0AF839B08EF801608EF802208EF8F7
:105690000310CEF8043094F8C195851CEDB2B9F131
:1056A000000F12D1D4F8F4A50AEBC50E03304FF069
:1056B0001A0B0AF835B0C0B28EF801908EF80220AD
:1056C0008EF80310CEF8043084E7284682E7000005
:1056D00090F8C00500F0FD00A0F180035842584149
:1056E000704700002DE9F04F85B002AF06460C462A
:1056F00092469B46FFF7ECFF20B900200C37BD46D1
:10570000BDE8F08F3046FFF799FC0023C7E900336E
:10571000804600F10F03706823F00703ADEB030D23
:1057200003689B6A98471FFA88F505F110039BB23E
:1057300098420DF10809E0D301233B707C6087F8A3
:1057400001B03C4603CC08350290039142465146D5
:1057500004A8ADB21BF0C0FB00954B468A2206217F
:105760003046FFF79FFCC9E77FB505460E46FFF7B9
:10577000AFFF98B10024CDE90244686803689B6AD2
:1057800098470F280CD9082300938B226B440621DD
:105790002846ADF808400396FFF784FC04B070BDBE
:1057A0002046FBE72DE9F04F87B002AF81460C465B
:1057B00090461D46FFF78CFF20B900201437BD46E8
:1057C000BDE8F08F0023C7E90233D9F80400531C69
:1057D0006A46DE00A2EBC3039D4603689B6A9847B6
:1057E0000836B0420DF1080AE7D301233B727D72FF
:1057F000BB68029303AE04EBC8084FF0040B4445AA
:1058000015D02346484653F8042B7B601146FFF71A
:1058100015FC46F8042B7B680546024619463046BF
:105820002E4404351BF058FBAB440834E7E71FFA5D
:105830008BF2009253468A2206214846FFF732FC3B
:10584000BCE7000013B5836893F924300446002BAD
:105850005BD0406803689B6A98470D2855D9D4F8F7
:10586000BC351A0706D594F8D6251AB123F00803DB
:10587000C4F8BC3594F896345A1C84F89624192B35
:1058800000F21081DFE813F01A0063006B002200C1
:10589000690067006D002000280035004A004F00B5
:1058A00041009D006F007100740076008200890045
:1058B0004100A700AC00CA00ED00F9000722012159
:1058C0002046FFF753FC12E02022F8E7204602B002
:1058D000BDE81040FFF738BC94F8C035FF2B14D159
:1058E00000230093302201212046FFF7DBFB60B943
:1058F00089E0A36893F92030022B08D0002300939D
:10590000162206212046FFF7CDFB02B010BDD4F8C9
:10591000BC3523F48053C4F8BC35F6E7002300936C
:1059200024220621E0E72046FFF7D2FE034658B1C5
:10593000236994F8D72593F901309A42E5D0D4F839
:10594000BC3543F40023E6E700903E22E9E700235C
:1059500000930822E5E70222B1E70322AFE706221F
:10596000ADE71222ABE70422A9E709220A21A7E743
:105970000B22FBE7A36893F9223023B9D4F8BC3596
:1059800023F48073C7E71022022199E7A36893F9F3
:105990002230002BF2D01522F6E794F898345BB948
:1059A000414B1B68DB6A93F89C302BB9204602B050
:1059B000BDE81040FFF74EBDD4F8BC3523F40073AA
:1059C000A9E72046FFF784FE00289ED037492046ED
:1059D000FFF7CAFE8BE7D4F8BC3523F480239AE79F
:1059E00094F8C03503F0FD03802B8ED12046FFF7DD
:1059F00059FD0246002888D0D4F8F4150323204628
:105A0000FFF7D0FE28B994F89634013B84F8963419
:105A10007BE70EF0D1F8C4F8900476E794F8C0352F
:105A200003F0FD03802B7FF470AF0EF0C5F8D4F8BF
:105A30009034C01AB0F5FA7FE5D30023C4F890344F
:105A40002046FFF72FFD024600283FF45EAF0323F8
:105A5000D4F8F41500934FF400232046FFF732FCEE
:105A600045E794F8C035822B7FF44FAF03230093B2
:105A70000F494FF480130822EFE794F8F135002B1B
:105A80003FF443AFA368DB8C13F0200F4FF0030308
:105A9000009314BF074908494FF4001314BF0222B2
:105AA0000122DAE70023B1E7D8100020010003202B
:105AB000A4650308EC650308E465030837B5069D93
:105AC0000095044600F092FF124B23604FF47F4391
:105AD000A4F8963441F6FF73C4F8BC35FF2384F86C
:105AE000C0359DF81C3084F8D035E168A0680123EA
:105AF00084F8D33584F8D53584F8D835002309786F
:105B00001A46FDF743FA2046FFF79CFE204603B0F5
:105B100030BD00BF046603082DE9F04F2DED028B68
:105B200090F87A14052997B0044640F0A08090F8C8
:105B30007554012D45D190F86230062B03D00A2B05
:105B40002FD000251BE090F86330242B1DD008D8FF
:105B5000092B0FD0162BF4D1D4F8BC3523F4805385
:105B600017E0312B18D03E2BEBD1D4F8BC3523F401
:105B700000630EE080F87B54002580F8D455284659
:105B800017B0BDEC028BBDE8F08FD0F8BC3523F424
:105B90008063C4F8BC35D4E7D0F8BC3523F4804327
:105BA000F7E790F86330092B06D00B2BC9D1D0F85A
:105BB000BC3523F08003ECE7D0F8BC3523F040037C
:105BC000E7E7002DBDD190F86230062BB9D190F8EF
:105BD00063308A2B34D08B2BB3D1D0F8DC65002E08
:105BE000AFD090F9ED2590F8E005571C4FF0010378
:105BF0000DD184F8ED5584F8F03594F9ED358342F4
:105C00009FDA56F833102046FFF7AEFD99E7D4F837
:105C1000E45503FA02F183402943013B9942C4F859
:105C2000E41501D0824207DBD4F8BC35D4F8E8157E
:105C300023EA0103C4F8BC35013284F8ED25DCE722
:105C4000D0F8DC35002B3FF47CAF90F9EE25C44949
:105C500053F832301A0C12048A427FF472AFC268D1
:105C6000C049127804200132F6F780FF87E7062941
:105C70000ED190F87524162A00F05B817FD8012A96
:105C800000F08081082A00F09A81002A00F09281B9
:105C900094F87A240A2A40F0898294F8758408F0EE
:105CA000FD03092B3FF44DAFB8F1040F40F08B8298
:105CB000012304F2B74684F8983404F18001304699
:105CC00004F299471BF02AFE04F18A051E2204F112
:105CD000620138461BF022FE4346A34AF0212846C3
:105CE0001BF008F904F2B158002800F02482011DCD
:105CF000082240461BF012FE9C4BE2689C49CDE90D
:105D0000016712780132009206204246F6F72EFF14
:105D10009849082230461BF0EDFD002840F018821B
:105D200095490A2238461BF0E5FDE8B994F8C035DC
:105D30009249802B1EBFD4F8BC3543F48033C4F89D
:105D4000BC35802384F8C035D4F8BC3523F4006317
:105D500043F40023C4F8BC354046F5F71BFB00288C
:105D600040F0EB8184F8C10585490A2238461BF0D2
:105D7000C1FD10B9812384F8C0350127E9E13E2A2D
:105D800041D08B2A00F03281242A81D100238268FD
:105D9000A0F8623092F914305D1C08D090F86410BD
:105DA00099421EBF80F864300123A0F8623092F956
:105DB0002130B4F8625013F1640F1BD094F96E20B7
:105DC0009A4217D045F0020584F86E30A4F862506C
:105DD000242204F16203009206212046FFF762F9B3
:105DE000D4F8BC3543F48063C4F8BC35012384F88F
:105DF000D435A6E6002DEBD1D4F8BC3523F480636E
:105E0000C4F8BC35BBE6D0F8108098F90160002ECC
:105E10003FF4ABAEFFF75CFC054600287FF4A5AE6F
:105E200004F1620207AF04F19A091346BE461068F6
:105E30005168BC46ACE8030008324A456746F6D1D3
:105E40001068CCF800000022114646FA02F0C007A4
:105E500003D5012A1CBF0131C9B20132072AF4D18E
:105E60004A0094F865600592002722464FF0080A20
:105E7000BE423FDD92F866C098F9010040FA0CF08E
:105E800010F001004FEAC7012AD0BCF1010F1DD06C
:105E900094F863900598A9F1030B9BFBF0F094F83C
:105EA000C0B5C0B2BBF1040F82F8670002D8BCF1E4
:105EB000020F12D082F868902144D1F86A0040F0B5
:105EC0000100C1F86A0001370832D1E74FF0030042
:105ED00082F867C082F86800EEE782F868A0EBE716
:105EE000214482F8670082F86800D1F86A0020F047
:105EF0000100E6E719463C22704605931AF0DCFFE4
:105F0000059B88B1F600043600963E220621204605
:105F1000FFF7C8F8D4F8BC3543F40063C4F8BC35C7
:105F2000012384F8D4352AE6D4F8BC3523F4006381
:105F300066E7836893F92050022D3FF40DAE90F888
:105F40006230AB423FF408AE034603F8625F0825B7
:105F50000095FFF7A7F8D4F8BC3543F4805343E726
:105F6000000031105C63030884630308E0B0030899
:105F700089630308A5630308AE630308B9630308D4
:105F8000C9630308B0F87634082B10D190F8973421
:105F9000052B02D9FFF7D8F8D3E5034493F8643012
:105FA00094F8632094F86210FFF724F9C9E590F89B
:105FB0006430F5E790F8623080F89734C1E5036902
:105FC000B0F86220B3F902309A4207D1436E012B38
:105FD00004D1D0F8BC3523F00103DAE52046FFF701
:105FE00043FAD4F8BC3543F00103FDE6B0F876344B
:105FF000DFF838A4043BDBB200F16607042B7FF620
:1060000047AEB846043B58F8049BDBB2D145059334
:1060100015D13B79002B72D04FF000038DF81C3066
:1060200007AA072351462046FFF75CFB012384F8AB
:10603000D435D4F8BC3543F48033C4F8BC35494674
:106040002046FFF707F805462046FEF7F7FF002D2C
:1060500006464BDBD4F8DC252BB202EBC303059AD2
:10606000824203F1040B0DD3012804D15B683A7915
:106070005340D90706D43246414658461AF01CFF11
:10608000002841D094F8EC355A4649462046FFF79F
:1060900029FBD4F8BC35D4F8E82584F8EE55134331
:1060A000C4F8BC350122D4F8E43584F8D42502FACA
:1060B00005F123EA0103C4F8E43594F9ED35002B2A
:1060C00014DB94F8E0158B4210DAD4F8DC2552F892
:1060D000330048450AD101335BB2994284F8ED356B
:1060E00004DD52F833102046FFF73EFB002E3FF44C
:1060F00028AD059B9B1BDBB208EB06077EE7D4F8B7
:10610000BC3523F4803398E794F8E025D4F8E4050F
:10611000012303FA05F59340013B05439D4204BF6B
:10612000D4F8BC35D4F8E825C4F8E45504BF93434B
:10613000C4F8BC35C1E7B84BDFE5B8494046F5F7D0
:1061400029F900287FF410AE012384F8C1350BE64D
:106150000027B349082230461BF0CCFB10BB82233A
:1061600084F8C035D4F8BC3523F4006343F48013BD
:10617000C4F8BC35012384F8F035AA4A0423F02181
:1061800028461AF0B7FE00283FF4DBAC012384F860
:10619000F135A5490620F6F7E9FCD4F8BC3543F4FF
:1061A0000013F6E4002F3FF4CCACE6E7022A0ED150
:1061B00094F87534102B04D1A36893F9223013B1ED
:1061C000BFE4152BF8D02046FFF706F8B9E4012A02
:1061D000F9D194F87524122A17D8012A1BD9931ED5
:1061E000102B18D8DFE813F02600AA00CE00170005
:1061F000DF002F0117001700170017001700170006
:1062000017001700170017003702202A00F0188225
:10621000302A00F08B8294F8D2550135EDB284F823
:10622000D255002D7FF48DAC2B4601212046FEF780
:10623000B5FFA4E494F8D63533B1D4F8BC3543F0B7
:106240000203C4F8BC3552E0D4F862109FED788A9E
:106250002046FFF721F9D4F86230C4F88034E368AF
:10626000D4F866209A61E368D4F86A205A61E3683A
:10627000012583F85C50D4F86E10D4F87230E268CF
:106280005B1A07EE903AF8EEE77A0A2367EE887A0F
:106290002046C2ED167AD4F87220E16892FBF3F240
:1062A00000F0ECFCE36894F8D3255A70D4F876201B
:1062B00094F8D13507EE102AB8EE477A2B4384F8CC
:1062C000D13527EE087AE36883ED117AD4F87A2085
:1062D000E36807EE902AF8EE677A67EE887AC3EDF6
:1062E000127AE36883F85250E36883F85350E36806
:1062F00093F8543063B10DF05FFCD4F8CC35C01A7C
:10630000B0F5C87F40F23E82E368002283F8542053
:1063100094F8D135D9077FF514AC9A07C3F340053B
:106320007FF50FACD4F87C14D4F8802491427FF42C
:1063300008AC23F0030384F8D13520E4D4F86210CC
:106340002046FFF7A9F894F8D63523B1D4F8BC3528
:1063500043F0040375E794F86710E26811F0010F49
:106360000BD094F86630032B05D18A0700D504239F
:1063700084F8D335BBE7022BFAD0012384F8D33558
:106380005370B4E7002384F8D535D4F86210204662
:10639000FFF782F8E368B4F86E20DA85E368B4F8B2
:1063A0006C201A86A3E7D4F862102046FFF774F831
:1063B00094F8D635E2681BB1B4F86A30138196E7D9
:1063C00094F86D10CB0739D594F86C30032B33D18A
:1063D0008F0700D5042384F8D33594F8D5351BB145
:1063E000E368B4F88E20DA85E36894F8912083F8A6
:1063F000322094F8D335012B7FF679AFE5680DF0A4
:10640000DBFB2866E368D4F862205A60E368B4F8DE
:106410006A201A816BE700BFEE570308C1630308C7
:10642000D4630308DD630308E2630308010003206B
:106430006F12833AACC52737022BCCD0012384F8E6
:10644000D3355370C9E70125D4F8621084F8D655C6
:106450002046FFF721F8D4F86230C4F8C435C4F8F8
:106460008034E368D4F87A209A61E368D4F87E2017
:106470005A61E3681FED128A83F85C50D4F88210E9
:10648000D4F88630E2685B1A07EE903AF8EEE77AC5
:106490000A2367EE887A2046C2ED167AD4F8862061
:1064A000E16892FBF3F200F0E9FB94F87630052BFB
:1064B00000F2C380DFE803F0C1C1039FB8C1E36805
:1064C00002225A70E2681FED250A537884F8D3350A
:1064D00094F8D13543F0010384F8D135D4F88A30EB
:1064E00007EE903AF8EE677A012567EE887AC2EDFA
:1064F000117AD4F88E20E36807EE902AF8EE677AD6
:1065000067EE887AC3ED127AE36883F85250E36845
:1065100083F85350E36894F8792083F83220D4F854
:106520009E20D4F86230C4F87C3407EE902AF8EE4E
:10653000E77AE36867EE887AC3ED077AD4F8A23089
:10654000E66807EE903AF8EEE77A27EE800AF9F768
:106550000DFD86ED080AE36883F85050D4F89220C8
:10656000E36807EE902AF8EEE77A67EE887AC3EDE3
:106570000D7AD4F89620E36807EE902AF8EEE77AD1
:1065800067EE887AC3ED0E7AD4F89A20E36807EEB6
:10659000902AF8EEE77A67EE887AC3ED0F7AE3681F
:1065A00083F85150D4F8A620E36807EE902AF8EE5D
:1065B000677A27EE888A83ED108A94F8D13543F004
:1065C000020384F8D13594F8D5353BB1E368B4F8CB
:1065D000AE20DA85E368B4F8AE201A8694F87630F7
:1065E000012B03D9E5680DF0E7FA2866E368D4F8D3
:1065F00062205A607BE6E36803225A7094F8773091
:106600009E0742BFE36804225A7094F877305D0613
:1066100042BFE36805225A7094F97730002BBFF629
:1066200051AFE36806224CE794F8772059490620D9
:10663000F6F79CFAE368032243E7E3685D7041E7FD
:106640002046D4F86210FEF727FF94F86D309807C3
:106650007FF54DAEDAE694F8D63523B1D4F8BC35E3
:1066600043F01003EDE5D4F862109FED4B8A20460D
:10667000FEF712FFD4F87620D4F86230C4F87C34E8
:1066800007EE902AF8EE677AE3689FED440A67EE1A
:10669000887AC3ED077AD4F87A30E56807EE903A45
:1066A000F8EEE77A27EE800AF9F760FC85ED080A34
:1066B000E368012583F85050D4F86620E36807EEBC
:1066C000902AF8EEE77A204667EE887AC3ED0D7AD5
:1066D000D4F86A20E36807EE902AF8EEE77A67EECE
:1066E000887AC3ED0E7AD4F86E20E36807EE902A1C
:1066F000F8EEE77A67EE887AC3ED0F7AE16800F08A
:10670000D3F9E36883F85150D4F87E20E36807EEAC
:10671000902AF8EE677A67EE887AC3ED107A94F8DB
:10672000D13543F0020384F8D135E0E5D4F86210A6
:106730002046FEF7B1FE94F8672002F00702022A15
:1067400084F8C02513D8AAB1D4F8BC3523F400636B
:10675000C4F8BC35D4F8BC3523F40073C4F8BC3598
:106760003022002301212046FEF718FDBFE5D31E8D
:10677000012BEFD90A4B0B491B68986903681B680A
:106780009847E7E7D4F8C825D4F8C4359A427FF48F
:10679000D8A9BDE5FA6303080AD7233CACC527375F
:1067A000D81000200E6403082DE9F74304460DF0CD
:1067B00003FAD4F88C34B4F89424C31A93420546EF
:1067C00062D32046FFF73EF8D4F8BC35C4F88C54A9
:1067D0007BB3C823A4F89434606803685B69984766
:1067E000B0F5005F28BF4FF40050002785B2B846CF
:1067F0000826BBB29D4240F2DC80606803680DF160
:106800000701DB699847002800F0D3809DF8073026
:10681000002019464FEA032C4FF0060E94F874241A
:10682000082A3BD8DFE802F03F35454F607192AF50
:10683000B6004FF4FA63A4F89434A36893F92330B4
:10684000002BC9D094F87B24002AC5D194F8882461
:10685000042AC1D8D4F8840441F288322D1A954212
:10686000BAD9564A1268D26A92F89C20002AB3D14B
:10687000012B05D0022BAFD194F8D435002BABD02F
:106880002046FEF76BFDA7E7D4F8BC35002BA3D15B
:10689000D3E7622B04D1022384F874340137A8E7CC
:1068A000002284F87424B52BF8D194F874340133A1
:1068B000F2E7032284F8742484F87A3484F872347A
:1068C00084F87334EAE7042284F8742494F8722478
:1068D00094F8731484F875341A44D2B284F872248C
:1068E0000A4484F87324D9E7052284F8742494F8C0
:1068F0007224A4F87614134494F87324DBB284F859
:106900007234134484F87334C8E794F8722494F80A
:10691000739484F874E41A44D2B284F872244A441A
:1069200084F87324B4F87624624492B2B2F5826F8C
:10693000A4F8762404D9A4F8760484F874046DE7E6
:10694000A4F87804002AA9D10723A5E794F87224B3
:1069500094F873141A44D2B284F872240A4484F866
:106960007324B4F87824B2F5826F3CBF121982F810
:106970006230B4F87834B4F8762401339BB2A4F8CA
:1069800078349A4290E794F8722484F874649A42B6
:10699000D3D183E7002284F8742494F873249A42B4
:1069A0007FF47CAF2046FFF7B7F8002818BF804679
:1069B00074E7404603B0BDE8F08300BFD810002064
:1069C00037B5054640680191144668B103689B6A73
:1069D0009847A04208D9686801990368DB68224695
:1069E00003B0BDE83040184703B030BD10B50446D1
:1069F0000C4820600298C4E90332C4E90101642212
:106A00004FF4FA7104F1200000F0A0FCE2680023CA
:106A100082F85130E26882F85230E26882F85330EE
:106A2000204610BD9866030810B590F8443013B99D
:106A3000C368586810BD046D0CB9006CFAE7D0E962
:106A400012014FF47A720023F4F72EFA2044F1E792
:106A500038B52DED028BC568DFED127A95ED088A09
:106A600028EE278A0446B0EE480A18F031FAD5ED30
